:020000040800F2
:1000000000000110A5000408317502085588000899
:10001000A9010408A9010408A901040800000000BE
:10002000000000000000000000000000377502081A
:1000300035750208000000003375020885CC000801
:10004000A9010408A9010408A9010408A9010408D8
:10005000A9010408A90104081DC3020849C4020833
:100060000DC40208D1C3020895C30208B1FC0208FE
:10007000A1FC020891FC020881FC020871FC020844
:100080005DFC020849FC0208A9010408A901040852
:10009000A9010408A9010408A901040859C3020818
:1000A000A9010408A9010408A9010408A901040878
:1000B0001D9C00085D9B0008A9010408A901040813
:1000C000A9010408A9010408A9010408A901040858
:1000D000A901040845CE0008A9010408A9CD00081B
:1000E000E1C20208A901040815A90208A90104082F
:1000F00005990008A9010408D199000835FC0208F7
:10010000A9010408A90104089D9A0008A90104088E
:10011000A9010408A9010408A140020885400208B9
:1001200021FC02080DFC0208F9FB0208E5FB0208AD
:10013000D1FB0208A9010408A9010408A9010408C7
:10014000A9010408A9010408A901040849800208BA
:10015000BDFB0208A9FB020895FB02080DCD0008B3
:10016000A9010408A9010408A9010408A9010408B7
:10017000A9010408A9010408A9010408A9010408A7
:08018000A9010408A90104080B
:080188004CFC03000100000023
:1001900003123300C0320020B638002000000000F7
:1001A0002C06000825005A00F33200204C380020AD
:1001B0000000000000000000F6110C008C3600204A
:1001C000DC37002000000000600600081500700009
:1001D000983600206C37002000000000000000006E
:1001E0002A006000343100200C370020000000009D
:1001F000E99401082C0010007A360020A63800206F
:1002000000000000151701082B0024000D39002004
:10021000E938002000000000E5160108290064000C
:100220009C350020E837002000000000000000009E
:1002300014000200243500200837002000000000D0
:100240006C060008100003001435002078390020E7
:10025000000000006E060008280010000435002091
:100260007C39002000000000AD00010823001000D0
:100270000C2D00208C39002000000000C500010872
:1002800019000500FC3400209C390020000000000B
:1002900072060008F811010022310020A439002064
:1002A000000000007806000800010400F834002077
:1002B000A8390020000000007A06000802000C00A7
:1002C00038510020645100200000000000000000B0
:1002D000080209002C51002070510020000000008D
:1002E00025070308F7010600205100207C5100205B
:1002F000000000007E0600080A020A00B443002045
:10030000845100200000000084060008270004003B
:10031000F842002090510020000000008E060008E6
:10032000012008002041002094510020000000001E
:10033000920600081A000800603B00209C51002033
:10034000000000009A060008030001004841002058
:10035000A451002000000000000000001B00F40079
:10036000885B0020F06F0020000000009D5C030807
:100370000E02020004630020E47000200000000070
:10038000A20600082F001100BA6F0020E8700020BC
:1003900000000000A406000805100600E46F00201D
:1003A000FC70002000000000B6060008F5216E0079
:1003B000005B00200471002000000000D1590208F9
:1003C00026000E00847100207471002000000000DF
:1003D000A95902080B201000705B002094710020C6
:1003E00000000000BC0600081F101C00E05A00209E
:1003F000A471002000000000CC06000805020100E6
:10040000645F0020C071002000000000E8060008C2
:1004100003010A00265D0020C471002000000000D6
:10042000EA06000816000800A87C0020CC7C00200A
:1004300000000000F40600080101040024770020F9
:10044000F47C002000000000000000000C103000D0
:10045000A4800020388600200000000097A4010836
:100460000E20EA00947F0020688600200000000033
:100470008D95010813000400FC82002054870020A1
:1004800000000000FC060008020103007F7F00203E
:100490005887002000000000C9A4010809020100DB
:1004A0007C8500205C870020000000000007000819
:1004B00001020500167F0020608700200000000078
:1004C000F554030800020500FC7C0020688700202A
:1004D00000000000000000001E000400F880002062
:1004E00070870020000000000207000822000C00B6
:1004F0009C8400207487002000000000060700088C
:100500000400800020B4002038BD0020000000005E
:1005100000000000F901040010A90020B8BD00206F
:100520000000000011820008FD012400E8A800205E
:10053000BCBD002000000000A181000806001600DC
:10054000489C0020E0BD0020000000001D9A01082A
:10055000FB010100849B0020F8BD0020000000008A
:10056000E9060308FC010900509A0020FCBD0020A8
:1005700000000000F10603080A101A001C9A00206F
:1005800008BE002000000000120700083400100020
:10059000FC90002024BE00200000000011950108FE
:1005A00012200C00EC90002034BE0020000000005F
:1005B0002C07000818102C003C90002040BE0020A2
:1005C00000000000692E01080D0034006890002032
:1005D0006CBE00200000000075070308FA0102004D
:1005E00070890020A0BE002000000000F1BD0208BC
:1005F00002020300A4870020A4BE00200000000027
:10060000000000000C02010094870020A8BE00201A
:100610000000000038070008FE010900488900209A
:0C062000ACBE00200000000045070308ED
:10062C0000000000000000000000000000000000BE
:10063C0000000000000000000000000000000000AE
:10064C00000000000000000000000000000000009E
:10065C00000001000000000000000000000000008D
:10066C0003000001050000002801000004009001B7
:10067C00000039010000000000004A01B400D6015E
:10068C00000020030000E8036400040A00017E055A
:10069C00EA05B40532000000000000000000000074
:1006AC00000000000000000000002000030100001A
:1006BC002B21231E64010200000001000A01290005
:1006CC000000000000000100000005000000000018
:1006DC000000000000000000000000000000040109
:1006EC0001006C1600000000C40900001901282844
:1006FC0008040400370000000100C800141E0100AB
:10070C0064002C01280000300100005A0000000099
:10071C0090012C01C80064000200000000000000E1
:0D072C000000000100054B54563100000193
:10073900FF010100B4480408C48A0408000000004D
:1007490000000000C4480408CC4804080000000068
:1007590001200000D0480408D8480408000000001F
:1007690001400000DC4804087C5404080000000033
:1007790001200000E8480408F448040800000000CB
:1007890004000000F8480408387D0408000000004F
:100799000400000004490408607704080000000010
:1007A9000100000002010000010100000001010137
:1007B90000D60100A10B01080000000000000000A4
:1007C900FFFFFFFF010000000000803F0000000064
:1007D90000000000000000000000803F0000000051
:1007E9000000000000000000000000000000000000
:1007F90000000000000000000000000000000000F0
:100809000000803F00000000000000000000000020
:100819000000803F010000000000803F0000803F91
:10082900000000000000000000000000643104081E
:100839000508040000000000CC3E0408C033040889
:10084900B83E0408000000009031040805080A00B9
:1008590000000000CC3E0408C0330408D83D040859
:100869000000000004030904120100020202004012
:1008790083044057000201020301000009024300FA
:10088900020100C03209040000010202010005242E
:1008990000100105240100010424020205240600B8
:1008A90001070582030800FF09040100020A00008C
:1008B9000007050102400000070581024000000011
:1008C900FF00000000FFFF0000000000AA5505011D
:1008D9000000010000000101FFFF0000000000000E
:1008E9000102030401020304060708099B760208B2
:1008F900A17502087D770208154E02080B510208FE
:10090900254E0208414E0208EF4D0208E14D02084A
:1009190000000000000000002D202D2D202D2D2D80
:100929002D202D2D2D2D00000000000000000000BD
:1009390000000000000000AA550B010000AA55079D
:10094900010000AA55090200000000000100000092
:10095900C012AA5503009F00EC6D040800000000B6
:1009690000000000BD060308A08601000400000085
:10097900000000000000000000000000000000006E
:10098900000000000000000000000000D4830408FB
:100999003C6D04080000000095D301087D000000AB
:1009A9000600000000000000000000000000000038
:1009B900000000000000000000000000000000002E
:1009C900547D04080000000000000000358D000877
:1009D900E803000003000000000000000000000020
:1009E90000000000000000000000000000000000FE
:1009F900000000005C7D0408000000000000000009
:100A090091A5010810270000030000000000000064
:100A190000000000000000000000000000000000CD
:100A29000000000000000000687D040800000000CC
:100A390081140108A9A30008204E00000500000048
:100A4900000000000000000000000000000000009D
:100A5900000000000000000000000000846F04088E
:100A6900000000000000000031FB00081027000012
:100A7900010000000000000000000000000000006C
:100A8900000000000000000000000000000000005D
:100A99006C7D04080000000000000000458000088B
:100AA900E80300000500000000000000000000004D
:100AB900000000000000000000000000000000002D
:100AC90000000000787D040800000000000000001C
:100AD900190D0308204E000003000000000000006B
:100AE90000000000000000000000000000000000FD
:100AF9000000000000000000887D040800000000DC
:100B0900000000000D0B0308204E00000300000048
:100B190000000000000000000000000000000000CC
:100B2900000000000000000000000000987D04089B
:100B3900000000000000000029820008400D0300A9
:100B49000300000000000000000000000000000099
:100B5900000000000000000000000000000000008C
:100B6900B06E04080000000000000000151F030813
:100B79001027000001000000000000000000000034
:100B8900000000000000000000000000000000005C
:100B9900000000005C6D0408000000000000000077
:100BA900E58703081027000003000000000000008B
:100BB900000000000000000000000000000000002C
:100BC90000000000000000008C6F04080000000015
:100BD900000000009DCF0008A00F000001000000E8
:100BE90000000000000000000000000000000000FC
:100BF900000000000000000000000000A87D0408BB
:100C09000000000000000000596C020810270000D5
:100C190001000000000000000000000000000000CA
:100C290000000000000000000000000000000000BB
:100C3900B86E0408000000000000000085B2020838
:100C49001A4100000100000000000000000000003F
:100C5900000000000000000000000000000000008B
:100C690000000000E86F0408000000000000000018
:100C7900755602081027000001000000000000005E
:100C8900000000000000000000000000000000005B
:100C990000000000000000001C7D040800000000A6
:100CA90000000000D97603081A4100000100000085
:100CB900000000000000000000000000000000002B
:100CC900000000000000000000000000B47D0408DE
:100CD9000000000000000000DD610208400D030073
:100CE90000000000000000000000000000000000FB
:100CF90000000000000000000000000000000000EB
:100D0900BC7D04080000000000000000018000080C
:100D1900400D03000000000000000000000000007A
:100D290000000000000000000000000000000000BA
:100D390000000000C47D040800000000000000005D
:100D4900458E0308A0860100030000000000000092
:100D5900000000000000000000000000000000008A
:100D69000000000000000000D07D04080000000021
:100D790000000000D90A030840420F0000000000EB
:100D8900000000000000000000000000000000005A
:100D99000000000000000000000000000100000049
:100DA900FFFFFFFF010000005001000007000000E5
:100DB900020000000000000000000000010203041E
:100DC9000607080900000000E47C00200800000074
:100DD90000000000D47C002008000000E0010101AF
:100DE90001000000E1560308000000002808002067
:100DF90094890408000000000000000000000000C1
:100E090000000000C48A040800000000000000007F
:100E1900B408002004000000408904080D00000007
:100E290025710308BC200020000000004483040849
:100E39000D0000004D710308B020002000000000E3
:100E4900448404080800000000000000A4200020D9
:100E590004000000B08304080D0000009557030842
:100E690098200020000000005484040803000000BA
:100E79005D7303088C20002000000000A489040889
:100E8900030000005D7303088020002000000000BB
:100E9900AC80040801000000000000000000000010
:100EA90000000000000000000E000000000000002B
:100EB9000000000000000000948904080000000000
:100EC900000000000000000000000000C48A0408BF
:100ED9000000000000000000B40800200400000029
:100EE900EC88040803000000396F0308742000200F
:100EF90008000000B08304080D000000955703089E
:100F09009820002000000000548404080300000019
:100F19005D7303088C20002000000000A4890408E8
:100F2900030000005D73030880200020000000001A
:100F3900AC8004080100000000000000000000006F
:100F490000000000000000000E000000000000008A
:100F59000000000000000000AC8904080000000047
:100F6900000000000000000000000000C48A04081E
:100F79000000000000000000B40800200400000088
:100F8900F4880408030000005D730308C8200020EA
:100F990000000000AC80040801000000000000000F
:100FA9000000000000000000000000000E0000002A
:100FB9000000000000000000000000002070002078
:100FC900702D720008000000000000000000000001
:100FD900301C0020FFFFFFFFFA00000001000000A5
:100FE900010000002D202D2D202D2D2D2D202D2D02
:100FF9002D000000000000000000000000000000BB
:1010090000000000948004089C800408A48004085F
:1010190000000000000000000000000000000000C7
:101029005880040804000000AF6E030800000000A7
:1010390000000000AC80040801000000000000006E
:101049000000000000000000000000000E00000089
:101059000000000000000000000000007E5E00208B
:101069000100C409000000007C5E00200100C409E1
:10107900000000007A5E00200100C40900000000A1
:10108900785E00200100C40900000000745E0020A1
:101099000100C40900000000765E00200100C409B7
:1010A90000000000725E00200100C4090000000079
:1010B900705E00200100C40900000000287F0020A4
:1010C9000100C80001000000267F002032003075B1
:1010D90032000000247F0020055A0500217F0020EE
:1010E90000FF0100237F002001000000D408002038
:1010F9001F7F002002000000B0340408207F002078
:1011090000FF0100227F002001000000D408002018
:101119001E7F002002000000B03404080000000017
:1011290000000000DC080020205F00209CFF2C014B
:1011390000000000AE0600200A000000D83D0408A7
:101149000C7F0020E0150C1700000000B0060020FD
:1011590008000000C0330408AF06002005000000A5
:10116900CC3E04080E7F002002000000F03D040878
:10117900E88000200100FF7F01000000E7800020D7
:1011890002000000FC3D0408887F002003000000E5
:101199000C3E0408877F0020030000000C3E040871
:1011A900868000200000F4010100000084800020F6
:1011B9000000F40101000000828000200000F40119
:1011C90001000000808000200000F40101000000FF
:1011D9007E80002000FF0100A2800020E803D007E4
:1011E9000A000000A0800020006401000A0000003D
:1011F90095800020006401009480002000640100B3
:101209009C800020006401000A0000009B800020EF
:10121900006401000A0000009A80002000640100B7
:101229000A0000009F800020006401000A000000FD
:101239009E800020006401000A0000009D800020BB
:10124900006401000A0000009980002000FF0100ED
:101259000A0000009880002000FF01000A00000039
:101269009780002000FF01000A000000907F002005
:101279000000F401010000008E7F00200000F4014D
:10128900010000008C7F00200000F4010100000033
:101299008A7F00200000F4010100000090800020F6
:1012A9001400E803010000008E800020E803307577
:1012B900010000008D80002000C801008C80002002
:1012C90000C801008B80002000C801008A8000202E
:1012D900016401000A0000008980002000FF01006C
:1012E9000A000000DD80002000C80100DC80002029
:1012F90000C80100DB80002000C80100DA8000205E
:1013090000C80100D980002000C80100D880002051
:1013190000C80100D780002000C80100D680002045
:1013290000C80100D580002000C80100DC80040845
:1013390000000000000000000000000000000000A4
:10134900EC8004080900000000000000800900206A
:1013590004000000F48004080900000000000000F7
:101369007409002004000000C48604080900000074
:101379000000000068090020040000007848040803
:1013890009000000000000005C09002004000000C2
:10139900FC8004080900000000000000500900203A
:1013A9000400000004810408090000000000000096
:1013B90044090020040000000C8104080900000011
:1013C900000000003809002004000000148104080E
:1013D90009000000000000002C09002004000000A2
:1013E900AC800408010000000000000000000000BB
:1013F90000000000000000000E00000000000000D6
:10140900000000000000000038820408000000000D
:10141900000000000000000000000000A06D0408AA
:101429000700000000000000A409002000000000DF
:101439004882040808000000000000009809002004
:1014490000000000548204080800000000000000A9
:101459008C09002000000000AC8004080100000095
:101469000000000000000000000000000000000073
:101479000E00000000000000000000000000000055
:101489005C82040800000000000000000000000069
:10149900000000006C8204080D000000000000003C
:1014A900E009002000000000748204080D0000001B
:1014B90000000000D4090020000000007C8204081C
:1014C9000700000000000000CC0900200000000017
:1014D900848204080D00000000000000C0090020FB
:1014E900000000008C8204080D00000000000000CC
:1014F900B4090020000000009482040807000000DD
:1015090000000000AC09002000000000AC800408C5
:1015190001000000000000000000000000000000C1
:10152900000000000E0000000000000000000000A4
:10153900000000009C820408000000000000000078
:101549000000000000000000A06D04080C0000006D
:10155900000000002A7F002000000000B08204087B
:101569000C000000000000002C7F0020000000009B
:10157900C08204080C00000000000000627F002007
:1015890000000000D08204080C00000000000000E8
:10159900567F002000000000E48204080C000000CF
:1015A900000000002E7F002000000000947E040847
:1015B9000C00000000000000307F00200000000047
:1015C900F08204080C00000000000000327F0020B7
:1015D90000000000048304080C0000000000000063
:1015E900347F0020000000000C8304080C00000078
:1015F90000000000367F002000000000148304086A
:101609000C00000000000000747F002000000000B2
:101619002C8304080C00000000000000387F002023
:1016290000000000388304080C00000000000000DE
:101639003A7F002000000000DC7C04080C00000058
:10164900000000003C7F00200000000040830408E7
:101659000C000000000000003E7F00200000000098
:101669004C8304080C00000000000000407F0020AB
:1016790000000000588304080C000000000000006E
:10168900427F002000000000648304080C00000071
:1016990000000000447F002000000000708304085F
:1016A9000C00000000000000467F00200000000040
:1016B9007C8304080C000000000000005A7F002011
:1016C90000000000848304080C00000000000000F2
:1016D900587F0020000000008C8304080C000000E3
:1016E90000000000667F00200000000098830408C5
:1016F9000C00000000000000687F002000000000CE
:10170900A48304080C000000000000006E7F002084
:1017190000000000A48104080C0000000000000083
:10172900487F002000000000B08304080C0000007E
:1017390000000000507F002000000000B88304086A
:101749000C000000000000004A7F0020000000009B
:10175900C48304080C000000000000004C7F002036
:1017690000000000D08304080C0000000000000005
:101779004E7F002000000000D88304080C00000000
:1017890000000000527F002000000000C06D040826
:101799000C000000000000005C7F00200000000039
:1017A900E48304080C00000000000000547F0020BE
:1017B90000000000F08304080C0000000000000095
:1017C900647F002000000000FC8304080C00000076
:1017D900000000005E7F002000000000048404086F
:1017E9000C00000000000000607F002000000000E5
:1017F9000C8404080C000000000000006A7F00202F
:1018090000000000148404080C000000000000001F
:101819006C7F002000000000AC800408010000007B
:1018290000000000000000000000000000000000AF
:101839000E00000000000000000000000000000091
:101849001C840408000000000000000000000000E3
:10185900000000002C8404080500000000000000BE
:10186900867F002000000000AC8004080100000011
:10187900000000000000000000000000000000005F
:101889000E00000000000000000000000000000041
:10189900348404080000000000000000000000007B
:1018A90000000000C48A04080000000000000000D5
:1018B900E801002004000000408404080D00000035
:1018C900116F0308340A0020000000004089040851
:1018D9000D00000099560308280A002000000000A6
:1018E900448304080D0000007D5603081C0A0020EB
:1018F9000000000044840408080000000000000003
:10190900100A002004000000B08304080D00000044
:10191900C7550308040A0020000000004C8404088D
:101929000900000000000000F80900200400000080
:1019390054840408030000005D730308EC090020C7
:1019490000000000AC800408010000000000000055
:101959000000000000000000000000000E00000070
:101969000000000000000000000000005884040886
:10197900000000000000000000000000000000005E
:10198900688404080D000000000000004C0A0020D3
:1019990000000000708404080A0000000000000034
:1019A900B1830020000000007C8404080A000000C4
:1019B90000000000B98300200000000084840408AE
:1019C9000A00000000000000C183002000000000A0
:1019D9008C8404080800000000000000400A002070
:1019E900000000009484040804000000F574030852
:1019F9000000000000000000AC80040801000000A5
:101A090000000000000000000000000000000000CD
:101A19000E000000000000000000000000000000AF
:101A2900A08404080000000000000000000000007D
:101A390000000000B48404080D000000000000004C
:101A4900640A002000000000C484040804000000A7
:101A5900997103080000000000000000CC8404080C
:101A69000D00000000000000580A002000000000DE
:101A7900E0840408040000007571030800000000F8
:101A890000000000AC800408010000000000000014
:101A99000000000000000000000000000E0000002F
:101AA900000000000000000000000000E8840408B5
:101AB900000000000000000000000000000000001D
:101AC900FC8404080700000000000000A00A0020B0
:101AD900000000000885040808000000000000005C
:101AE900940A002000000000148504080800000082
:101AF90000000000880A002000000000208504087A
:101B090008000000000000007C0A0020000000001E
:101B19002C8504080800000000000000700A00205D
:101B290000000000AC800408010000000000000073
:101B39000000000000000000000000000E0000008E
:101B490000000000000000000000000038850408C3
:101B590000000000000000008F08002000000000C5
:101B6900448504080B00000000000000300B002031
:101B790000000000508504080B0000000000000070
:101B8900240B0020000000005C8504080B00000005
:101B990000000000180B0020000000006885040800
:101BA9000B000000000000000C0B002000000000EA
:101BB900748504080B00000000000000000B0020E1
:101BC90000000000808504080B00000000000000F0
:101BD900F40A0020000000008C8504080B000000B6
:101BE90000000000E80A00200000000098850408B1
:101BF9000B00000000000000DC0A002000000000CB
:101C0900A48504080B00000000000000D00A002091
:101C190000000000B0850408070000000000000073
:101C2900C80A002000000000B88504080700000069
:101C390000000000C00A002000000000C48504085C
:101C49000B00000000000000B40A002000000000A2
:101C5900D08504080800000000000000A80A002040
:101C690000000000AC800408010000000000000032
:101C79000000000000000000000000000E0000004D
:101C8900000000000000000000000000DC850408DE
:101C9900000000000000000000000000000000003B
:101CA900F08504080800000000000000600B002017
:101CB90000000000FC850408080000000000000086
:101CC900540B0020000000000886040808000000EA
:101CD90000000000480B00200000000014860408E2
:101CE90008000000000000003C0B0020000000007C
:101CF900AC800408010000000000000000000000A2
:101D090000000000000000000E00000000000000BC
:101D190000000000000000001C860408000000000C
:101D2900000000008C080020000000002C86040838
:101D39000B00000000000000A80B002000000000BC
:101D4900388604080B000000000000009C0B0020EE
:101D5900000000004486040807000000000000009D
:101D6900940B0020000000005086040807000000C2
:101D7900000000008C0B0020000000005C860408B5
:101D89000700000000000000840B00200000000094
:101D9900688604080800000000000000780B002095
:101DA9000000000070860408080000000000000020
:101DB9006C0B002000000000AC800408010000004A
:101DC900000000000000000000000000000000000A
:101DD9000E000000000000000000000000000000EC
:101DE9007886040800000000000000008C0800202C
:101DF90000000000848604080700000000000000BD
:101E0900F40B0020000000008C8604080700000085
:101E190000000000EC0B002000000000948604087C
:101E29000700000000000000E40B00200000000093
:101E3900404804080700000000000000DC0B0020F7
:101E490000000000484804080700000000000000E6
:101E5900D40B0020000000005048040807000000CF
:101E690000000000CC0B0020000000009C86040844
:101E79000700000000000000C40B00200000000063
:101E8900A48604080700000000000000BC0B002025
:101E990000000000AC8604080700000000000000F4
:101EA900B40B002000000000AC8004080100000011
:101EB9000000000000000000000000000000000019
:101EC9000E000000000000000000000000000000FB
:101ED9000000000099590308FC0B0020847F0020B2
:101EE9001B0000001C3E0408837F00200A32010009
:101EF900827F002001FA01007E7F002000C80100D6
:101F09007C7F0020E803D007010000004B414B55BE
:101F190054454634000000001D7F002000030100E5
:101F29001C7F002000030100B958030891580308D9
:101F3900D80C00204D58030801580308500D002003
:101F4900F9580308E1580308040E0020AF590308A3
:101F5900D965030810110020055603080000000088
:101F690060110020D1740308195C03083C12002099
:101F7900D559030800000000F0120020795A03081F
:101F8900495A03087C130020055B0308495B0308D1
:101F99001C1400209280002001030100155A030837
:101FA900E95903085C150020A95A0308BD71030803
:101FB900E8150020755B030819720308B0160020A4
:101FC9008880002001030100B48604080000000095
:101FD900000000000000000000000000C0860408A6
:101FE9000800000000000000D017002000000000D9
:101FF900C88604080700000000000000C817002078
:1020090000000000D8860408070000000000000056
:10201900C017002000000000E48604080700000043
:1020290000000000B817002000000000F086040836
:102039000D00000000000000AC17002000000000A7
:10204900FC860408030000005D730308A017002044
:1020590000000000AC80040801000000000000003E
:102069000000000000000000000000000E00000059
:1020790000000000000000000000000004870408C0
:102089000000000000000000000000000000000047
:10209900148704080A00000000000000687E040894
:1020A900000000001C8704080A000000000000006E
:1020B9001047040800000000248704080A000000F3
:1020C90000000000DE800020000000002C870408CA
:1020D9000A00000000000000DC17002000000000DA
:1020E900AC800408010000000000000000000000AE
:1020F90000000000000000000E00000000000000C9
:1021090000000000000000003487040800000000FF
:1021190000000000000000000000000040870408E3
:10212900030000005D730308101800200000000080
:102139004C870408030000005D730308041800209D
:102149000000000054870408030000005D730308C1
:10215900F8170020000000005C8704080500000053
:10216900000000001B7F00200000000064870408B5
:102179000700000000000000F01700200000000028
:10218900708704080700000000000000E81700201D
:1021990000000000AC8004080100000000000000FD
:1021A9000000000000000000000000000E00000018
:1021B9000000000000000000000000007C87040807
:1021C9000000000000000000000000000000000006
:1021D900487F0408030000005D73030834180020D9
:1021E9000000000090870408030000005D730308E5
:1021F900B4060020000000009887040803000000CE
:102209005D7303082818002000000000A087040857
:10221900030000005D7303081C1800200000000083
:10222900AC8004080100000000000000000000006C
:1022390000000000000000000E0000000000000087
:102249000000000000000000AC8704080000000046
:10225900000000000000000000000000B88704082A
:1022690007000000657203089018002000000000B4
:10227900D4830408030000005D7303088418002058
:1022890000000000C4870408030000005D73030810
:102299007818002000000000CC8704080300000023
:1022A9005D7303086C18002000000000D48704083F
:1022B90007000000497203086418002000000000AC
:1022C900D4470408030000005D7303085818002070
:1022D90000000000E0870408030000005D730308A4
:1022E9004C18002000000000EC87040803000000DF
:1022F9005D7303084018002000000000AC8004084A
:1023090001000000000000000000000000000000C3
:10231900000000000E0000000000000000000000A6
:1023290000000000555903081159030898180020A6
:10233900E55B0308000000004C190020DD57030885
:10234900B9570308D8190020000000000000000058
:102359008C1A0020BD5B030881720308181B00203A
:10236900F8870408000000000000000000000000D9
:102379000000000004880408030000005D730308DE
:10238900241C0020000000000C8804080300000041
:102399005D730308181C002000000000B86E0408D3
:1023A900030000005D7303080C1C002000000000FE
:1023B90018880408030000005D730308001C00204E
:1023C9000000000024880408030000005D7303086E
:1023D900F41B0020000000002C8804080200000003
:1023E900417503080000000000000000348804085B
:1023F9000200000041750308010000000000000010
:10240900408804080200000041750308020000002A
:1024190000000000000000000E00000000000000A5
:102429000000000000000000127F002088136F17D1
:1024390001000000147F002088136F1700000000BE
:102449004C880408000000000000000000000000A3
:10245900000000005C88040808000000000000007B
:10246900041D00200400000068880408080000001A
:1024790000000000F81C002000000000548404083B
:1024890004000000796F030800000000000000004C
:10249900AC800408010000000000000000000000FA
:1024A90000000000000000000E0000000000000015
:1024B9000000000000000000107F002088136F1743
:1024C900010000005C5F002088136F170000000006
:1024D9004957030800000000101D00205483002004
:1024E900010000008C3E04085E5F0020010000002E
:1024F900983E0408545F002002000000A03E040832
:10250900F6B400200000000000000000F4B4002030
:102519000000000000000000F2B4002000000000EC
:1025290000000000F0B400200000000000000000DE
:10253900EEB400200000000000000000ECB4002010
:102549000000000000000000200200200000000040
:10255900000000000F7F002002000000AC3E0408CC
:10256900A48804080000000000000000000000002A
:10257900000000005C88040808000000000000005A
:10258900941D002004000000688804080800000069
:1025990000000000881D0020000000005484040889
:1025A90004000000195703080000000000000000A3
:1025B900AC800408010000000000000000000000D9
:1025C90000000000000000000E00000000000000F4
:1025D9000000000000000000B488040800000000AA
:1025E900000000000000000000000000C48804088A
:1025F9000D000000C9700308C41D0020040000007C
:10260900D08804080D00000071570308B81D002088
:1026190004000000DC8804080D0000008D70030828
:10262900AC1D002000000000E88804080300000039
:10263900596F0308A01D002008000000F488040851
:10264900030000005D730308C8200020000000009B
:10265900AC80040801000000000000000000000038
:1026690000000000000000000E0000000000000053
:102679000000000000000000A48004080000000021
:10268900000000000000000000000000588004085D
:1026990004000000916F0308000000000000000022
:1026A900AC800408010000000000000000000000E8
:1026B90000000000000000000E0000000000000003
:1026C9000000000000000000488904080000000024
:1026D9000000000000000000000000007C700408F9
:1026E9000D00000000000000241E0020040000006E
:1026F900588904080800000000000000181E002086
:1027090004000000648904080800000000000000BB
:102719000C1E0020040000006C8904080800000059
:1027290000000000001E0020040000007489040855
:102739000800000000000000F41D00200400000053
:102749007C8904080800000000000000E81D002042
:10275900040000008489040808000000000000004B
:10276900DC1D0020040000008C890408080000001A
:1027790000000000D01D002004000000AC80040807
:10278900010000000000000000000000000000003F
:10279900000000000E000000000000000000000022
:1027A900000000003157030800000000301E00201F
:1027B9000000000000000000A81E0020000000002A
:1027C90000000000481F00205A5F0020040000009C
:1027D900B83E0408585F0020E0150C1700000000FF
:1027E900575F002008000000C0330408565F00202E
:1027F90005000000CC3E04080000000000000000B5
:10280900981F00200800000000600240106002408C
:1028190000000000000B0000000020000000000084
:102829000000000000600240286002400000000033
:10283900060C00000000200000000000000000005D
:10284900006002404060024000000000100D0000DE
:1028590000002000000000000000000000600240AD
:102869005860024000000000160E00000000200021
:10287900000000000000000000600240706002409B
:1028890000000000200F00000000200000000000F0
:102899000000000000600240886002400000000063
:1028A90026100000000020000000000000000000C9
:1028B90000600240A06002400000000030110000EA
:1028C900000020000000000000000000006002403D
:1028D900B860024000000000362F00000000200010
:1028E9000000000000000000006402401064024083
:1028F9000000000000380000000040000000000057
:10290900000000000064024028640240000000004A
:10291900063900000000400000000000000000002F
:10292900006402404064024000000000103A0000C8
:1029390000004000000000000000000000640240A8
:102949005864024000000000163B000000004000EF
:1029590000000000000000000064024070640240B2
:1029690000000000203C00000000400000000000C2
:10297900000000000064024088640240000000007A
:102989002644000000004000000000000000000094
:1029990000640240A06402400000000030450000CD
:1029A9000000400000000000000000000064024038
:1029B900B8640240000000003646000000004000F4
:1029C90000000000000000000000000100000000FD
:1029D900000000000000000055530208775002086B
:1029E900655F020800000000BD4D02083D52020863
:1029F900275302089F510208000000000000000050
:102A0900B14D0208954D0208934D0208914D0208F7
:102A19008B4D0208894D02088F4D02088D4D020821
:102A2900A54D0208974D02083D5F0208515F020853
:102A3900295F0208155F0208015F02080100000012
:102A49000000803F18230020000000000000000063
:102A5900000000000000000000000000000000006D
:102A6900000000000000000000000000000000005D
:102A7900000000000000000000000000000000004D
:102A8900000000000000000000000000000000003D
:102A9900000000000000000000000000000000002D
:102AA90000000000000000004300000000000000DA
:102AB900000000000000000000000000000000000D
:102AC90000000000000000004300000000000000BA
:102AD90000000000000000000000000000000000ED
:102AE900000000000000000043000000000000009A
:102AF90000000000000000000000000000000000CD
:102B09000000000000000000430000000000000079
:102B190000000000000000000000000000000000AC
:102B29000000000000000000430000000000000059
:102B3900000000000000000000000000000000008C
:102B49000000000000000000430000000000000039
:102B5900000000000000000000000000000000006C
:102B69000000000000000000430000000000000019
:102B7900000000000000000000000000000000004C
:102B890000000000000000007B0504085705040848
:102B990000000000DD8A0408548004084A4E040835
:102BA9004A4E04084A4E04084A4E04084A4E04088C
:102BB9004A4E04084A4E04084A4E04084A4E04087C
:102BC900FFFFFFFFFFFFFFFFFFFFFFFFFFFF00000A
:102BD9000100415343494900000000000000000082
:102BE90000000000000000000000000000000000DC
:102BF9000000415343494900000000000000000063
:102C090000000000000000000000000000000000BB
:082C19000000000001000000B2
:108000000C4B1B78DB0700D570470B4A1368002B1D
:10801000FAD04FF47A7101FB03F39842F4D3074B83
:108020001B781BB9064B99681B690B600023136012
:10803000704700BF045D0020C0430020B44300200F
:10804000A043002038B50B4C23688BB15A68821AC4
:10805000002A054604DA0BE05A68AA1A002A07DB50
:108060009A68226018461A6890472368002BF3D15B
:1080700038BD00BFF4300020436A8269D154436A9E
:108080000169826B01338B4228BF00234362DAB15E
:10809000EFF31183502282F31288826B1168C907B3
:1080A0000ED470B45468FCB9D0E909518D4211D195
:1080B000012280F85C20DBB283F3118870BC70472A
:1080C000DBB283F311887047826DD36843F080037D
:1080D000D360704786690E44D6600ED9691A516024
:1080E0008562002180F85C10116841F00101DBB26B
:1080F000116083F3118870BC70470569691A51607B
:108100008462EEE7034610B4446BD968406954B109
:10811000DA6C8C1A013A005D5DF8044B08BF0A4620
:10812000C0B2DA6470471A6A805C01328A4228BFA2
:108130002246C0B21A625DF8044B7047836B13B1DC
:1081400090F85C007047D0E90903181AB0FA80F083
:1081500040097047D0E909120369914238BFC91834
:108160008A1A816B013B19B149680A449A4201D2CB
:10817000981A704700207047436B43B1C26C5B682C
:108180009A4291BF981AC0689B1AC0187047D0E9EC
:1081900007239A422FBFD01AC0688018C01A7047B0
:1081A0000A4B30B503F1140493F900205D78072AD7
:1081B000C8BF143A811804330D7313F8025C855458
:1081C00013F8012C0A769C42EED130BDDC10040875
:1081D00003682DE9F041DD691DB12B46BDE8F04192
:1081E0001847002A174611DD04460E460F4400E0EA
:1081F00023689B68204698470028F9D0236816F822
:10820000011B1B6820469847BE42F1D1BDE8F081B2
:1082100010B424212524262200230470417082708A
:10822000C3705DF8044B70472DE9F0478C4A8D4BC5
:1082300012781C78D207064648D58B4D012C00F0E9
:1082400091801ED3022C40F09B808849884A09887F
:108250001288884F914201D901241C70EB7AFBB13E
:108260002B89EBB1844B1B78D3B11BF061FF002845
:1082700000F0E2802B7B83422CBF012300233B7064
:108280000FE0DFF8E8C17B4F7C4CBCF8000022888F
:10829000697B521A8242DFDAEB7A0024002BDFD1AD
:1082A0003B782A79632A07D87549022C087800F0B0
:1082B000B880002840F0A0807249AA7A9C4238BF5A
:1082C0001C460C70002A44D1BDE8F087DFF89CC141
:1082D000654DBCF80000BCF8021095F803E06A4F49
:1082E000411A0029A4F10302B8BF4942704597F82A
:1082F0000080D2B211D32F7887420ED3012A45D9FC
:10830000B8F1020F9AD15C48604A00789080022947
:10831000CCBF00210121D18090E7B0EB4E0FEDDC06
:10832000012A40F28C800229EADC0324514F524892
:1083300052494F4A1C70B8F1020F4FF000033C70D5
:1083400003700B80138089D1504A01219380D18022
:1083500084E7012C6BD0022CB6D10720BDE8F04792
:1083600029F098BD424A41491288687B0988121A4F
:10837000914207DD414A12888A423CBF00241C70AA
:108380003C4F6BE702241C703A4F67E70229B7DCC9
:1083900095F800E090FBFEFE0EF1010EBEF1080F15
:1083A000DFF8D4A0AA786978DFF8C490334C314F55
:1083B000A8BF4FF0080E8AF800E01FFA8EFA11FBF2
:1083C0000AF112FB0AF2DFF8B8A0A9F8001092B285
:1083D00000214FF06409B8F1020F22803970197042
:1083E000CAF804108AF801907FF452AF274A01219D
:1083F000A2F804E0D18048E74868301A244EB04221
:10840000C8BF4A703FF758AFC2F16402214E00FB6B
:1084100002F086FB0062C017A0EBA25064304870E7
:108420004AE70028E8D101274E600F70ECE70820EA
:10843000BDE8F04729F02EBD02233B7031E7032C45
:108440007FF471AFB8F1020F9AD10B4A0F4B12783B
:108450009A800229CCBF00210121D980054FFDE679
:10846000045D00207A760020705B0020445D0020CF
:108470007E760020D87600204A5D00207C760020A1
:10848000807600206E5B0020958700209887002072
:108490007F9698006BCA5F6B30B50446806D617142
:1084A0008389A26823F400531B041B0C838185B0CD
:1084B000A379009213F0040F4FEA03324FEA03232B
:1084C0000CBF00254FF4805503F4806302F4005282
:1084D000ADF80450ADF80830002511F00103ADF8F7
:1084E0000620ADF80C501ED1ADF80A3008238D07D8
:1084F000694648BFADF80A3020F00AF9A279A36DA9
:10850000D10715D412F0080F9A8A05BF22F008028D
:10851000120442F00802120C9A829A8942F4005224
:108520009A8105B030BD0423ADF80A300C23DEE794
:108530000A498B4210D0A1F548418B4205D001F584
:108540004C418B42DED1052000E00220012127F0C2
:10855000F7FAA279A36DD5E70020F7E700100140F4
:1085600030B50446806DA160838923F400531B0459
:108570001B0C838185B0A379009113F0040F6179FE
:108580004FEA03324FEA032303F48063ADF8083067
:108590000CBF00254FF48055CB0748BF0423ADF82E
:1085A00004504FF00005ADF80A5002F400524ABFE3
:1085B000ADF80A3008230C23ADF80C508D0769463E
:1085C00048BFADF80A30ADF8062020F0A1F8A27936
:1085D000A36DD10710D412F0080F9A8A05BF22F0BC
:1085E0000802120442F00802120C9A829A8942F49C
:1085F00000529A8105B030BD0A498B4210D0A1F5D6
:1086000048418B4205D001F54C418B42E3D1052016
:1086100000E00220012127F093FAA279A36DDAE7A6
:108620000020F7E700100140604B614870B5582208
:10863000012500211D7037F0DBFF5E4A5E495F4C6B
:108640005F4800230B60136028F040FD2946052099
:1086500028F08AFD6579291C4FF0070018BF012119
:1086600028F082FDA679311C4FF0080018BF0121C7
:1086700028F07AFDA37A002B6FD0524C002D76D1D2
:10868000311C18BF0121504E092028F06DFD3168C2
:10869000CA077CD44A4D11F002016AD1003118BFDB
:1086A0000121032028F060FD484A494B128E93FBBC
:1086B000F2F301210420C5F8143128F055FD454B93
:1086C0000620197828F050FD01210A2028F04CFDE1
:1086D00021680B20C1F3C01128F046FD21680C2051
:1086E000C1F3802128F040FD21684B0508D53A4BA5
:1086F0001B7A083B012B9CBF4FF4FA63C5F880320C
:10870000C1F300410D2028F02FFD21680E20C1F398
:10871000804128F029FD21680F20C1F3C06128F0B5
:1087200023FD0121142028F01FFD0121102028F035
:108730001BFD0121112028F017FD0121122028F036
:1087400013FD4FF4804029F0A9FA011C18BF012144
:108750001320BDE8704028F007BDE37A194C002BC8
:108760008CD1216811F480218DD0002D88D0012179
:1087700089E70121022028F0F7FC184B31685B6A79
:108780000A2BB8BF0A2301F00201AB6786E7144B3E
:108790000B4D1B680A2B4FF00101B8BF0A23084696
:1087A0006B6428F0E1FC316875E700BF8C7700202E
:1087B000347700209077002030770020705B002015
:1087C00028020020489A00209C5D0020689000202C
:1087D00040420F00003600203C9000205C5D0020ED
:1087E000389A002010B40B4B0B4A1C7801238340AD
:1087F000234052F8200031B9B3FA83F149095DF8FA
:10880000044B23F05BBD191C18BF01215DF8044B1C
:1088100023F054BD9C900020A0900020022828BF87
:10882000022010B4084C094B207000EB8002C0EB12
:10883000C20207495DF8044B013003EB4203C0B2AA
:108840000B6029F043BC00BFEC900020947F002017
:108850005461002008B501210220FFF7C3FF094B36
:108860001B7803F00503052B08D000210120FFF73A
:10887000B9FF00210846FFF7B5FFFEE714F068F8DE
:10888000F3E700BF0451002008B50EF07DF826F094
:108890000DFEBDE808400EF01DB800BF3F4B5A89E1
:1088A0009989914210B524BF00225A81198ADA8928
:1088B000914224BF0022DA81D978394A92F85020B7
:1088C00081B107290ED0374C012000210A2A2070DF
:1088D0009870D97159D00C2A01D00A2A5BD0DFEDEB
:1088E000327A0AE00A2AD97952D0DFED307A9FED48
:1088F000307A0C2A18BFF0EE477A9FED2E7A0029C5
:1089000018BFF0EE477A2C4CA278062A97BF2B4965
:10891000DFED286A01EB8201D1ED056A217971B1A1
:10892000013A032A0AD8B7EE000A80EE260A38F088
:108930003BF82388984228BF1846208010BD9B78BA
:10894000184907EE103A0A78B8EEC77A67EE277A28
:1089500007EE102AB8EEC77A27EE277AF4EEC76A38
:10896000F1EE10FAEADD86EEA77AFDEEC77A17EE91
:10897000903A102BA8BF1023012BB8BF0123DBB204
:108980009A4238BF1A460A7010BDDFED0D7ABAE779
:10899000DFED0C7AB1E7DFED0A7AAEE71C9A002032
:1089A000CC910020223100206F12833A0AD7A339DC
:1089B0006F1203396F120338489C0020DC10040842
:1089C0000F506E3A5304E9382DE9F84F0DF0DCFFF3
:1089D000DFF83C83B04B434525D2DFF83893AF4FE7
:1089E00003F114069A464C462588621985B1BA42AD
:1089F0000ED2052D0CD936F8143C6188C3F30B0355
:108A0000994200F0E280144625886219002DEED1CB
:108A100056F8101C50460AF1140A28F0D7FBC2453C
:108A200006F11406DFD39E4A1378A3F11701022939
:108A30000FD99C4911F83300002840F01F81D8005D
:108A40000144497829B1984911F833300BB91823FA
:108A50001370964B5A78022A00F2DE8094499548AA
:108A600001EB02111A780160022A00F2DE8002EBAB
:108A70008201914BC2EBC10203EB4203998C5A8CE9
:108A80008E4C9142236001D300225A848C4B9A78F9
:108A9000042A00F0D08032B91A88B2F5F07F84BF82
:108AA0004FF4F0721A80874DFFF7F8FE2B68864A64
:108AB0001A40002A00F0EB80D80700F1CC8059045E
:108AC00000F1D0801A0700F1D4809B0400F1BC8033
:108AD00032F0B2FE10B97D4827F04CFE4FF4007022
:108AE00024F026FD4FF4003024F022FD4FF4001056
:108AF00024F01EFD4FF0007024F01AFD4FF080604E
:108B000024F016FD19F0BCFD00213022704837F02A
:108B10006FFD206813F060FB6E4B256803F1640164
:108B200003E00533994200F084801A78002AF8D1D6
:108B30009C78D8788442F4D2674B654C1A702846EA
:108B4000256330F0B9FB654A654B1079654A62636D
:108B50006421C82211FB00210022C3E90112C3E9EC
:108B60000322C3E90522DA6183F8202083F821205B
:108B70000DF068FD5C4B9FED5D5A1B885C4A9FEDD4
:108B80005D6A50795C4906EE903AF8EEE66A138821
:108B9000C5EE265A07EE103A53881279C1ED005AF5
:108BA00007EE903AB8EEC77AF8EEE77A534B27EE25
:108BB000067A67EE867A18725A7283ED017AC3EDEF
:108BC000007ABDE8F84F0DF085BE63799B077FF40E
:108BD0001AAF56F8101C94F804B0504628F0F6FA74
:108BE00036F8143CBBEB133F07D00AF1140AC24518
:108BF00006F11406FFF4F7AE15E736F8123C56F806
:108C0000100CAA1FC3F30B039A4204F10601A8BF7C
:108C10001A4637F0D3FBE8E700225A701A78254845
:108C200023490160022A7FF622AF00221A70224BEC
:108C300024E7012280E79A8AB2F57A7FBFF433AF46
:108C40004FF47A729A822EE72D4824F071FC40206E
:108C500024F06EFC3CE72B4824F06AFC2B68590496
:108C60007FF530AF284824F063FC2B681A077FF5A6
:108C70002CAF264824F05CFC2B6826E7D8000C18A3
:108C80006468002C7FF4DCAE17241470D8E643F03F
:108C900008032B6010E700BF900100080080000867
:108CA00024350020FC400408EC2C0408EC90002043
:108CB000A480002058610020947F0020546100208F
:108CC000489C0020FC82002009600002689000207F
:108CD000E82400209C350020E400002020410020F2
:108CE000A85E0020122D0020F8420020C0C9FB48D9
:108CF000A87C002017B7D138FC4200209C3B002004
:108D00000940000208600002092000020160000220
:108D10002C0600080240000808B50DF035FE26F0CC
:108D2000C5FB0DF0D7FDFFF74FFE0120BDE8084061
:108D300029F0CCB92DE9F047C84C63682046984724
:108D4000002800F0C180C64B1B780122042B84F858
:108D5000342000F0BB80B4F91610B4F91820B4F92F
:108D60001A302363C4E90A12BE4B1B88002B69D05A
:108D7000BD4DD4ED0A7AD5ED004A95ED050A95ED85
:108D8000015A95ED067AD5ED035A95ED026AF8EE93
:108D9000E76AD5ED047AA4EEA60AA5EE267A67EE78
:108DA000C07AA5EEC07AE6EE267A85ED057AC5EDA5
:108DB000067A37F0F9FDD4ED0B6AD5ED094A95ED49
:108DC0000E0A95ED0A5A95ED0F7AD5ED0D7AD5ED8F
:108DD0000C5A95ED0B6AA062F8EEE66AA4EEA60ABC
:108DE000A6EE857A67EEC07AA0EE657AE6EE867A20
:108DF00085ED0E7AC5ED0F7A37F0D6FDD4ED0C6A0D
:108E0000D5ED124A95ED170A95ED135A95ED187A9E
:108E1000D5ED167AD5ED155A95ED146AE062F8EEA7
:108E2000E66AA6EEA40AA6EE857A67EEC07AA0EE00
:108E3000657AE6EE867A85ED177AC5ED187A37F011
:108E4000B3FD2063894DA17F8948DFF840820DF092
:108E50007BFB2B88D8F83410002B7DD1854B1B6809
:108E60005B0741D4B1F90070A26AB1F90260B1F9AF
:108E700004508149D4E90B30D21B07EE902A9B1B8A
:108E8000401BB8EEE77A06EE100A07EE903A7B4DEB
:108E900091ED005AD1ED015AD1ED026AE362F8EE8C
:108EA000E77AB8EEC66A2B68A26237EE057A77EEEB
:108EB000A57A76EE866A0133206381ED007AC1EDF2
:108EC000017AC1ED026A2B60BDE8F0876C4BB4F902
:108ED0001600B4F91810B4F91A201880A06259804D
:108EE000E1629A8022633FE7B8F84460322E00F0D6
:108EF0008F80002E40F0CC8098F86230002BB1D0EB
:108F000008F154000DC85F4DA68A85FB03C7DB1727
:108F1000C3EB27139B1B85FB007685FB0275D217DD
:108F2000C2EB2512C017584D8B80C0EB26100023D2
:108F300008804A80AB81EB8188F862300DF024FD17
:108F400026F0B4FA0DF0C6FCFFF73EFD012029F033
:108F5000BDF8D8F8341085E7B3F5C87F4FF00003AB
:108F6000A26AA3620B80288814BFD8F83860002654
:108F7000B0F5C87F18BFD8F83C30E06A32442E887C
:108F8000C8F8382000270344B6F5C87FE762C8F860
:108F90003C304F805BD0D4F830C0D8F84000276315
:108FA0006044012E8F80C8F840002ED1DFF8D4C075
:108FB000B4F814E0C8308CFB00A9C832C833C0171D
:108FC000C0EBE9108CFB02A98CFB03ACDB17C3EBF5
:108FD000EC13D217DFF8B0C04B80A0EB0E00C2EB51
:108FE000E91288800A80ACF80C70ACF80E700DF0B5
:108FF000CBFC26F05BFA0DF06DFCFFF7E5FC30468C
:1090000029F064F82E88D8F83410701E288025E7DF
:109010001D4A0B68D2688888C8F85020A26AC8F830
:109020005420C8F84830226BA8F84C000023E06AAE
:10903000A3620B80E362C8F858004B802363C8F832
:109040005C208B8006F1FF3CA8F844C054E7236BFA
:10905000C8F8403027638F80D7E700BF5C5D0020F1
:10906000958700201C2D0020202D00208243002009
:10907000845D0020489A0020C83B0020C43B0020AB
:10908000988700201F85EB510C2D0020E82400203C
:10909000D8F85470A06AD8F85C50D4E90B2338444F
:1090A000D8F85870C8F854002B443A440025012ED3
:1090B000A5620D80E562C8F858204D802563C8F888
:1090C0005C308D80BED10B2088F8616088F86050DC
:1090D00028F0E0FED8F83410D8F84820054B0A6094
:1090E000B8F84C00D8F850208880B8F84460DA60AE
:1090F000A8E700BF0C2D002038B50D4C0D4DAC423B
:1091000006D261682046143428F060F8AC42F8D3E7
:1091100025F02EFA084A094B094C1460002209492F
:109120001A705A7008480860BDE838402EF0E4BE56
:10913000900100082C06000854610020EC900020EB
:10914000947F002058610020A480002008B5FFF71C
:10915000D3FF0DF019FC26F0A9F9BDE808400DF089
:10916000B9BB00BFF0B50C2934D8DFE801F08A3371
:1091700033335F333333343333330700048C96890E
:10918000B2F802C01788744D24F480542404240CCF
:109190000484038C8488818B23F4005321F4E641FA
:1091A0001B0409041B0C46EA0C06090C43EA0633AF
:1091B00041EA0721A8429BB2A4B289B200F09E8086
:1091C00005F58065A84200F09980926884808183CB
:1091D00002640384F0BD048C9589B2F802E017881C
:1091E0005D4E24F480742404240C0484038CB0F8B1
:1091F00004C0818B23F400731B0421F0730145EA42
:109200000E041B0C090443EA0423090CB0429BB270
:109210001FFA8CF541EA07015BD0504CA04258D0B0
:10922000926885808183C2630384F0BD048C958934
:10923000B2F802E0B2F800C0474E24F01004240453
:10924000240C0484038C8788018B23F0200321F4F1
:10925000E6411B0409041B0C45EA0E04090C43EA11
:10926000041341EA0C21B0429BB2BFB289B25BD079
:109270003A4CA04258D0926887800183826303846D
:10928000F0BD048C9589B2F802C01788324E24F0E4
:1092900001042404240C0484018C8488038B21F0B1
:1092A000020123F0730309041B04090C45EA0C05B1
:1092B0001B0CB04241EA0501A4B243EA070324D0E3
:1092C000264DA84221D092688480038342630184A2
:1092D000F0BDD489168A578A23F4006343EA042335
:1092E0004FF6FF341C40938825F440553E4344EA32
:1092F000032345EA06149BB2A5B291E7158A24F42C
:10930000804444EA8514A4B25FE7D689158A578A57
:1093100021F008013143968824F4407421F00401BF
:109320003D4331432C43CEE7D489168AB2F812C0AC
:1093300023F0800343EA04134FF6BF741C40938864
:1093400027F4406546EA0C0644EA031345EA86041E
:109350009BB2A7B28FE700BF0000014000040140AC
:109360002DE9F84FA022DFF868B29048904DDFF861
:1093700064A2904FDFF86082DFF86092002137F03E
:1093800037F98D48DFF858C2DFF858E20BF59076D0
:109390005C462368AB4200F0E580B3F1804F00F0FB
:1093A000E380BB4200F0E280634500F0ED8073454E
:1093B00000F0EC80434500F0EB804B4500F0EA8084
:1093C0007E4A934200F0E88002F57052934200F02A
:1093D000E58002F58062934200F0E28002F580624F
:1093E000934200F0DF80A2F59832934200F0DC80D7
:1093F00002F58062934200F0988002F58062934209
:1094000008BF0D2300F092802434A642C1D16C4ED7
:109410006C4D4FF003094FF002089BF80630002B0B
:109420007CD09BF804301F09013F032F03F00F038A
:1094300074D836F8170040FA03F2D2076ED54FF011
:10944000010A0AFA03F3013B184036F0AFFC5E4B09
:10945000DB5D184415EBC00760D055F830305B4831
:109460009BF8081003F13F4202F57E02920A825CEB
:1094700002F01F005209032A0AFA00FA7ED0042AD9
:1094800076D0022A04D14C48426C4AEA0202426475
:10949000B7F804C0BCFA8CF2C2F11F0292B2D00835
:1094A00003EB800002F00702076A92004FF00F0EF4
:1094B0000EFA02FE27EA0E070762076A01FA02F2B5
:1094C0003A4302624FF0010E00220EFA02F737EA29
:1094D0000C0120D15000D3F800A009FA00F1C943D3
:1094E0000AEA010AC3F800A0D3F800A008FA00F0C5
:1094F00040EA0A0018609868084098609868986088
:10950000586820EA07075F6058685860D8680140CB
:10951000D960D968D9600132102AD6D10BF1240B59
:109520005C457FF47AAFBDE8F88F0C230AEBC303E8
:1095300001211B7903F01F025B09032B01FA02F2E0
:1095400008D0042B0AD0022B7FF45EAF416C0A4393
:10955000426459E7016C0A43026455E7016B0A4310
:10956000026351E70023E1E70123DFE70223DDE7A0
:109570001148026B4AEA0202026389E70E48026C54
:109580004AEA0202026483E70323CFE70423CDE71C
:109590000523CBE70623C9E70723C7E70823C5E769
:1095A0000923C3E70A23C1E70B23BFE7A8890020EB
:1095B0000000014000040040003802400004014067
:1095C0006C400408AC87002074400408E83E04089E
:1095D000203F04088C4004080010004000140040A4
:1095E00000080040000C004000B9704703682DE9F6
:1095F000F04F03F13F4404F57E04534EA40A0125C5
:10960000345D04F01F066409032C05FA06F500F02A
:109610009580042C00F08D80022C45D08588B5FA09
:1096200085F0C0F11F0080B2C40803EB840400F091
:109630000700266A80000F27874026EA0706266271
:10964000276A01F003068240701E3A430128226215
:10965000C1F3810EC1F300184FF000024FEA51111F
:109660004FF0010C25D94FF0030E0CFA02F0A8437D
:1096700015D150001F680EFA00F4E44327401F6024
:10968000D3F8008006FA00F747EA08071F60DF6892
:109690003C40DC60DC6801FA00F02043D860013215
:1096A000102AE2D1BDE8F08F284C666C3543656422
:1096B000B4E74FF003090CFA02F737EA050033D19B
:1096C0005000D3F800A009FA00F4E4430AEA040ABF
:1096D000C3F800A0D3F800B006FA00FA4AEA0B0A71
:1096E000C3F800A0D3F808A004EA0A0AC3F808A047
:1096F000D3F808B00EFA00FA4AEA0B0AC3F808A039
:10970000D3F804A02AEA07075F60D3F804A008FA98
:1097100002F747EA0A075F60DF683C40DC60DC680C
:1097200001FA00F02043D8600132102AC3D1BDE80D
:10973000F08F064C266B354325636FE7034C266C90
:10974000354325646AE700BFE83E0408003802405C
:1097500003682DE9F04F03F13F4404F57E04534EB6
:10976000A40A0125345D04F01F066409032C05FAE0
:1097700006F500F09680042C00F08E80022C46D076
:109780008588B5FA85F0C0F11F0080B2C40803EBEC
:10979000840400F00700266A80000F27874026EA2D
:1097A00007062662276A01F0030602FA00F0721E1D
:1097B0003843012AC1F3810EC1F3001820624FEA39
:1097C00051114FF000024FF0010C25D94FF0030E5C
:1097D0000CFA02F0A84315D150001F680EFA00F4ED
:1097E000E44327401F60D3F8008006FA00F747EAF9
:1097F00008071F60DF683C40DC60DC6801FA00F0AD
:109800002043D8600132102AE2D1BDE8F08F284C05
:10981000666C35436564B3E74FF003090CFA02F751
:1098200037EA050033D15000D3F800A009FA00F45C
:10983000E4430AEA040AC3F800A0D3F800B006FA29
:1098400000FA4AEA0B0AC3F800A0D3F808A004EA19
:109850000A0AC3F808A0D3F808B00EFA00FA4AEAD8
:109860000B0AC3F808A0D3F804A02AEA07075F6030
:10987000D3F804A008FA02F747EA0A075F60DF6836
:109880003C40DC60DC6801FA00F02043D860013223
:10989000102AC3D1BDE8F08F054C266B35432563F4
:1098A0006EE7034C266C3543256469E7E83E0408FF
:1098B0000038024010B50409013C032C17D80E4BA8
:1098C00033F8142000F00F0042FA00F313F0010304
:1098D0000FD0012303FA00F00138104036F066FA89
:1098E000064A074B125D104403EBC00010BD002078
:1098F00010BD184610BD00BF6C4004087440040839
:10990000AC8700202DE9F8432F4D2B8AB5F80C8049
:1099100018EA030827D02D4E4FF00047B8FA88F315
:1099200027FA03F2D24391B21B3B08EA02082982CC
:10993000042B15D8DFE803F0352B22190300D6F8E5
:109940009C30002B37D1EB6A1FFA83F9D6F8984088
:1099500034B123682046494698476468002CF8D102
:10996000B8F1000FDAD1BDE8F883B06F696B036816
:1099700089B29847B8F1000FD0D1F4E7F06FA96B26
:10998000036889B29847B8F1000FC7D1EBE7D6F862
:109990008000E96B036889B29847B8F1000FBDD128
:1099A000E1E7D6F88400296C036889B29847B8F1DA
:1099B000000FB3D1D7E703F1FF3900231FFA89F96C
:1099C000C6F89C30C2E700BF00040140A88900200F
:1099D0002DE9F8432F4D2B8AB5F80C8018EA0308BF
:1099E00027D02D4E4FF00047B8FA88F327FA03F23C
:1099F000D24391B21B3B08EA02082982042B15D8F6
:109A0000DFE803F0352B22190300D6F89C30002B39
:109A100037D1EB6A1FFA83F9D6F8984034B123683E
:109A20002046494698476468002CF8D1B8F1000FE9
:109A3000DAD1BDE8F883B06F696B036889B29847E3
:109A4000B8F1000FD0D1F4E7F06FA96B036889B2C9
:109A50009847B8F1000FC7D1EBE7D6F88000E96B63
:109A6000036889B29847B8F1000FBDD1E1E7D6F895
:109A70008400296C036889B29847B8F1000FB3D10C
:109A8000D7E703F1FF3900231FFA89F9C6F89C30A4
:109A9000C2E700BF00040140A88900202DE9F84377
:109AA0002C4D2B8AB5F80C8018EA030825D02A4ED5
:109AB0004FF00047B8FA88F327FA03F2D24391B285
:109AC0001B3B08EA02082982042B13D8DFE803F0C5
:109AD000322920170300736F002B34D1EB6A1FFA71
:109AE00083F9346F34B12368204649469847646847
:109AF000002CF8D1B8F1000FDCD1BDE8F883306D4F
:109B0000696B036889B29847B8F1000FD2D1F4E7C6
:109B1000706DA96B036889B29847B8F1000FC9D17D
:109B2000EBE7B06DE96B036889B29847B8F1000FB5
:109B3000C0D1E2E7F06D296C036889B29847B8F1AB
:109B4000000FB7D1D9E703F1FF3900231FFA89F9D4
:109B50007367C6E7000C0040A88900202DE9F84390
:109B60002C4D2B8AB5F80C8018EA030825D02A4E14
:109B70004FF00047B8FA88F327FA03F2D24391B2C4
:109B80001B3B08EA02082982042B13D8DFE803F004
:109B9000322920170300F36C002B34D1EB6A1FFA33
:109BA00083F9B46C34B12368204649469847646809
:109BB000002CF8D1B8F1000FDCD1BDE8F883B06A11
:109BC000696B036889B29847B8F1000FD2D1F4E706
:109BD000F06AA96B036889B29847B8F1000FC9D140
:109BE000EBE7306BE96B036889B29847B8F1000F77
:109BF000C0D1E2E7706B296C036889B29847B8F16D
:109C0000000FB7D1D9E703F1FF3900231FFA89F913
:109C1000F364C6E700040040A88900202DE9F8435A
:109C20004FF080452B8AB5F80C8018EA030825D040
:109C3000294E4FF00047B8FA88F327FA03F2D243CF
:109C400091B21B3B08EA02082982042B13D8DFE8F3
:109C500003F0322920170300736A002B34D1EB6A1A
:109C60001FFA83F9346A34B123682046494698477D
:109C70006468002CF8D1B8F1000FDCD1BDE8F8839E
:109C80003068696B036889B29847B8F1000FD2D188
:109C9000F4E77068A96B036889B29847B8F1000FC0
:109CA000C9D1EBE7B068E96B036889B29847B8F1AE
:109CB000000FC0D1E2E7F068296C036889B29847C9
:109CC000B8F1000FB7D1D9E703F1FF3900231FFA2C
:109CD00089F97362C6E700BFA8890020F0B506685D
:109CE0003F4CB30AA3426CD065D93E4CA3425AD034
:109CF0003E34A34256D1982703254379B6F80CE0A9
:109D0000022023FA00F4A0401FFA80FCA80023469A
:109D1000441903EB4403344C002955D04CEA0E0C93
:109D200003F1040E44F8231044F82E20A6F80CC0CA
:109D3000E319EFF31181502282F31288421904EBE8
:109D4000C202D2F810C0BCF1000F03D044F807C023
:109D500013690433421904EBC202576917B11F603B
:109D600053690433421904EBC202976917B11F60AB
:109D700093690433421904EBC202D76917B11F601B
:109D8000D36904330027CAB21F6082F311882844C4
:109D900004EBC004236A4BB9B38923F001031B040D
:109DA0001B0CB381F0BD70270225A6E7B38943F0F1
:109DB0000103B381F0BDB3F5801FF3D12027002547
:109DC0009BE74827012598E72EEA0C0C03F1040EC7
:109DD000A6F80CC044F8231044F82E20A8E700BFD2
:109DE0000100100003001000A889002010B50368CE
:109DF0007C487D4C0139834282B0246889B200F0EE
:109E0000AF80A0F58060834200F0AA8000F580401A
:109E1000834200F0818000F5806083427CD000F5B1
:109E20008060834278D018886408B4FBF2F4013C67
:109E3000A4B282B2B3F1804F0AD06C48834207D0FB
:109E400000F58060834203D000F58060834202D138
:109E500022F0700292B26648834200F08F8000F5D3
:109E60008060834200F0938022F4407200F56C40E1
:109E700092B283421A80D9621C8540F09180012100
:109E800000221A86998219885A4841F001018342BA
:109E9000198049D0B3F1804F00F08D80534A93422E
:109EA00000F08B8002F58062934200F0888002F51A
:109EB0008062934200F0858002F58062934200F058
:109EC000828002F5806293427FD002F57042934215
:109ED0007DD002F5705293427BD002F580629342AE
:109EE00079D002F58062934277D0A2F598329342FE
:109EF00075D002F58062934215D002F580629342DC
:109F000008BF0D2210D002A84FF0012340F8043DF5
:109F10001EF0C6FB02B010BD1888B4FBF2F4013C81
:109F2000A4B282B286E70C22334B03EBC20201A833
:109F300054798DF80440012300228DF805308DF806
:109F400007308DF806201EF0ABFB1B2C0FD02E2CFB
:109F5000E0D12A4B019301A81EF0A2FB02B010BD74
:109F60001888B4FBF2F4013CA4B282B270E7244B2F
:109F7000019301A81EF094FB02B010BD01201A80CD
:109F8000D9621C8598821A8802431A8086E70120CC
:109F90001A80D9621C8598821A8802431A8079E750
:109FA000104A93423FF46BAF01229A821A8842F022
:109FB00001021A806EE70122B6E70222B4E703220B
:109FC000B2E70422B0E70522AEE70622ACE707229B
:109FD000AAE70822A8E70922A6E70A22A4E70B229B
:109FE000A2E700BF00040140B0A800200004004028
:109FF00000100040000001408C4004082C010001CA
:10A00000190100012B4B98423CD0B0F1804F3BD05E
:10A01000A3F57C43984239D003F58063984237D04A
:10A0200003F58063984235D003F58063984233D0BE
:10A0300003F58063984233D003F57043984231D0E2
:10A0400003F57053984229D003F5806398422BD0D2
:10A0500003F58063984229D0A3F59833984227D01E
:10A0600003F58063984207D003F58063984208BFE8
:10A070000D2202D0002070470C220F4B03EBC203CD
:10A08000187970470022F8E70122F6E70222F4E788
:10A090000322F2E70422F0E70522EEE70822ECE7CC
:10A0A0000622EAE70722E8E70922E6E70A22E4E7D0
:10A0B0000B22E2E7000001408C4004082DE9F04F3C
:10A0C00083B08E4DDFF8408201908B460BF1FF3359
:10A0D0009B46013300F00E8132F0B8F8884C894F6E
:10A0E000DFF828C24FF4FA7A4FF0100E4FF47A7668
:10A0F000DCF80430C3F30803002B40F0DF80EFF3FB
:10A100001183002B40F0DA802168AA6800BF236821
:10A110009942F9D1386806FB00F39A1AB2FBF0F2C3
:10A1200006FB0121DCF80430C3F30803002B40F0E8
:10A13000A680EFF31183002B40F0A1802368A8686C
:10A1400000BF22689342F9D1D7F8009006FB09F2CC
:10A15000101AB0FBF9F006FB03035B1AB3F57A7F24
:10A16000E0D3BAF1010AC3D1019B581CC0B231F04F
:10A17000C9FEDFF898C1DCF804304FF47A7AC3F3F3
:10A18000080356464FF0100E002B38D1EFF3118321
:10A19000002B34D12168AA6800BF23689942F9D105
:10A1A000386806FB00F39A1AB2FBF0F206FB0121B5
:10A1B000DCF80430C3F30803002B41D1EFF3118323
:10A1C000002B3DD12368A86800BF22689342F9D1D3
:10A1D000D7F8009006FB09F2101AB0FBF9F006FB65
:10A1E00003035B1AB3F57A7FE2D3BAF1010A3FF4B5
:10A1F0006DAFDCF80430C3F30803002BC6D0EFF3D7
:10A2000011828EF31288A8682B68D90303D5012325
:10A21000C8F80030A8682368D8F80010D2B282F3DA
:10A2200011883A68194406FB02F31B1AB3FBF2F3D8
:10A2300006FB0131DCF80430C3F30803002BBDD06A
:10A24000EFF311808EF31288D5F808902B68DB03AA
:10A2500004D50123C8F80030D5F808902368D8F851
:10A260000020C0B280F311883868134406FB00F266
:10A27000A2EB0902B2FBF0F206FB0323B1E7EFF316
:10A2800011808EF31288D5F808902B68DB0304D573
:10A290000123C8F80030D5F808902368D8F80020CA
:10A2A000C0B280F311883868134406FB00F2A2EBB9
:10A2B0000902B2FBF0F206FB03234EE7EFF3118233
:10A2C0008EF31288A8682B68D90303D50123C8F838
:10A2D0000030A8682368D8F80010D2B282F3118841
:10A2E0003A68194406FB02F31B1AB3FBF2F306FBB0
:10A2F000013117E703B0BDE8F08F00BF10E000E0C8
:10A30000D4900020D8900020D090002000ED00E0F4
:10A31000204B5B68C3F3080330B4BBB9EFF3118380
:10A32000A3B91D4A1D481368846800BF11688B4299
:10A33000F9D11B4A11684FF47A7202FB01F0001B3D
:10A3400030BCB0FBF1F002FB03007047EFF3118269
:10A35000102383F312881149124D8C680B68DB03BC
:10A3600044BF01232B600C4B48BF8C681B682868D6
:10A37000D2B282F311880A4A11684FF47A721844F3
:10A3800002FB01F31B1B30BCB3FBF1F302FB0030FB
:10A39000704700BF00ED00E0D490002010E000E026
:10A3A000D8900020D09000202DE9F04F2DED068BA5
:10A3B000834B844A1D7800F59C4720379BB00646A6
:10A3C0001760002D01F0A5807F49804A0968079237
:10A3D000884284BF05F1FF351D707D4B12680693DE
:10A3E0007C4B05937C4B099302F48052002A41F088
:10A3F0005E807A4B1B78022B01F06780042B01F002
:10A40000B982012B00F00186754B099A9E42927821
:10A4100000F24486002A40F04486724B0893079B62
:10A420001E68059B16F48059B3F9065040F0F68675
:10A43000069B6D4F5C8BAC42CCBF002401246B4A61
:10A44000089B12681B78D00003F0010340F1688577
:10A45000002B40F01985664D002285F8F020002C75
:10A4600000F02085634A01211170002B40F02B85FC
:10A47000614B1B78002B40F08E80069B059A598B10
:10A48000B2F900009A8B5A4D8142B4BF8023002359
:10A4900082420598B0F90200C8BF43F040039B0810
:10A4A0008142BCBF63F07F03DBB282420598B0F902
:10A4B0000400C8BF43F040039B088142BCBF63F067
:10A4C0007F03DBB282420598B0F90600C8BF43F0B3
:10A4D00040039B088142BCBF63F07F03DBB2824232
:10A4E00095F8F220C8BF43F040039A4201F04D8333
:10A4F000424A85F8F23011780022A5F8F42085F858
:10A50000F620002901F072845F2B44D06F2B42D0DB
:10A51000089B1A78079BD0071B683ED495F8F62055
:10A52000002A3AD1B5F9F410322936DD95F8F21047
:10A530000120572985F8F60001F01B865B0702D53C
:10A540005A2902F0D2815D2902F014815E2902F0BD
:10A550000A815B2902F0F880562902F0A081972930
:10A5600002F0B981A72902F0AD81DFF89490B9F823
:10A5700000309E0742F09981A1F1B703072B02F248
:10A580004F82DFE813F0BA124D124D124D12B31282
:10A590004D12AC12A512079B1B68DFF864905D0793
:10A5A00001F16C80DFF85C80CDF828800023CDE9D4
:10A5B0001633CDE918334446DDF814A02FE000BF70
:10A5C000503500208C2B00204C350020489A00206C
:10A5D0003C900020705E0020A85E0020B03000207B
:10A5E000404B4C00045D0020003600206833002002
:10A5F000E8240020CC420020C9830020E400002091
:10A60000585D00209C350020294618A823F0A2FFA1
:10A61000834668B9464511D30534A74237D025781B
:10A62000272DF9D82379A67894F80380012BEBD154
:10A63000464580F012834FF0010B5846637804338F
:10A6400040F6330C3AF913106145A8BF6146B1F5E5
:10A65000617F4FF0190340F2833CB8BF4FF4617142
:10A6600013FB06C68E4280F2008313FB08C38B42A5
:10A67000B4BF00260126002840F0F282B345CBD0BB
:10A68000294616A8053423F055FFA742C7D19DF8E7
:10A6900059009DF861109DF858509DF860309DF864
:10A6A0005A20DDF8288041409DF862008DF859104D
:10A6B0006B4042408DF858309DF85B009DF8633048
:10A6C0008DF85A2043408DF85B3016AA584B92E81B
:10A6D00003001B78574A82E80300002B40F0CF8626
:10A6E000554B1F78002F00F0CF85544B0A935148EB
:10A6F000012123F02FFFB9F8006020B9099BDB7816
:10A70000002B00F0B4824E4D2B689A0740F1B082C6
:10A71000F30741F1B38333B223F002039BB2B34298
:10A72000A9F800300AD0474B41F20241FF221980BC
:10A730000E209A7027F0AEFBB9F80060424B1978F2
:10A74000424BB607586801F0020100F097830031D0
:10A7500018BF012121F0B2FD2421364823F0FAFE72
:10A7600030B9089A1378590744BF23F004031370D3
:10A770002B68B9F8007013F00A0F1DD005212D4881
:10A7800023F0E8FE002801F07D817A0741F1AF81D6
:10A790002848062123F0DEFE002801F08D817B068B
:10A7A00041F19D810721234823F0D4FE002841F088
:10A7B0001B812B68B9F800709E0600F11387244EA8
:10A7C0001C480C2123F0C6FE002800F0368347F415
:10A7D0008073BB42A9F8003008D01A4B41F2024105
:10A7E000FF2219800E209A7027F054FB194B1B781A
:10A7F000082B00F02F830E2B00F02C83079B1F6883
:10A80000780560D5144B1B79002B40F09083089B92
:10A810001B78D90700F192831FF03EFC012027F03E
:10A820003DFA00284DD0DFF834B00B9400251AE033
:10A830005E9C002068330020305D002058610020BD
:10A840009C5D0020343900209C900020A0900020C6
:10A85000085D002024350020E05A0020BCB1002013
:10A86000DDB2032D2CD0CC2303FB05FA6B1C5BF867
:10A870000A70002FF4D1032290F90230029701925E
:10A88000C278E34951F82220009218463A463B46E6
:10A89000012126F03FFE05EB450202EB02120446C1
:10A8A0000BEB820240B1101D3946C82235F0A0FEE4
:10A8B00001354BF80A40EDB231F0D0FF0028D0D17D
:10A8C0000B9C079B1F68089B93F800A0D14B1AF0C4
:10A8D000010A00F0328201221A700A9BCE481A68DF
:10A8E000059BD189B3F9063001258B42057080F2B2
:10A8F0000C82CA4A4FF07E511160C949069A0598E8
:10A90000158BB0F900C091F90420087891F801E0A6
:10A91000002AACEB050214BF01214FF0FF31002AE1
:10A92000B8BF5242B2F5FA7FA8BF4FF4FA72824222
:10A93000C4BF121A07EE902A059AD4BFDFEDB97A88
:10A94000F8EEE77A6545B2F902C0C6ED007AACEBE5
:10A950000502C4BFF1EE677AC6ED007A002AB8BFDF
:10A960005242B2F5FA7FA8BF4FF4FA729042BCBFD0
:10A97000121A07EE902A059AA8BFDFEDAA7AB2F95B
:10A980000400B8BFF8EEE77A6545A0EB0502C6ED16
:10A99000017AC4BFF1EE677AC6ED017A002AB8BF2A
:10A9A0005242B2F5FA7FA8BF4FF4FA72964580F290
:10A9B000A981A2EB0E0201FB02F107EE901AF8EE5C
:10A9C000E77A8542C6ED027A9749C4BFF1EE677A0D
:10A9D000C6ED027A17F48057087800F08081B3F54D
:10A9E000FA6FA8BF4FF4FA63B3F57A7FB8BF4FF49C
:10A9F0007A73A3F57A73002841F081808B49DFF8E0
:10AA000040C281FB0320DA17C2EB6012501C6FF0CA
:10AA1000630E3CF910003CF912C00EFB0233A0EBB0
:10AA20000C0003FB00F381FB0321DB17C3EB611375
:10AA30009C440FFA8CFC07EE90CAB8EEE78A86EDCC
:10AA4000038A002F40F0D784B9F800305A0640F14D
:10AA5000F9807749774A91ED018A92ED027A92ED79
:10AA6000014AD1ED033AD2ED006AD1ED028A92EDAE
:10AA7000036AD1ED005AD6ED011A96ED002A6E4A0E
:10AA80006E4938EE635A74EE470A76EE867A65EEC2
:10AA9000200A75EEE84A36EEC69A75EEA89A64EE7C
:10AAA000A74AB0EE603AA9EE893A13F00303B0EE7C
:10AAB000645A38EE231A74EE077AA9EE895AA1EE89
:10AAC000273AB0EE600A91EE270AA1EE675A33EEFC
:10AAD000243AF0EE407AB6EE000A35EE88AAB0EEDF
:10AAE000671A20EE433A35EE605A76EE840AA9EEF4
:10AAF000C91AAAEE203A77EEE47A77EE460A33EEE8
:10AB0000E8AA25EE005AE9EE897AAAEE205A71EEFB
:10AB1000244A36EEC44A63EE036A73EEA83A64EE42
:10AB2000804A75EEC85A37EE066A67EE807AB0EE54
:10AB3000667AE3EE844A95EE057AE5EE056AE5EE7F
:10AB4000867AB1EE648AF0EE665AF0EE476AB1EEAC
:10AB5000674AE8EE246A63EE270A67EEA43AE4EE59
:10AB6000275AB1EE450AB0EE606AB0EE631AA4EE61
:10AB7000277A23EE244AE7EEA76AA5EE246AA0EE20
:10AB8000031AE8EE245AB0EE448A31EEA19AE0EEC0
:10AB9000240AA5EE278A66EEA16A72EE028AE5EE25
:10ABA000033A61EE211A26EE096AA4EEA47AA0EE19
:10ABB000274A0CBFD6ED022ADFED1A2A82ED005A91
:10ABC000A2EE256AE8EEA06AE2EE081A73EEA33A56
:10ABD00027EE227A34EE044AF0EE005AE3EEA26A3F
:10ABE000A2EE846AA1EEA57AC6ED016AC1ED406AC3
:10ABF00081ED3F6A86ED006A81ED417A82ED013A8E
:10AC0000C2ED027AC2ED034AE3B986ED027A19E099
:10AC10000C340408E45E0020004300207C42002045
:10AC2000FC34002000000000807600201F85EB51DE
:10AC3000EC00002098000020D0000020E824002034
:10AC400068430020BAF1000F40F0518217F016FF60
:10AC50001BB0BDEC068BBDE8F08F00264FF0010B5A
:10AC6000294618A823F066FC08E5002603E5C04D38
:10AC700026F001039BB2B342A9F800300AD0BD4BC5
:10AC800041F20241FF2219800E209A7027F002F94A
:10AC9000B9F80060B848022123F05CFC33B2002808
:10ACA0003FF43AAD23F001039BB2B342A9F8003060
:10ACB0000AD0B04B41F20241FF2219800E209A7057
:10ACC00027F0E8F8B9F80060B7073FF537AD46F070
:10ACD0000203B342A9F800307FF425AD2EE5069AB1
:10ACE000528B934280F27E813B4600283FF486AE31
:10ACF0004A78A24903FB02F381FB0312DB17C3EB83
:10AD000062137BE6DFED9E7A5BE6B3F5FA6F127BAA
:10AD10009FED9C7ABFBF581A4243C1F5FA6192FB7E
:10AD2000F1F2C2F1640207EE902AF8EEE77A964A51
:10AD300067EE877AC2ED007ADFE51A780792002A7B
:10AD40007FF4CBAD914B1B68002B3FF4C6AD904B0D
:10AD5000904A13F8030C08931946A3F1030B1578D6
:10AD600011F05AFF089B002801F01781079A002D67
:10AD700055D10BF108019BF8050011F04DFF00289B
:10AD800041F07A8584499BF80A0011F045FF0028BC
:10AD900001F01781022D41F06B8580499BF80F006F
:10ADA00011F03AFF002841F05F857D499BF81400BF
:10ADB00011F032FF002801F01781042D41F0508579
:10ADC00078499BF8190011F027FF002841F04485CD
:10ADD00075499BF81E0011F01FFF002801F0178134
:10ADE000062D41F0358571499BF8230011F014FFC1
:10ADF000002841F029856E499BF8280011F00CFFCE
:10AE0000002801F01781082D41F01A8569499BF847
:10AE10002D0011F001FF00283FF45FAD0922134619
:10AE200003EB83039B445B4D634B9BF801109BF842
:10AE300002002A70197058704FE527F480739BB296
:10AE4000BB42A9F800307FF4C8AC5C4B1B78082BE0
:10AE50007FF4D1ACB9F8002022F040039BB29A42B3
:10AE6000A9F800303FF4CAAC424B41F20241FF2244
:10AE700019800E209A7027F00DF8BFE4B1FA81F125
:10AE8000490921F01BFA67E4069A528CAA4240F362
:10AE90006386002C7FF4E6AA494D95F8F020002A3D
:10AEA0007FF4E0AA474A4849106890F82D00002234
:10AEB0000A604A608A6000287FF4D4AA434A10706E
:10AEC000002B3FF4D5AAF2067FF5D2AA404B1B789F
:10AED000DB063FF5CDAAB9F1000F7FF4C9AA11F046
:10AEE000C5FE00287FF4C4AA3A4B1B78002B01F062
:10AEF0001F85394B9B78002C41F00B853BB1374ABD
:10AF0000374B12681B689B1A002BC1F2DA851020A0
:10AF10002B4D26F0BFFF012385F8F130FFF7A8BACB
:10AF200071027FF598AA002BAED1FFF794BA1421D5
:10AF3000114823F00FFB00283FF46EAC4FF40F7064
:10AF400033F002FE00283FF4BCAC26F0CBFA4FF4FD
:10AF50000F7033F099FD00283FF4B3AC26F0C2FA2D
:10AF60004FF40F7033F090FD0028EED1A9E400BF3C
:10AF70009C5D002034390020683300201F85EB5190
:10AF8000000000000AD7233C7C420020345D0020F2
:10AF9000C332002000000020CD320020D232002039
:10AFA000D7320020DC320020E1320020E6320020DF
:10AFB000EB320020F0320020265D002024350020F6
:10AFC000E824002054610020C42C0020CC42002042
:10AFD0009C5E0020E400002014350020D490002066
:10AFE00098430020B3F5FA6FD4BFC2EB030CC2F54F
:10AFF000FA6C4FF47A73C2F5FA6203FB0CF3B3FBFD
:10B00000F2F300283FF4FAAC72E68C4DD5F8EC3040
:10B01000F31A002BFFF6F8A9894A8A4B527CDFED20
:10B020008A7A33F812309FED896AC5F8EC7006EE23
:10B03000903A069B9A7DD97D07EE102AF8EEE66AD3
:10B04000B8EEC77A66EE866A27EE277A40F2FF32BC
:10B05000C6EE877AFCEEE77A17EE903A9BB29342FF
:10B0600028BF134609B1D31A9BB27948794D0178AC
:10B07000794C35F81170226825F81130D21B134431
:10B08000764D236001311B0901F00F022B80744BB8
:10B090000270099A9E4292787FF6BCA9002A00F0BD
:10B0A0006F85704B099A1C7892F8215008931B20E9
:10B0B00011F0EAFD012D04F00107814600F0FB8646
:10B0C00004F00204099A684E92F82030DFF8B0A12B
:10B0D000DFF8B0810A949346052B00F23485DFE84F
:10B0E00013F06F00ED05130085009405F0055F4B2C
:10B0F00019785F4B01F00101186821F0DFF81BB0EF
:10B10000BDEC068BBDE8F08F012D04BF05238BF845
:10B11000203097B1069B3088B3F9181000221346EF
:10B1200061F30F0361F31F4361F30F02059960F3AD
:10B130001F420B6003234A600A934E4CDBF8141045
:10B140002268914280F0E48647F230510322CBF826
:10B150001C108BF82020022028F04EF917F04CFE2E
:10B160002168DBF81C200A440421CBF818208BF856
:10B170002010012D41F05A832268DBF8181091420B
:10B1800080F0E1849AF80000002800F0D784D8F815
:10B19000002022F00202C8F800202268738864218F
:10B1A00001FB03234FF480600022CBF810308BF8B2
:10B1B00020208BF8032028F0EFF89BF820308BE755
:10B1C000002F01F0268317F001FA012800F06885AE
:10B1D000B9F1000F0CD0B37953B111F0DBFC0322AD
:10B1E0004FF47A738BF82020CBF81C30214CB2E757
:10B1F000012D00F0A8841F4CDBF81010226891424A
:10B20000C0F0F88401238BF82030F379012B00F093
:10B21000738611F0BFFC9BF820305DE71D211648B6
:10B2200023F098F9002800F0A786144F069B5C8B4A
:10B23000AC42CCBF00240124FFF701B9E824002070
:10B2400034890020588900200000C8420000804452
:10B25000B1300020B8300020B4300020985E0020CB
:10B26000404B4C00045D0020204100209C900020B9
:10B27000A0900020D49000206833002000360020E9
:10B28000E4000020CC5E0020DFF8E0A2A84DDFF84B
:10B29000E0B20AF15A0651461AF8010C11F0BCFC52
:10B2A000E8B19AF804109AF8023001EB410C05EB72
:10B2B0008C00013B426803EB43035B4493420ED096
:10B2C00095F8F9204360012303FA01F19AF803305D
:10B2D00005F82C3022EA0101876085F8F9100AF19F
:10B2E000060AB245D7D1934B934A0A931946934B1A
:10B2F000126809681B788E4E0C940D910B934FF0D9
:10B30000FF3B4FF0000A14467368002B69D01F788A
:10B31000002F66D0B268A21A002A0FDB95F8F92038
:10B32000012101FA0AF122EA010285F8F920844A92
:10B3300004F5FA704FF0FF31B06011600B9A002AEB
:10B340004FD0327859780432D2B200293AD10699D6
:10B350000598098B30F9120095F8F92001F1C80C15
:10B36000604540F3FF8342FA0AF1C8079A7838D45F
:10B37000002A0CBF012002200E9226F0A7FE7B1EA1
:10B380000E9A1B2B01F22281DFE813F00909ED0868
:10B39000D108BA08A7088A086D085008380820089C
:10B3A000F0072009BA08DD078A086D085008C507AC
:10B3B000AD07960784076D0754072009090942075E
:10B3C000ED082B07012900F02384BBF1FF3F40F07B
:10B3D000578495F8F920012303FA0AF3134385F8FB
:10B3E000F9300AF1010ABAF1040F06F10C068BD10B
:10B3F0000C9CFFF77CB91D21524823F0ABF830B10B
:10B4000000F095BD08F10508A0453FF41DAB98F884
:10B4100000102629F6D198F8022098F803309A42B5
:10B42000F0D2099BDB78002B7FF40EAB454823F06C
:10B4300091F8DFED457A454A78EE677AFDEEE77AD6
:10B4400017EE903A1BB21B0382FB0312DB17C3EB10
:10B45000A213002801F02981C5F57A7212B203FB0C
:10B4600002F343F30F332B4407EE903A384BF8EED8
:10B47000E77A0122C6ED037A1A70FFF7E5BA354B79
:10B4800003E00533A3423FF42BA919782329F8D10F
:10B490009878DA789042F4D22A4823F05BF80028B2
:10B4A0003FF41EA9142026F0F5FCFFF719B900217E
:10B4B000244823F04FF800287EF49BAF17F09CFC43
:10B4C000254B1B78022B7EF499AF069A0599537D84
:10B4D000D27D013B31F913301AB1C3F53B63083318
:10B4E0001BB2A3F57A7307EE903A9FED1C7A1C4AC3
:10B4F000F8EEE77A40F2FF3167EE877AFCEEE77A02
:10B5000017EE903A9BB28B4228BF0B461380FEF792
:10B510007BBF144B1C78002C00F0E385DFF854B09F
:10B52000114CDFF854A00694DFF85090D8464FE055
:10B53000E824002058610020D4900020065D0020FF
:10B54000700600206833002000007A44D34D62105A
:10B55000F44200209C350020B03000206F12833F61
:10B56000985E0020743600203C900020F4320020C9
:10B570000C110408782B00204C2500207A3600207E
:10B58000615D9847032D03462ADCC8B109EB8503AA
:10B5900039F825105A88401A4FF47A7303FB00F0EB
:10B5A000521A40F6CA0390FBF2F000F57A70984206
:10B5B000A8BF184640F2EE239842B8BF184600B222
:10B5C000414B2AF8020B1B7801359D4280F2948092
:10B5D000072D4046DBF80430D2DDE9B29847034638
:10B5E00018B2EDE7394B1B789D071FD5384D2B7DE1
:10B5F000042B1BD90A2011F047FB07F010038246E9
:10B60000002800F09A85002B01F0F480314D95F868
:10B61000FA30002B7FF4D3A80D2026F03BFC012349
:10B6200085F8FA30B9F80070FFF7C9B817F0300F95
:10B630003FF4C5A8102027F0AFFE202027F0ACFE75
:10B64000254BB9F80070254E00221A702449254870
:10B65000254D002300220B608B604B61CB614A605B
:10B660008A610260214922482A6002600B604A60B8
:10B670008B604B618A61CB61FFF7A2B8154D95F8DD
:10B68000F8305BB1089B1B78DC0707D5059BB3F945
:10B690000620069B5B8B9A4200F3418511211548D9
:10B6A00022F058FF002800F0378295F860302BB95F
:10B6B00095F8613013B93223A5F84430012385F899
:10B6C0006030FEF76FBF00BF743600209C5E002024
:10B6D00018A90020E82400200C840020085D002028
:10B6E000A8840020A842002060430020D0840020CD
:10B6F000F8840020683300201C46A54BA54A079318
:10B700001B68A2FB061242F2010C920913EA0C0C10
:10B710000E9200F0FD81A04DA049A148A14A95F8E4
:10B720000080097880F800801170B8F1000F04D013
:10B730009C4A92F8008088F001089B4D4FF00F0A58
:10B7400085F888A0002C00F05F830699974A109234
:10B750001078CA8C09920A8B1492954A0592954AE0
:10B76000B1F824E00F90A2FB0021490801EB410150
:10B77000411AC9B203F480530C9115934B000E99F2
:10B78000DFF85C9295F889B00D93601E032801F5EF
:10B790009672A8BF03200A92CDE912462A46844C2D
:10B7A00011976546CDF82CA0844600234046774685
:10B7B00008919046002800F0AB827F4A32F91320AE
:10B7C0001FFA82FE77454FEA430103D8099EB6452A
:10B7D00040F2ED8259F82320089E964280F0A28222
:10B7E000625E002D40F0BB82013363456252E1DDB1
:10B7F000BE46DDE91174A342AC46139E4546804621
:10B800005FDA6E4A1196580000EB030A02EB4A0A0F
:10B8100048320D920E9A089202F596710E972A46BA
:10B820007746A64644460A91654605999446CCB1AA
:10B83000614A125E1FFA82F8474502D8099E4645C2
:10B8400013D259F82320089E964280F0B4820A5EF3
:10B8500085B9013373450A520AF1060A2ED0580001
:10B86000002CE5D1002FECD13A460A9E49F823601E
:10B87000002DEED00C9E2AF81620BBF1000F02D14D
:10B880000F9E022EE5D9BAF800B0BAF80220BAF835
:10B8900004805A4490444A4A0FFA88F882FB0862AE
:10B8A000A2EBE8720D9E013312B2734526F80080B8
:10B8B0004FF0010B0A520AF1060AD0D10E9F119ED9
:10B8C00065460B993F4B85F889B00F290CBF0122C3
:10B8D000002285F888101A7000F09D823A4C2F499A
:10B8E000304ADFF800B10994012304200B70137073
:10B8F00027F082FDDBF80030A1686268E3605B1A24
:10B90000934202D9002384F82130304B1878079BEA
:10B910001A6802F4805238B3069B254DB3F8248090
:10B92000B3F818E02A49002A40F0C88213460CE018
:10B930009CF8014004EB840404EB840404F2EE243C
:10B940000133984225F8024B0ED011F8134001EB59
:10B95000430C002C00F04182022CE9D001332C88EA
:10B9600025F8024B9842F0D110990B7801330B70F7
:10B97000FEF73CBDFEF7CCFC164B174A1B68C31AFA
:10B9800093427EF741AD154B00221A80FEF73CBD75
:10B99000489A0020D34D6210542B002078000020DC
:10B9A000065D002079000020E824002051350020A9
:10B9B000705E0020ABAAAAAA4C25002074250020A6
:10B9C0005655555570330020A85E0020743600206F
:10B9D0000D390020C87C002060E31600985E00202E
:10B9E00054350020D4900020B74AB2F90030002B23
:10B9F000B8BF5B42B3F5E17FBEF6DBAEB2F9023011
:10BA0000002BB8BF5B42B3F5E17FBEF6D2AEAF4BC1
:10BA1000AF4E93ED057AD3ED077AD3ED096A93ED36
:10BA2000030A77EEA67A30EE070AF7EE000AB0EEC8
:10BA3000007AE7EEC70A30EE000A22F0D3FABEEE33
:10BA4000008A20EE088AB0EE480A22F039FBFDEEAB
:10BA5000C87A86ED000A17EE903ADFED9E7A203321
:10BA6000402BC6ED017AC6ED027A00F27F83B0EE7C
:10BA7000480A22F035FA0A2086ED030A26F00AFA6F
:10BA8000FEF797BE27F004039BB2BB42A9F8003033
:10BA90003EF47EAE904B41F20241FF2219800E200F
:10BAA0009A7026F0F7F98D48B9F80070062122F057
:10BAB00051FD00287EF473AE27F040039BB2BB42D9
:10BAC000A9F800303EF46EAE834B41F20241FF22F2
:10BAD00019800E209A7026F0DDF9FEF763BE47F05C
:10BAE0004003BB42A9F80030EED1FEF75BBE47F041
:10BAF0000403BB42A9F80030CCD1FEF749BE4A7816
:10BB0000774903FB02F3A1FB03235B09FEF776BF32
:10BB1000744A92F8008008E695F86130002B3EF4F4
:10BB200041AD089B1B7813F001037EF43BAD01226D
:10BB300085F8613085F86220FEF734BD11F0A4F875
:10BB400000283FF424AB0A9C002C3EF468AC20464D
:10BB500026F0A0F9FEF763BC634D012285F8F020C2
:10BB6000FEF780BCC839884280F2378542FA0AF273
:10BB7000D1079B783FF535AC5A420120FFF7FCBB5B
:10BB8000099A01239370FFF78CBA58485849006806
:10BB9000B5F9F4C0C66981FB06018911F617701A60
:10BBA00000F5FF407F30844540F3238551490978F3
:10BBB000002900F01B815F2A00F05E856F2B7EF468
:10BBC000A7ACBCF5FA7FFEF6E6AC95F8F620002AA5
:10BBD0007EF4E1AC089B1B780121DC0785F8F610A8
:10BBE00000F1968517F074FD079BDFF820911B6824
:10BBF000FEF7D5BC10F0CEFF032140F6B8328BF82B
:10BC00002010CBF81C20FFF7A6BA3B4CFFF7B1BAC7
:10BC1000059931F91220B2F5617FC0F2668240F6D3
:10BC200033018A42A8BF0A460C2FA2F561729978A7
:10BC30004FF4966B9BFBF1FB92FBFBFB5FFA8BFBDC
:10BC400000F00485182F1BD15A46C82AA8BFC82265
:10BC5000D1B2286B90F817C08C4511D0B2EB0C0212
:10BC6000264BC17548BF0732D2109978531CDBB2FE
:10BC7000002940F0AF8213B1184626F027FA736806
:10BC80001B780C2B3FF4A5AB1D4B1E4A03EB87071B
:10BC90001D4BC3F800B0D7F880301360FFF799BB95
:10BCA000154C72882368642101FB0233CBF81030F5
:10BCB000B9F1000F3FF49CAAFFF78DBA012D7FF474
:10BCC000A4AA0D4CFFF769BA945D0020A8000020DB
:10BCD000EC00002000000000343900206833002010
:10BCE0001F85EB51065D0020E8240020D071002064
:10BCF000D34D6210E4000020D4900020E46F0020B7
:10BD0000DC100408D06F002070060020585D002071
:10BD1000002F4AD059F82320089E96424FEA43014B
:10BD2000FFF45EADCA4E725C06EB010E002A00F015
:10BD30009C80022A40F0A0809EF8012002EB820243
:10BD400002EB820202F2EE22012606FA03FE0B9EAD
:10BD500026EA0E0612B20B96002D3FF445ADBD4EFD
:10BD600001EB030A06EB4A0E0D9E2EF80620BBF1EE
:10BD7000000F03D10F9E022E7FF636ADB54EBEF8F2
:10BD80000220BEF804E036F81AA072449244B24A87
:10BD90000FFA8AFA82FB0A62B04EA2EBEA7226F828
:10BDA00001A012B24FF0010B1EE53A4659000A9E5F
:10BDB00049F8236015E5A64E325C06EB0008002A20
:10BDC0004AD0022A4FD198F8012002EB820202EBFE
:10BDD000820202F2EE2212B23AE5DCB2022C40F20A
:10BDE0007081032C7FF4BAAD4446A9E500219C483C
:10BDF00022F0B0FB002800F05981002385F8F730CD
:10BE000017F066FCFEF784BB964B974A109201220E
:10BE10001A70964B05931B21914822F09BFB00283A
:10BE20007FF45CAD9248DFF854B2C168DBF80030B3
:10BE3000079A8360126809905B1AC82B02F480523B
:10BE40007FF692AD8B490B6823F004030B60884B9F
:10BE5000012083F8210087E5DAB2022A40F2D1837B
:10BE6000032A00F04D810A5AB5E7DAB2022A40F2FD
:10BE7000CB83032A00F04A81625A65E746F001034A
:10BE8000B342A9F800303EF446AC7B4B41F202418C
:10BE9000FF2219809A700E2025F0FCFFB9F800608F
:10BEA00033B223F002039BB2B342A9F800307EF410
:10BEB0003AACFEF743BC0024FFF704B900230DE0C1
:10BEC0009CF8014004EB840404EB840404F2EE24A7
:10BED0000133834225F8024B3FF446AD11F813407D
:10BEE00001EB430C1CB1022CEAD02C88F0E7DCB249
:10BEF000032CFAD87446EBE710F04CFE032240F610
:10BF0000B8338BF82020CBF81C305C4CFFF723B9FA
:10BF10005B4A1278002A7FF417A9002F3FF414A976
:10BF2000012D7FF410AE9BF82030FFF7D5B8099BA8
:10BF3000DB78002B7FF46BAADFED527A524978EE62
:10BF4000677AC5F5FA63FDEEE77A1AB217EE903A12
:10BF50001BB21B0381FB0301DB17C3EBA11302FB25
:10BF600003F343F30F332B4407EE903AB8EEE78A1E
:10BF700086ED038AFFF74BBA444B03F1640703E0F5
:10BF800005339F4200F09F801A78262AF8D19978CD
:10BF9000DA789142F4D2FFF749B9591D9BF80500B0
:10BFA00010F03AFE00283EF4EDAE012D40F064841E
:10BFB0000BF10D019BF80A0010F02EFE002840F056
:10BFC000578433499BF80F0010F026FE00283EF4FA
:10BFD000ECAE032D40F048842E499BF8140010F07D
:10BFE0001BFE002840F03C842B499BF8190010F000
:10BFF00013FE00283EF4ECAE052D40F02D842749B9
:10C000009BF81E0010F008FE002840F0218424490F
:10C010009BF8230010F000FE00283EF4ECAE072D44
:10C0200040F012841F499BF8280010F0F5FD00280D
:10C0300040F006841C499BF82D0010F0EDFD00280F
:10C040003EF44BAC092D3EF448ACFEF7E7BE00BF12
:10C050000D3900207425002056555555BC2500206B
:10C06000683300207033002051350020705E0020BE
:10C07000A85E0020CC5E002034390020D49000203F
:10C08000C442002000007A44D34D62109C35002049
:10C09000D2320020D7320020DC320020E1320020F2
:10C0A000E6320020EB320020F0320020089BBB4A31
:10C0B0001B781060DE0700F1AA82079B1B68FEF761
:10C0C0002DBA74463CE4B64A069BD4881B8B1A1BD7
:10C0D000AA4221DA2344AB42CCBF00240124FEF75C
:10C0E000AEB9B04B0693FFF708BB0C2F00F0AC8243
:10C0F000182F40F009834FF0000B59465A46A8E527
:10C10000DDE91426002E08BF3A4664E6DDE9142670
:10C11000002E08BF3A4617E60124FEF790B9002129
:10C12000A14822F017FA00287FF4B8AA322385F834
:10C13000F800A5F84430FFF7B1BA002B40F04F8368
:10C140000B2010F0A1FD07F02003002840F0198318
:10C15000964E002B40F0E482954D95F8FA305BB393
:10C16000BAF1000F7FF472AAFEF72ABBB0EE670A9D
:10C1700081E4904A904910684FF47A72B2FBF0F271
:10C18000C2EB421002EB8002D200A1F8A4201906F3
:10C190007EF503AA894A127892077EF5FEA9884A9D
:10C1A000127D042A7EF6F9A92BF03CFF079BDFF8ED
:10C1B00018921B68FEF7F3B90D2025F06BFE0123E2
:10C1C00085F8FA30B9F80070BAF1000F7FF43EAA92
:10C1D000FEF7F6BA594618200E9316F037FA0E9B62
:10C1E00049E5784B0D999B7891F807B09344BBF1E2
:10C1F000640FA8BF4FF0640B2BEAEB7B81F807B00C
:10C20000002B40F04683286B10F046F9736837E541
:10C210006C4B0D999B7891F804B093448BF3080B09
:10C2200081F804B0002BEED01A20594616F00EFA11
:10C23000286BE9E7286B634B90F836B09B78934402
:10C24000BBF1640FA8BF4FF0640BBBF1010FB8BF87
:10C250004FF0010B80F836B0002BD5D0594617208F
:10C2600016F0F4F9CFE7286B564B90F837B09B786F
:10C270009344BBF1FE0FA8BF4FF0FE0B2BEAEB7B04
:10C2800080F837B0002BBFD01620594616F0DEF9E3
:10C29000286BB9E70D994B4B91F805B09B78934407
:10C2A0008BF3080B81F805B0002BACD01520594654
:10C2B00016F0CCF9286BA7E7286B424B90F802B038
:10C2C0009344BBF1C80FA8BF4FF0C80B2BEAEB7B20
:10C2D00080F802B09B78002B96D01420594616F0B7
:10C2E000B5F9286B90E7286B364B90F801B0934472
:10C2F000BBF1C80FA8BF4FF0C80B2BEAEB7B80F84F
:10C3000001B09B78002B3FF47FAF1320594616F005
:10C310009DF9286B78E7286B2A4B90F800B093447E
:10C32000BBF1C80FA8BF4FF0C80B2BEAEB7B80F81E
:10C3300000B09B78002B3FF467AF1220594616F0EF
:10C3400085F9286B60E71F4B0D999B7891F809B030
:10C3500093448BF3080B81F809B0002B3FF453AFE3
:10C360000E20594616F072F9286B4DE7286B154BD5
:10C3700090F808B09B789344BBF1C80FA8BF4FF06A
:10C38000C80B2BEAEB7B80F808B0002B3FF43CAFE6
:10C390000B20594616F05AF9286B35E79C430020CC
:10C3A000603B00203C90002068330020085D0020A6
:10C3B000E8240020389A0020CC9100209C5E0020C8
:10C3C00018A90020E46F0020585D0020286BC84B9E
:10C3D00090F807B09B789344BBF1C80FA8BF4FF00B
:10C3E000C80B2BEAEB7B80F807B0002B3FF40CAFB7
:10C3F0000A20594616F02AF9286B05E7286BBC4B32
:10C4000090F806B09B789344BBF1C80FA8BF4FF0DB
:10C41000C80B2BEAEB7B80F806B0002B3FF4F4AEA0
:10C420000920594616F012F9286BEDE6286BB04B3F
:10C4300090F805B099789344BBF1C80FA8BF4FF0AE
:10C44000C80B2BEAEB7B80F805B041B111205946AF
:10C45000CDE90E2316F0FAF8DDE90E23286B112F33
:10C460007FF42CAFD0E6286BA14B90F804B09978FC
:10C470009344BBF1C80FA8BF4FF0C80B2BEAEB7B6E
:10C4800080F804B041B110205946CDE90E2316F0D2
:10C49000DDF8DDE90E23286B102F7FF426AFB3E61D
:10C4A000286B934B90F803B099789344BBF1C80F75
:10C4B000A8BF4FF0C80B2BEAEB7B80F803B041B16B
:10C4C0000F205946CDE90E2316F0C0F8DDE90E2302
:10C4D000286B0F2F7FF421AF96E60D99844B91F8CE
:10C4E0000BB09B7893448BF3080B81F80BB0002BB7
:10C4F0003FF489AE0520594616F0A8F8286B83E66C
:10C500000D987B4B90F80AB0997893448BF3080B05
:10C5100080F80AB039B159460D20CDE90E2316F046
:10C5200095F8DDE90E230D2F7FF40EAF6BE60D9924
:10C530006F4B91F801B00E939344BBF1640FA8BF09
:10C540004FF0640B2BEAEB7B81F801B016F098F802
:10C550000E9B9B78002B3FF456AE0320594616F0F5
:10C5600075F8286B50E60D98614B90F806B09978F5
:10C570009344BBF1640FA8BF4FF0640B2BEAEB7B35
:10C5800080F806B039B159461B20CDE90E2316F0CC
:10C590005DF8DDE90E231B2F7FF424AE33E60D9802
:10C5A000534B90F803B0997893448BF3080B80F8C1
:10C5B00003B039B159461920CDE90E2316F046F8DB
:10C5C000DDE90E23192F7FF424AE1CE6286B0FF053
:10C5D00063FF4FF0FF3BFEF7FCBE012303FA0AF3B3
:10C5E00022EA030204F5FA7385F8F920B360FEF736
:10C5F000F8BE891B8C440FFA8CFCA5F8F4C0FFF739
:10C60000D5BA149AFFF7E7BB149AFFF79DBB394BD5
:10C610001B78002B3DF4BFAF099BDB78002B7DF42A
:10C62000BAAF95F8F7300133DBB2032B85F8F7305A
:10C630007DF6B1AF304B5B7813B9002C7DF4ABAF16
:10C6400016F0DAFBFDF764BF4FF0000B2B49497879
:10C6500059453FF415AB264B0F935846CDF838B0EB
:10C6600017F046FD0F9B0E9A9B78002B40F0088137
:10C67000531CDBB2FFF7FFBABCF5FA7FFDF68BAFB8
:10C6800095F8F630002B7DF486AF089B1B780122CD
:10C6900013EA020485F8F62019D016F0ADFB079BCB
:10C6A000DFF860901B68FDF77ABFC5F5FA6212B239
:10C6B00003FB02F343F30F332B4407EE903A104B86
:10C6C000F8EEE77A1870C6ED037AFEF7BDB90F20D1
:10C6D00025F0E0FBB5F8F43085F8F640FA3BA5F814
:10C6E000F430079BDFF81C901B68FDF758BF00BFB4
:10C6F000E46F0020065D002014350020EC9000203F
:10C70000F4420020585D00204FF0000BFFF7B8BA4C
:10C71000B149079B0A601B68DFF80093FDF73FBF34
:10C72000202026F039FEAD4B00221A70AC4D95F852
:10C73000FA302BB90D2025F0ADFB012385F8FA3036
:10C74000B9F80070FEF782BFA64AA749A74B11604F
:10C75000022001221A7025F0B9FC079BDFF8BC9279
:10C760001B68FDF71CBF9F4AA14911609F4B022225
:10C770000320EFE79B4A9F4911609C4B0022012058
:10C78000E8E79D4A9D4E528996ED007A07EE902A81
:10C79000F8EEE77AB0EEC77AB4EEE77AF1EE10FA87
:10C7A0007FF5D7AC96ED017AB0EEC77AF4EEC77A92
:10C7B000F1EE10FA7FF7CDAC002B7FF4CDAC20204A
:10C7C00026F002FED5E900238D490A60084641F8AB
:10C7D000043F2CF023FD814B01221A70A6E71020A4
:10C7E00026F0DAFD7D4BB9F8007083F800A04FF019
:10C7F000010AA5E4102026F0E7FD202026F0CCFD5C
:10C8000080497E4E081F2CF009FD744B02221A70DD
:10C810008CE70A9C4FF48060B9F1000F36D026F007
:10C82000D3FD099A00231361FFF78EB9A346099936
:10C83000DBF80020CB690A9C13448B61FFF784B9B5
:10C8400008221346FEF7ECBA07221346FEF7E8BAB1
:10C8500006221346FEF7E4BA05221346FEF7E0BAB5
:10C8600004221346FEF7DCBA03221346FEF7D8BAB9
:10C8700002221346FEF7D4BA01221346FEF7D0BABD
:10C8800059460C2015F0E2FE0E9AF1E626F084FDE2
:10C89000C7E71C20594615F0D9FE286BB4E4FCF715
:10C8A0003BFA95F8F210FDF75ABE0022A1F1B7034A
:10C8B0001892072B00F2B480DFE803F077B2B2B22F
:10C8C00073B26E495049079B0A781B6842F0040214
:10C8D0000A70FDF762BE4D4A079BDFF840911B6866
:10C8E0004FF4C8711180FDF75ABE95F8611095F8A4
:10C8F000F83009BB83F0010385F8F830002B62D1D2
:10C900000C2025F0C7FA079BDFF810911B68FDF794
:10C9100046BE002B4ED1324D95F8F130002B3DF440
:10C92000A7AD25F09BFA002385F8F130FDF7A0BDF7
:10C93000002CF0D1FEF7EBBA85F8612085F8620093
:10C94000DFF8D890002B3EF4A9AEFEF79BBE022381
:10C95000ADF860302E4BBDF862009989DA89BDF8D8
:10C960006040024421449981DA810AF00DF822F0F6
:10C970009DFD09F0AFFFFCF727F8012025F0A6FB8D
:10C98000B5F8F420079BFA3A00211B68A5F8F420BB
:10C9900085F8F610FDF703BE4FF6FE73ADF8603074
:10C9A000D8E70223ADF86230D4E74FF6FE73ADF856
:10C9B0006230CFE71749184A09684FF47A7000FBD4
:10C9C00003131360A7E70B2025F064FA079BDFF839
:10C9D0004C901B68FDF7E3BD9C4300200C840020B5
:10C9E000E824002054610020E27F0020EC90002029
:10C9F00030800020947F00209C840020085D00206F
:10CA0000B07C0020048400209C5E00208243002033
:10CA10000C2D0020D490002098430020585D002069
:10CA20009E2903D10021012033F0D2FB95F8F2308A
:10CA30009D2B03D10021FF2033F0CAFB95F8F23083
:10CA4000AE2B03D10121002033F0C2FB95F8F23068
:10CA5000AD2B03D1FF21002033F0BAFB95F8F23063
:10CA6000EF2B2BD0FD2B26D0FB2B21D0FE2B1CD067
:10CA7000F72B0AD07B2B04D14FF4FA61022017F078
:10CA80004FFA079B1B68FDF78ABD0021042017F0B1
:10CA900047FAB5F8F420079B963A00211B68A5F8E1
:10CAA000F42085F8F610FDF77ABD00210320EEE7AB
:10CAB00000210220EBE700210120E8E700210846E1
:10CAC000E5E7114D16F098F985F8F140FDF7D0BC77
:10CAD000022017F00DFB079B1B68FDF760BD0320CC
:10CAE00017F006FB079B1B68FDF759BD002017F0E8
:10CAF000FFFA079B1B68FDF752BD012017F0F8FAFB
:10CB0000079B1B68FDF74BBDE82400202DE9F84F7B
:10CB10000746264E264DFDF7FBFB264A2649DFF841
:10CB20009CC04FF0100E4FF47A744FF001086B6800
:10CB3000C3F30803CBB9EFF31183B3B91368D1F88A
:10CB400008A000BFD2F800904B45F7D1D6F800906E
:10CB500004FB09FBABEB0A0ABAFBF9FA04FB03A3DB
:10CB60001B1ABB42E3D3BDE8F88FEFF3118A8EF3B3
:10CB70001288D1F808B00B68DB0344BFCCF8008002
:10CB8000D1F808B01368DCF800905FFA8AFA8AF3EB
:10CB90001188D6F800A04B4404FB0AF9A9EB0B0955
:10CBA000B9FBFAF904FB0393DAE700BFD890002041
:10CBB00000ED00E0D490002010E000E0D0900020D4
:10CBC0002DE9F84F2A4C2B4E2B4D2C4F804618F157
:10CBD000FF384AD3FDF79CFB29494B68C3F3080390
:10CBE0004FF0100C4FF47A724FF0010EEBB9EFF3E7
:10CBF0001183D3B92368D5F808A000BFD4F80090FA
:10CC00004B45F7D1D6F8009002FB09FBABEB0A0AC3
:10CC1000BAFBF9FA02FB03A31B1AB3F57A7FD6D24B
:10CC20004B68C3F30803002BE1D0EFF3118A8CF3B8
:10CC30001288D5F808B02B68DB0344BFC7F800E0C2
:10CC4000D5F808B02368D7F800905FFA8AFA8AF31B
:10CC50001188D6F800A04B4402FB0AF9A9EB0B0996
:10CC6000B9FBFAF902FB0393D6E7BDE8F88F00BFE2
:10CC7000D4900020D890002010E000E0D090002058
:10CC800000ED00E030B4EFF31183102282F312883C
:10CC90000649074C0A680748013200250A602560EA
:10CCA000DBB2026883F3118830BC7047D490002057
:10CCB000D090002010E000E00E4B1B88014643B9E5
:10CCC0000D4B0E4A1B7810680BB981F001011FF063
:10CCD000F5BA0B4B5A691AB11A6810B9106058743A
:10CCE000704708480849008891FBF0F10120116065
:10CCF00058747047AC900020AE900020B090002097
:10CD0000B4900020CC90002020A1070038B5254B1E
:10CD10005C69626BA36D62B1A26BC2B1998A1A8819
:10CD2000C90592B204D5D20744BF4FF6F7721A80F4
:10CD300038BD99891A88890692B2EDD59206EBD54D
:10CD4000E26AFAB19888216B9047A36DE4E799896C
:10CD50001A880D0692B2E1D51006DFD5D4E9091282
:10CD60008A420AD0A1692569885C98800132B2FBA9
:10CD7000F5F105FB1122A262D0E7DA6822F0800209
:10CD8000DA60CBE79B88E2696169DBB28B54E269C8
:10CD9000E068A36D0132B2FBF0F100FB1122E26109
:10CDA000BAE700BF0851002038B5254B9C68626B7C
:10CDB000A36D62B1A26BC2B1998A1A88C90592B2F9
:10CDC00004D5D20744BF4FF6F7721A8038BD99894F
:10CDD0001A88890692B2EDD59206EBD5E26AFAB1CD
:10CDE0009888216B9047A36DE4E799891A880D060E
:10CDF00092B2E1D51006DFD5D4E909128A420AD0F1
:10CE0000A1692569885C98800132B2FBF5F105FBC8
:10CE10001122A262D0E7DA6822F08002DA60CBE762
:10CE20009B88E2696169DBB28B54E269E068A36DBB
:10CE30000132B2FBF0F100FB1122E261BAE700BF60
:10CE40000851002038B5254B1C68626BA36D62B198
:10CE5000A26BC2B1998A1A88C90592B204D5D207C9
:10CE600044BF4FF6F7721A8038BD99891A8889062F
:10CE700092B2EDD59206EBD5E26AFAB19888216BB1
:10CE80009047A36DE4E799891A880D0692B2E1D51F
:10CE90001006DFD5D4E909128A420AD0A1692569B2
:10CEA000885C98800132B2FBF5F105FB1122A26289
:10CEB000D0E7DA6822F08002DA60CBE79B88E2698B
:10CEC0006169DBB28B54E269E068A36D0132B2FBA9
:10CED000F0F100FB1122E261BAE700BF0851002027
:10CEE000002A12DD70B504460D468E1823682046D0
:10CEF0009B6898470028F9D0236815F8011B1B6828
:10CF000020469847B542F1D170BD704703685B6A0F
:10CF100003B11847704700BF03681B6A03B1184785
:10CF2000704700BF03682DE9F041DD691DB12B4654
:10CF3000BDE8F0411847002A174611DD04460E46A9
:10CF40000F4400E023689B68204698470028F9D0EA
:10CF5000236816F8011B1B6820469847BE42F1D192
:10CF6000BDE8F08103689B69184700BF03685B69EF
:10CF7000184700BF03681B69184700BF0368DB68D8
:10CF8000184700BF03689B68184700BF03685B68C9
:10CF9000184700BF03681B68184700BF2DE9F04F12
:10CFA0002DED028B95B006461DF076F8034B1D78EB
:10CFB00035B115B0BDEC028BBDE8F08F305D0020BF
:10CFC000C54B1B685805F4D5C44B1B78012B00F0EA
:10CFD0005082C34B0393C34B1B78002B3BD0C24CF6
:10CFE000C24AD4F82432F31A934200F2BF82DFF827
:10CFF00048A39AF80070002F00F0B783BC4F3A683E
:10D000004AB3D4F8343240F6B731F31A8B4222D9FE
:10D0100094F83032002B00F0F08594F839C2B5490D
:10D0200094F838E20868013BDBB20CF1010C84F89B
:10D0300030325FFA8CFC002B00F06C8512F8011B7B
:10D0400084F839C201EB0E033A6084F83832FFF7F6
:10D05000A1FFC4F83462A84A039B12781B68012A16
:10D0600003F101030C9300F0B781A44B1B78002B54
:10D0700000F0C980DFF8C482D8F80030002B00F03F
:10D08000C280039B984CD3F800B0D4F85432ABEB79
:10D090000303632B40F2B780DFF8A4A2984FDFF8B8
:10D0A000A49241201CF0B2FBBAF9023087FB0320A6
:10D0B000DB17C3EBA00080B21CF08CFBBAF9003088
:10D0C00087FB0320DB17C3EBA00080B21CF082FBC0
:10D0D000BAF9043087FB0320DB17C3EBA00080B252
:10D0E0001CF078FB99F80010D8F80000FFF752FF09
:10D0F00094F858A21AF0010700F01785814B1B68BD
:10D100009F0671D5804B814F1B78980742F198801C
:10D110003B7D042B8CBF03230223049347201CF088
:10D1200075FB38681CF022FB78681CF01FFBFB893C
:10D13000774AD8F80000A2FB0323C3F3471A5146ED
:10D14000FFF728FF3A8999F8001064208AEA010362
:10D1500000FB02F089F800301CF008FB049B3F7DC7
:10D16000D8F8000043EA8707FFB23946FFF712FFFD
:10D1700099F80030D8F800005F40394689F800700F
:10D18000FFF708FF94F858A2BAF1000F2CD1614FB5
:10D190004F201CF03BFB38681CF0E8FA78681CF064
:10D1A000E5FA50461CF0E2FA0121D8F80000FFF73A
:10D1B000F1FE554A99F800301778D8F8000007F0CA
:10D1C0000107394683F0010389F80030FFF7E2FEDA
:10D1D00099F80030D8F800005F40394689F80070AF
:10D1E000FFF7D8FE94F858A24B4AC4F854B20AF19B
:10D1F0000103DBB2A2FB0312D20802EB8202A3EB13
:10D20000420384F85832454F97F800A0BAF1020F54
:10D2100000F04083DFF8308198F87430032B00F081
:10D22000FB833F4B1B78002B3AD0DFF82081D8F8E6
:10D230000030ABB32C4CFDF76BF8D4F8603204909F
:10D2400044F61F62C31A93422AD994F86632002B1F
:10D2500001F0F082013B84F8663294F86722002ADC
:10D2600001F0D381013A84F8672294F86A32002BE6
:10D2700000F0C086013B84F86A3294F86E72002F89
:10D2800000F0CE85013F84F86E7294F86F72002F23
:10D2900001F0D483013F84F86F72049BC4F86032BC
:10D2A000204B1B78002B40F0CB821F4B1B7843B1E7
:10D2B0000D4CD4F8B03303F50043E8339E4280F0C0
:10D2C00002811A4B1B78002B3FF473AE064F184CAB
:10D2D000184D07F574763BE0489A0020F561002070
:10D2E000D490002002620020E82400203F0D0300BB
:10D2F0006C61002064610020036200201062002045
:10D30000676666669C5D00209C5E002018A9002070
:10D310001F85EB5100840020CDCCCCCC4B2C0020C1
:10D32000186200208862002099620020226200209A
:10D33000286200202C6200207061002048610020DB
:10D34000945D00204C610020000000201C62002041
:10D350002068FFF71BFE00283FF42BAE2068FFF784
:10D360000DFE2B78804673B1013B20682B70FFF7D0
:10D370000DFE00283FF41DAE2068FFF7FFFD2B785F
:10D380008046002BF0D16B490322304633F017F969
:10D3900097F8D01387F8D383023911F0FF0100F01A
:10D3A0007182314432464FF6FF7312F8010B1B1A9B
:10D3B00091429BB2F9D11A0A1FFA88F89045C7D159
:10D3C00097F8D223DBB29A42C2D15B481BF088FFA8
:10D3D0002B7818442870BBE7584F386800283FF472
:10D3E00044AE574CDFF87C81AA46B3464FF00109A2
:10D3F0000025FFF7CBFD38B3D4F8406226BB386870
:10D40000FFF7BCFD83B27E2B00F01B8398F802204F
:10D41000002A40F03B8294F83C12002900F0DD81A4
:10D420001B2B84F83C22386840F02482FFF7AEFDC5
:10D43000002800F02383386888F80290C4F840522E
:10D44000FFF7A4FD0028D7D1FCF762FFD4F85032D3
:10D45000C01AB0F5FA7F55465E46FFF606AE0CAA36
:10D460003849D4F840021CF0EBF90023C4F84032EC
:10D47000FBE5354B1B68002B3FF4ABAD304C334A1A
:10D48000D4F81832F31A93427FF7A3ADDFF8D880AF
:10D4900094F81C32D8F80020C4F818620133DBB2CB
:10D4A000910784F81C3201F1968513F0070701F00B
:10D4B0001E85282B264B01F08B860393254B5E207F
:10D4C0001B68984787E594F8B433C4F8B063012B20
:10D4D00040F2DC8294F8B5231F49D01801EB80019B
:10D4E000013202F00102D1F8085184F8B523B5B138
:10D4F0001A4F0D970DF15009A7F1120849F8208D28
:10D5000048F2A502152331464846A4F8B82384F80A
:10D51000BA33A847002840F01C8494F8B433104A6A
:10D520000133A2FB0312520802EB42029B1A84F859
:10D53000B433C6E6B9280020B82800206061002076
:10D54000E824002022270020405D002047E8010059
:10D55000D4900020FC5A0020DC100408B5280020DC
:10D56000ABAAAAAA000000209C5D0020D34AD44B9D
:10D5700092F80AE0039AD4F8280217681B88D14A67
:10D580004FF47A71381A01FB0EF15FFA83FC002721
:10D590001B0A884282F81EC0D37782F814C05375E4
:10D5A0009770177180F0A782C749C8480B688968CF
:10D5B000DFF85CC3C64F9CF800C097F814B080FB3E
:10D5C00003E8DB1780FB010EC817C3EBA801117736
:10D5D0000912C0EBAE00BF4B51774FF4FA714FEA1E
:10D5E000202E82F82000518347F2305078211CF021
:10D5F000020F82F821E083F81AB0508482F82410D8
:10D6000000F03982D7F80080D7F804E0B249B34A75
:10D61000DFF800A381FB08094FEAE87C81FB0E01DB
:10D620004FEAEE70CCEBA95CC0EBA15002FB0C8181
:10D6300002FB00E202EB4202520001EB41010492C4
:10D6400049008AFB0129049A8AFB022A4FEAAA426E
:10D650000792B7F80EA0049A3F890CEB8C0C00EBF4
:10D6600080000CEB8C0C00EB8000CDF818C008900B
:10D670004FEAE17CD0174FEAA9494FEAD878984A97
:10D6800083F8098007F5FA77A9EB0C08BFB202FB13
:10D69000181905970699079F914A4FFA88FC0CEBD9
:10D6A000810C391A049FDFF87082BBF1050F084620
:10D6B000DFF868B202FB11710AEBCA0A089A4FEA56
:10D6C0008A0A4FEADE7E40B283F80EE000EB820267
:10D6D00088FB097EABFB0A7088FB0178814FDFF87D
:10D6E00040B2B7F800A09DF814705F751FFA8CFC6B
:10D6F00092B2059F83F80AC04FEAE9794FEAE171D7
:10D70000C9EB6E19C1EB6811BBF800E083F80C900F
:10D710004FEA1C284FEA122B4FEA90104FEA292CAF
:10D7200083F80B80DA7383F810B04FEA17274FEABB
:10D7300021284FEA10224FEA1A2B34BF4FF032094A
:10D740004FF0330983F80DC0597483F812809F7528
:10D75000D8711A7283F813A083F814B083F81B9061
:10D7600083F81CE0C4F8246241E4DFF8B891D9F8EA
:10D770000000FFF70BFCC0B2012810D90228DFF827
:10D78000A88140F0458298F80130002B41F04D848B
:10D79000D4F82C32F31AB3F57A6F81F01A86524F0F
:10D7A0003A68002A3FF457AC9AF80030002B7FF417
:10D7B00028AC4E4BD9F800001B689B781E3B012B10
:10D7C00041F22E84043002211CF070FB0122002360
:10D7D0008AF8002084F838323BE47D2B00F0118277
:10D7E00094F8462222B180F02003DBB284F846127E
:10D7F000B4F8442294F83B121A44062992B20BD88A
:10D800006018013180F84832A4F84422C4F840522C
:10D8100084F83B123868ECE5130A53FA82F2FF2AC7
:10D8200088F80290A4F8442240F02181304BC4F8DB
:10D830004032FCF76DFD0346C4F850323868D5E538
:10D840002C4C227832B12C4B2C491868FFF76AFB1C
:10D85000002323702A4F3C78002C69D0DFF8CCA03D
:10D86000DAF86050002D40F01781264B3D70C3F868
:10D87000A8631AE50D2B7FF4DEADA4F84422C4F8AA
:10D880004022B6E5FF224FF6FF7395E5C4F84062EB
:10D890003868AEE5FCF73CFD1B4B1B68A0EB030BA7
:10D8A00040F6B8339B4500F2D880184B1A793A2AD3
:10D8B00001F0C48300233B70B3E400BFE05A0020B2
:10D8C000445D0020306200204C5D00206766666683
:10D8D00018A900205C6200206BCA5F6B806967FF3B
:10D8E00040420F005C6100206C61002068610020F4
:10D8F00030270020F46100208C620020B4610020F9
:10D9000091620020E8240020502C0020102C0020E0
:10D910009C5E002083DE1B431F85EB51D34D6210BC
:10D92000B86F00206461002000000020A062002089
:10D93000BA4D2B78002B40F09781B94CB94DD4F8F3
:10D94000A8232978B84B93FBF1F313449E42FFF4CC
:10D95000ACACB64A94F8AC33C4F8A86312F80380B0
:10D9600018F0010F41F0EB8418F0020F41F0A88489
:10D9700018F0040F41F0688418F0080F41D0AC4B48
:10D98000AC4F0D930DF15009A3F13D0249F8202D44
:10D990004FF48851022223F8401C03F83E2C4846DD
:10D9A000396820F0B9F84846796820F0B5F8FB8965
:10D9B000A14A03EBC30399000531A2FB0131C1F376
:10D9C000CF01484620F0C0F83B8A03EB830359009F
:10D9D00089B2484620F0B8F8984B1B78980743BFA7
:10D9E000398901F57A7189B24FF47A71484620F08D
:10D9F000ABF80C9B3A7D591C0C9148461A701CF0F0
:10DA0000F0FA94F8AC332978013393FBF1F201FB7F
:10DA1000123384F8AC3348E4DFF84492D9F80000BC
:10DA2000FFF7A4FA00283FF4FCABD9F8000001216D
:10DA3000FFF798FA0222002388F874203B70FFF762
:10DA4000F0BB84F83A6284F83B6284F83C9288F830
:10DA50000260C4F840623868CBE4714AB2F85A32C6
:10DA600000210133A2F85A323970FFF7DABBC4F84B
:10DA700040523868BDE42D22DA7673E6C4F84002DD
:10DA800084F83A9288F802903868B2E46C4A02EB63
:10DA90008302D2F808512AE50024DFF8C891254610
:10DAA0004FF050080BE01C44EFF3118388F3128809
:10DAB000DAF86020944217DADBB283F311881AF89F
:10DAC00004B0601C594650441BF050FD0BF101039B
:10DAD0000028E8D049463A201BF0AAFC0BF1010BC4
:10DAE0000543EDB25C44DFE70022DBB2CAF86020F8
:10DAF00083F31188B9E6534B03991B780968C4F87E
:10DB00002812013B012B3FF64FAD102102239170EB
:10DB1000137149E50EF10103714684F839C284F8A6
:10DB20003832FFF737FAFFF794BA474B1A88D10516
:10DB300001F18182D00601F14984910601F1278526
:10DB4000570601F17B85100701F19185D10701F19D
:10DB50001C8612F0020F0CBF04230C233B493C4AE5
:10DB60000F78D27807F001070AB147F00207532077
:10DB700004931BF04BFE374A128802EB820202EB41
:10DB80008202900080B21BF025FE00201BF022FED6
:10DB9000314A32491288D8F80000C2EBC212520052
:10DBA00081FB023111444FEAE27ACAEB612A5FFA43
:10DBB0008AFA5146FFF7EEF999F80020049BD8F84D
:10DBC00000001F438AEA020A002189F800A0FFF73B
:10DBD000E1F93946D8F80000FFF7DCF999F8003090
:10DBE000D8F800007B40DBB2194689F80030FFF717
:10DBF000D1F994F858A2FFF7C7BA1CF08DF9FFF7D6
:10DC000028BA84F84692C4F840123868FFF7F1BB8E
:10DC10001CF072F9012388F80130C0E59062002001
:10DC2000E824002098620020A08601009462002071
:10DC3000B461002018A90020CDCCCCCC9C5E002083
:10DC4000DC1004086E5B0020585D0020045D00209D
:10DC5000A85E0020445D0020985E0020030820801C
:10DC60004C3600201DA002086449654B0093A1F1C9
:10DC70003F07644B644A0B9101F8404C0CA8634980
:10DC80000A9720F059F80A9F7B1C0A933C700A9B64
:10DC90002922591C0A911A700A9BEA22591C0A91DE
:10DCA0001A700A9BC822591C0A910CA81A7031F0EC
:10DCB00049FB00F101080CA942460A9832F07EFBAC
:10DCC0000A9A02EB080301330A9302F808400A9B00
:10DCD0005A1C0A921C700A9B5A1C0A921C700A9BBE
:10DCE0005A1C0A921C700A9B5A1C0A921C700A9BAE
:10DCF0005A1C0A921C700A9B5A1C0A921C700A9B9E
:10DD00005A1C0A921C700A9B5A1C0A921C700A9B8D
:10DD10005A1C0A921C700A9B5A1C0A921C700A9B7D
:10DD20005A1C0A921C700A9B5A1C0A921C700A9B6D
:10DD30000122991814A80A911A7050F8283DDB1B8B
:10DD40003B701CF04EF9324B2C70C3F8A863FFF700
:10DD5000ACBA0C9D454541F22A84A7F11302013D5E
:10DD6000002141F2210012F8013F81EA03231BB296
:10DD700099B2002BACBF4B0080EA41039BB219045F
:10DD800054BF5B0080EA43039BB21F0454BF5B0097
:10DD900080EA43039BB21E0454BF5B0080EA430346
:10DDA0009BB2190454BF5B0080EA43039BB21F047B
:10DDB00054BF5B0080EA43039BB21E0454BF5B0068
:10DDC00080EA43039BB2190454BF5B0080EA43031B
:10DDD000954299B2C7D148461FF0DCFE0D490C9D13
:10DDE0000D486D1A152DA8BF15252A4632F0E6FA02
:10DDF0000A4A94F8B4331570FFF791BBB461002060
:10DE0000F29000201047040818470408244704082B
:10DE1000E8240020A02800205C2A0020712A00208D
:10DE20006F4B94F876C2B3F90220B3F90010B3F93E
:10DE300004309FED6C6A84F80D7107EE103A039B75
:10DE400084F80CC11B680C938CF06A0383EA0313FB
:10DE500006EE901AD9B20B0983F0D50343EA0123E9
:10DE600083EAC1031BB283EA031AC3F307255342B3
:10DE70005FFA8AFA07EE903A85EA1A1545EA0A250A
:10DE8000F8EEE77AF8EEE66AB8EEC77A85EACA05F0
:10DE90000FFA85FA67EE867A66EE866A27EE067ACC
:10DEA00000208AF0C805CDED0E7ACDED0D6A8DED1E
:10DEB0000F7A10901190129085EA051E0DF130092D
:10DEC000B9E80F005FFA8EFECAF3072585EA1E1532
:10DED00045EA0E2585EACE05DFF814E12DB2AEE85D
:10DEE0000F0085F01E0799E8070087EA071A5FFA16
:10DEF0008AFAC5F3072787EA1A1747EA0A278EE83E
:10DF000007000CF10103C82287EACA07AEF1100529
:10DF10004FF005094FF01E0C41F6FE4184F86E9259
:10DF200084F80FC1A4F80A1184F80E2105F11C022F
:10DF300084F87632A4F8087115F8013B7B4083EA37
:10DF40000313DBB2190981EA172141EA032181EAAF
:10DF5000C3031BB29FB29542A4F80871ECD183F0C1
:10DF6000270383EA0313DBB23A0A82EA131282EA36
:10DF7000032282EAC3031BB29AB24FEA122CDDB22B
:10DF8000DFF868E0A4F8082184F82DC184F82C514A
:10DF900004F5857904F5957AD9F80000D9F80410CC
:10DFA000D9F80820D9F80C3077460FC709F11009C5
:10DFB000D145BE46F0D10C4FB9F80030AEF8003074
:10DFC00007F1240984F8C25284F8C3C217F8011F6C
:10DFD000D8F80000FEF7DEFFB945F7D1FFF755B9D5
:10DFE000945D002088C3E43A87270020882700201A
:10DFF000F8250020DC4B1B681922990684F86A2258
:10E000007FF53BA9D94BDA4F1B789A0741F1BB82C8
:10E010003B7D042B8CBF4FF003094FF00209FCF746
:10E0200077F93B8A3A890C9003EB83035B00ADF8E8
:10E030004A304FF47A703B688DF84C900E93B7F8E5
:10E040000EC0397D7B68ADF848C000FB02F20025A8
:10E050004FF0FF300DF130090D9510920F938DF8B0
:10E060004D101190CC46BCE80F00DFF814E3AEE889
:10E070000F009CE80F00AEE807007146182221F857
:10E080001C39059194F8761284F80F2181F07803F9
:10E0900083EA0313DAB2130983F0F60343EA022397
:10E0A00083EAC2031BB283EA0312D2B2C3F307238B
:10E0B00083EA121343EA022383EAC2031BB283F00A
:10E0C000C80282EA0212D2B2C3F3072383EA121310
:10E0D00043EA022383EAC2031BB284F80D5183F0A2
:10E0E000180585EA0515EDB2C3F30722481C82EA3C
:10E0F000151242EA052284F87602059884F80C117C
:10E1000082EAC505C82341F6FE620146A4F808511B
:10E110001E30A4F80A2184F80E3111F8013B6B403F
:10E1200083EA0313DBB21A0982EA152242EA0322C8
:10E1300082EAC3031BB29DB28142A4F80851ECD11C
:10E1400083F0180383EA0313DBB24FEA152B8BEA43
:10E15000131B8BEA032B8BEAC30B0FFA8BFB1FFA03
:10E160008BF3844AA4F808315FFA8BFB1B0A0692F2
:10E17000079384F82F3184F82EB1964604F58575FF
:10E1800004F5957A28686968AA68EB68F446ACE8F3
:10E190000F0010355545E646F4D12868CCF800004C
:10E1A000DFF8E8A19DF81C3084F8C4B20AF1260516
:10E1B00084F8C532D3461BF8011FD8F80000FEF7DB
:10E1C000E9FE5D45F7D1FCF7A3F894F876B20C9020
:10E1D0008BF06A0181EA0111C8B2010981F0D50111
:10E1E00041EA002181EAC00109B281EA0110624BD3
:10E1F000624DB3F904303A8984F80CB1C0B2C1F36E
:10E20000072181EA101141EA002181EAC00185FB62
:10E210000305DB174FF47A70C3EBA50500FB02F092
:10E22000D7E9002309B2ADF84A5081F0C805CDE91D
:10E230000D2385EA0513DBB2CDE90F00C1F30725F5
:10E240004FF0000E85EA1315CDF844E0ADF848E034
:10E2500045EA0325CC4685EAC305BCE80F00059FC7
:10E2600084F80DE12DB20FC785F0210383EA031373
:10E27000DBB29CE80700C5F3072585EA131545EADC
:10E28000032585EAC3053E4B059387E80700C823AD
:10E29000212141F6FE4284F80F11A4F80A2184F8E6
:10E2A0000E31374BA4F808510BF1010B194684F8D5
:10E2B00076B203F11C0211F8013B6B4083EA0313B1
:10E2C000DBB2180980EA152040EA032080EAC30384
:10E2D0001BB29DB29142A4F80851ECD183F06802C0
:10E2E00082EA0212D2B22D0A85EA121B8BEA022BB5
:10E2F0008BEAC20B0FFA8BFB1FFA8BF34FEA132E3C
:10E300005FFA8BFBA4F80831DFF868C084F82DE1D0
:10E3100004F5957384F82CB104F585750793EB68C3
:10E3200028686968AA6867460FC7079B10359D4231
:10E33000BC46F4D12B883B80069B84F8C2B203F123
:10E34000230584F8C3E2574617F8011FD8F80000E8
:10E35000FEF720FEBD42F7D10A4A94F876C20A4F72
:10E3600084F80CC114E000BF9C5D00209C5E00207E
:10E3700018A9002088270020945D00206766666643
:10E38000F825002000840020F225002087270020A7
:10E39000D2E900230D938CF0EB0383EA0313D9B287
:10E3A0000B0983F0C50343EA012383EAC1031BB2CF
:10E3B00083EA0311C9B2C3F3072383EA111343EAC3
:10E3C000012383EAC1031BB283F0C80585EA051562
:10E3D000EDB24FF0000EC3F30723CDF838E083EA27
:10E3E00015130C9299E8070043EA052383EAC50355
:10E3F0000FFA83F9059B84F80DE189F0310583E874
:10E40000070085EA0515EDB2C9F3072383EA151362
:10E4100043EA052383EAC50394F8105194F81101E7
:10E4200094F8121194F813211BB25D4085EA05158A
:10E43000EDB2C3F3072383EA151343EA052383EA06
:10E44000C5031BB2584080EA0010C0B2C3F30723D3
:10E4500083EA101343EA002383EAC00318B2414061
:10E4600081EA0113DBB2C0F3072181EA131141EA0B
:10E47000032181EAC30109B24A4082EA0212D2B200
:10E48000C1F3072383EA121343EA022383EAC20398
:10E4900094F8145194F8150194F8161194F8172172
:10E4A0001BB25D4085EA0515EDB2C3F3072383EA8D
:10E4B000151343EA052383EAC5031DB2684080EAC9
:10E4C0000010C0B2C5F3072383EA101343EA002308
:10E4D00083EAC0031BB2594081EA0111C9B2C3F3F8
:10E4E000072383EA111343EA012383EAC1031BB222
:10E4F0005A4082EA0212D2B2C3F3072383EA12130C
:10E5000043EA022383EAC20394F8185194F81901EC
:10E5100094F81A1194F81B211BB25D4085EA051589
:10E52000EDB2C3F3072383EA151343EA052383EA15
:10E53000C5031DB280EA050383EA0310C0B2C5F328
:10E54000072383EA101343EA002383EAC0031BB2C4
:10E55000594081EA0111C9B2C3F3072383EA1113B9
:10E5600043EA012383EAC1031BB25A4082EA021242
:10E57000D2B2C3F3072383EA121343EA022383EAE6
:10E58000C2031BB283F0270585EA0512D2B2C3F39A
:10E59000072585EA121545EA022585EAC2052DB24E
:10E5A000AAB20CF10103EDB24FEA122C4FF0310E7A
:10E5B00040F6FE40C82184F87632A4F8082184F899
:10E5C0000FE1A4F80A0184F81C5184F80E1184F8B4
:10E5D0001DC13868FB687968BA68B7F810E007F5BC
:10E5E000CB770FC7069BA7F800E003F1130984F867
:10E5F000B25284F8B3C21AF8011FD8F80000FEF72F
:10E60000C9FCD145F7D1FEF738BE8449039B087891
:10E610001B680A2184F86712002800F00286804FE8
:10E6200001283988079141F20381798805910228F0
:10E6300000F0C087B9880691032801F015810428ED
:10E64000B7F806B001F00A810528398901F0018187
:10E650000628B7F80A9001F0F8800728BD8901F074
:10E66000C580B7F80EE094F876A20C938AF03003D8
:10E6700083EA0313DBB218096A4A84F80CA180F01C
:10E680007A00128840EA032080EAC3036648C2EB9E
:10E69000022280FB02701044D217C2EB602207985E
:10E6A0008DF845204FF0000C60F30F0C0698002702
:10E6B00060F30F0700201BB261F30F00002165F328
:10E6C0000F0183EA0315C3F307230693059B69F340
:10E6D0001F4063F31F4C6EF31F416BF31F47069BF4
:10E6E000CDE90DC7EDB2CDE90F0183EA15134FF067
:10E6F00000098DF8449043EA05270DF1300EBEE87D
:10E700000F0087EAC5052DB285F0C80C474F84F885
:10E710000D918CEA0C1C5FFA8CFCC5F307250FC722
:10E7200085EA1C1545EA0C239EE8030083EACC0C1D
:10E730000FFA8CF383F0230247F8040B82EA0210ED
:10E74000C0B2C3F3072282EA101242EA002227F87D
:10E75000141982EAC0000AF1010A232541F2FE627F
:10E76000C82384F876A2A4F8080184F80F51A4F80D
:10E770000A2107F1160184F80E3117F8013B4340D6
:10E7800083EA0313DBB21A0982EA102242EA032267
:10E7900082EAC3031BB298B28F42A4F80801ECD1FD
:10E7A00083F0F40383EA0313DBB2020A82EA131252
:10E7B00082EA032282EAC3031BB29FB2DDB2D4F81D
:10E7C0000E11D4F81221D4F80A01D4F81631DFF86A
:10E7D00060C0A4F80871ACE80F00D4F81A01D4F8AE
:10E7E0001E11D4F8222184F826514FEA172EACE8E6
:10E7F000070084F827E104F29F2704F2BD2984F87A
:10E80000BDE284F8BC5217F8011FD8F80000FEF7EB
:10E81000C1FBB945F7D1FEF728BD00BF782B00201A
:10E82000705E0020985E002003082080F8250020FC
:10E83000882700207C4B1B6803F00802002A4AF658
:10E840000B4048F6034149F607454BF60F4204BF1B
:10E850000D46024613F0040F18BF154698064FF0F8
:10E86000190148BF45F4804584F8661248BF45F059
:10E87000200515F04FFC6D4B9979C5F3090300286D
:10E8800040F0D185002940F0C7858A464FF0FF3B14
:10E89000642094F876720C9587F0F10181EA0111F9
:10E8A000C9B20A0982F0E70242EA0122CDE90D531A
:10E8B00082EAC1054FF000092DB2ADF83EA0ADF8D7
:10E8C00040B08DF84E00ADF83C90CDF84290CDF8B8
:10E8D0004690CDF84A9085EA051C0DF1300EBEE851
:10E8E0000F005FFA8CFCC5F3072585EA1C1545EA85
:10E8F0000C2585EACC05DFF840C184F80D91ACE821
:10E900000F009EE80F002DB285F0C80E8EEA0E1E95
:10E910005FFA8EFEC5F30725ACE8070085EA1E15F1
:10E9200045EA0E2181EACE0109B22CF8023B81F0C2
:10E93000010585EA0515EDB2C1F30722614682EAB9
:10E9400015121B0C01F81E3942EA05224FF0010C8A
:10E9500082EAC50541F6FE70C82207EB0C03A4F855
:10E960000A0184F80FC184F80E2101F11F0084F818
:10E970000C71A4F8085184F8763211F8013B6B4011
:10E9800083EA0313DBB21A0982EA152242EA032260
:10E9900082EAC3031BB29DB28142A4F80851ECD1B4
:10E9A00083F07C0383EA0313DBB22D0A85EA131597
:10E9B00085EA032585EAC3052DB2ABB24FEA132ED3
:10E9C000EDB2DFF87090A4F8083184F830E184F8F3
:10E9D0002F5104F5857C04F5957ADCF80000DCF80D
:10E9E0000410DCF80820DCF80C304F460FC70CF19F
:10E9F000100CD445B946F0D1DCF8000038600C4F5B
:10EA00009CF8043089F8043007F1270984F8C552CE
:10EA100084F8C6E217F8011FD8F80000FEF7BAFA2A
:10EA2000B945F7D1FEF719BC9C5D0020705B002052
:10EA30008727002088270020F8250020914B1B689D
:10EA400005229B0684F86F2240F1F5838E4BDFEDA3
:10EA50008F6ADA891B8907EE902A07EE103AF8EEE2
:10EA6000E77AB8EE477A67EEA67A94F876A2884BF2
:10EA7000884AB3F90410B2F90620874D8748CDEDD6
:10EA80000D7A8AF0220383EA03135FFA83FC4FEACC
:10EA90001C13B2F5FA6F83F05903A8BF4FF4FA6262
:10EAA00043EA0C2383EACC03B2F57A7F1BB2B8BFEA
:10EAB0004FF47A72A2F57A7E83EA031C64225FFA2D
:10EAC0008CFCC3F3072302FB0EF283EA1C1EA5FB9A
:10EAD000023280FB0130CB174FF0000B4EEA0C25C1
:10EAE000C2F38F12C3EBA0030DF13009CDF830B0A3
:10EAF000CDF83CB08DED0E7A85EACC05ADF842201C
:10EB0000ADF84030CB46BBE80F002DB285F0C80C05
:10EB10008CEA0C1C5FFA8CFCC5F30725DFF894E146
:10EB2000DBF800B084F80CA185EA1C15AEE80F00F4
:10EB300045EA0C2585EACC031BB283F04A0585EA39
:10EB400005117046C9B2C3F3072282EA111242EAE4
:10EB5000012240F810B982EAC1050AF1010A4FF01A
:10EB60004A0E41F2FE4C0022C8230590014684F86B
:10EB700076A2A4F80851143084F80FE1A4F80AC171
:10EB800084F80D2184F80E3111F8013B6B4083EAC3
:10EB90000313DBB21A0982EA152242EA032282EA4F
:10EBA000C3031BB29DB28142A4F80851ECD183F09B
:10EBB000140383EA0313DBB22D0A85EA131585EAF1
:10EBC000032585EAC3052DB21FFA85FC344BD4F822
:10EBD0000E11D4F80A0106934FEA1C2ED4F8122124
:10EBE000D4F81631A4F808C1DFF8B4C0B4F822B1E3
:10EBF00084F825E1ACE80F00D4F81A01D4F81E110E
:10EC0000ACE80300EDB204F29F2AACF800B084F83F
:10EC1000245184F8BA52D34684F8BBE204F2BB25EF
:10EC20001BF8011FD8F80000FEF7B4F95D45F7D1D5
:10EC30001C4B1D4A1B781278013B12F00100DBB21D
:10EC400014BFC0214021172B03D8184A134493F84E
:10EC5000F070174B1A8895071ABF002341F0100176
:10EC6000012312F4027F18BF022312F0100F18BF05
:10EC7000062312F0200F18BF1023002840F0E9836C
:10EC8000032019E09C5D002018A900200AD7233C2E
:10EC9000945D0020705E0020D34D6210676666664A
:10ECA0008827002024350020045D0020DC100408A3
:10ECB000585D0020F825002094F876520C9385F0DA
:10ECC000460383EA0313DAB2130983F0920343EA9B
:10ECD000022383EAC2031BB283EA031C5FFA8CFCA3
:10ECE000C3F3072282EA1C1242EA0C2282EACC0217
:10ECF00012B282F0C80383EA03134FF0000CDBB2B8
:10ED00008DF83470C2F3072203278DF835C08DF8D3
:10ED100038708DF8361082EA13178DF8370099E8AD
:10ED2000070047EA032787EAC3031BB2DDF814E0B4
:10ED300084F80FC183EA0317AEE80300FFB2C3F300
:10ED4000072383EA171343EA072383EAC70394F8E8
:10ED5000107194F8110194F812118EF800201BB272
:10ED60005F4087EA0717FFB2C3F3072383EA17134D
:10ED700043EA072383EAC7031BB2584080EA001026
:10ED8000C0B2C3F3072383EA101343EA002383EAE4
:10ED9000C0031BB2594081EA0111C9B2C3F3072372
:10EDA00083EA111343EA012383EAC10394F813E1D0
:10EDB00094F8147194F8150194F8161194F8172129
:10EDC00084F80DC11BB28EEA030E8EEA0E1E5FFAA6
:10EDD0008EFEC3F3072383EA1E1343EA0E2383EA5E
:10EDE000CE031BB25F4087EA0717FFB2C3F30723C6
:10EDF00083EA171343EA072383EAC7031BB2584089
:10EE000080EA0010C0B2C3F3072383EA101343EA79
:10EE1000002383EAC0031BB2594081EA0111C9B241
:10EE2000C3F3072383EA111343EA012383EAC103EF
:10EE30001BB25A4082EA0212D2B2C3F3072383EA1A
:10EE4000121343EA022394F818E1D04F84F80C51CE
:10EE500083EAC2031BB28EEA030282EA0212D2B232
:10EE6000C3F3072383EA121343EA022383EAC203AC
:10EE70001BB283F0320282EA0212D2B2C3F307233A
:10EE800083EA121343EA022383EAC2031BB29AB253
:10EE900040F6FE10C8214FEA122C84F80E11DBB2A6
:10EEA0000135A4F80A01386884F8765284F81AC14A
:10EEB00084F81931A4F808217968BA68B7F80C9079
:10EEC000069D07F5CB7707C7103587F802E0A7F84E
:10EED000009084F8B0C284F8AF321AF8011FD8F855
:10EEE0000000FEF757F8AA45F7D1FEF7D6B9FF2084
:10EEF0001AF080F90378FF2B14BF90F901103946FE
:10EF000002201BF025F8FF201AF074F90378FF2B7C
:10EF100014BFB0F90810002103201BF019F89C4B16
:10EF20001B78042B4ED09B4FB4F81E223878DFF8A4
:10EF3000789292FBF0F300FB13239BB2B9F8002008
:10EF4000A4F81E32190189B2642303FB02034200B4
:10EF5000B3FBF2F341EA0321C3F30323194309B2DC
:10EF600006201AF0F5FF8C4AB4F81E32507AB9F830
:10EF7000001001330128A4F81E3200F06283137BD5
:10EF800001EB81011FFA81F9002B40F05183834F7F
:10EF9000A7FB09377F0939B23A201AF0D9FF64215B
:10EFA00001FB179189B27E4B0531A3FB0131C908E2
:10EFB0003B201AF0CDFFDFF8049299F80630002BC1
:10EFC00040F00083D8F800309A0600F16F8294F880
:10EFD0001C32FEF76EBADFF8E8A19FED728AAAF143
:10EFE00028092427B9F81430FAEC016A07EE103A20
:10EFF000F8EEE66AB8EEC77A3846C6EE877A013789
:10F00000FFB267EE887AFDEEE77A17EE903A19B212
:10F010001AF09EFF272FE5D194F81C32FEF745BA6F
:10F020000221FDF79FFFFEF7D1BBC4F82C6288F8E0
:10F030000170FEF7B4BB3B46FEF790BD9978049390
:10F04000184608F0A5F900287EF434AC5649DFF8DC
:10F050007481564A564C0988DFF86C919368C8F859
:10F060001C101168B4F85A22C8F83C00C8F86CB0FB
:10F07000C8F84C30C8F82C10D9F80000C8F85C204B
:10F08000FDF784FF834600287EF4C6A85146D9F8D0
:10F090000000FDF767FF049B94F85C22DB78069381
:10F0A000642A4FF0040388F8743000F0E78298F87F
:10F0B0007530DFF818B105941A0704BF0133DBB2CD
:10F0C000072B28BF0123180108EB0002C0B2117CF6
:10F0D000384A049011445A1C5FFA82FE4FEA0E101F
:10F0E0006FF00F0C4FF0000A0890334807928BF82E
:10F0F0000AA01AB20BF10D0A0CFB03F391F8E4100D
:10F10000049C099300EB0212D446107B93682043C1
:10F1100001298CF800000CF1010E0ED90239C8B299
:10F12000811C059C8C44714601F8013B61454FEA06
:10F130001323F9D101300594864423F06000517BFC
:10F140009DF81C3001430EF1010C082B8EF80010C5
:10F15000ACEB0A0000F01C830999089C114421447F
:10F16000049C097B04F1100E124C21445FFA8EF4CA
:10F1700091F8E410049401EB000EBEF1130F02F1BC
:10F18000100200F3058301330793BEE7F225002048
:10F190006E5B00204A5D0020E05A00201F85EB5185
:10F1A000CDCCCCCC00007A44445D00204C5D0020E6
:10F1B000E8240020DC10040804000020705B00201C
:10F1C000845D0020000000204C36002030A9002083
:10F1D0001A4603931768A24BDFF8C882A3FB0723E4
:10F1E0009B0BA8FB03214909C1EB0111A3EB810390
:10F1F000190209B20023172084F81C321AF0A8FE65
:10F20000984BA3FB07239B09A8FB03125209C2EBEF
:10F210000212A3EB820319B218201AF099FEFEF72E
:10F220004DB90546814601468346CDE90500079064
:10F230008646FFF718BADFED8C7AB0EE677A14E4F1
:10F2400001230493FDF76ABF884B0D93A3F1400996
:10F2500000212122A3F13D0A23F8401C89F8022055
:10F26000CDF830A00DF002FD814B824F824A1B8801
:10F27000002808BF1746590500F18C81DA0700F114
:10F28000DB817E4A13F0020F18BF1746384630F074
:10F2900059F8394683460246794831F08FF80AEB2F
:10F2A0000B0314A87749013340F8203D00225B1A74
:10F2B0000AF80B2089F801301AF093FEFEF75CBBC8
:10F2C0006A4B714ADFF8D49111880D9314AFA3F102
:10F2D0003D0247F8202D4FF4206C082223F840CC43
:10F2E000384603F83E2C1EF02FFCD9F80030674951
:10F2F000DA1781FB0313C2EBA30399B238461EF061
:10F3000023FC14F015FFD9F808900C9B4FEA194222
:10F31000591C0C911A700C9B4FEA1922591C0C9124
:10F320001A700C9B5A1C0C9283F800900C9B5A1C70
:10F330000C92187038461AF054FEFEF719BBDFF82D
:10F3400068919FED538AB9F9023007EE903AF8EED2
:10F35000E77A464B0D9367EE887A14AFFDEEE77AB5
:10F36000A3F13D0247F8202D17EE902A91B24FF4F9
:10F37000006223F8402C1E2203F83E2C38461EF073
:10F38000E3FBB9F9003007EE903AF8EEE77A384639
:10F3900067EE887AFDEEE77A17EE903A99B21EF0A2
:10F3A000D3FBB9F9043007EE903AF8EEE77A384625
:10F3B00067EE887AFDEEE77A17EE903A99B21EF082
:10F3C000C3FB38461AF00DFEFEF7CEBA3423FEF723
:10F3D000C5BB0123D9F8000088F80130FDF7CEFD48
:10F3E0000746D9F80000FDF7C9FD7A067EF4D7A9D3
:10F3F0008A2800F02B818E287EF4D1A99AF800305B
:10F40000002B7DF4FBAD234F234B3B602D2384F871
:10F4100030323A68FEF7C8B9204A8246B2F900B0E5
:10F420006420FFF736BA184A128802EB820202EB18
:10F4300082024FEA820A1FFA8AFA002940F001820A
:10F440004FF0FF3B059314F073FE059B40B2FFF7AE
:10F4500020BA134AD278002A0CBF042005202BE4DE
:10F4600073B2E745D34D621000000000B461002084
:10F47000585D0020FC460408F44604080C470408C4
:10F480007761002075610020445D00206766666634
:10F4900058A08B416C610020306200204C5D002040
:10F4A000A85E002089888888945D0020DFF8748336
:10F4B000D04F98F800309B0700F19980002109B2E5
:10F4C00001201AF045FD002109201AF041FD798A3A
:10F4D00094F81C223B7DB1F5967F08D902F00F020B
:10F4E000072A04D842F20F738B4228BF0B46DFF87D
:10F4F000389399F80820CAB1203B07EE903A9FED67
:10F50000BE7AF8EEE77AF6EE006A67EE877ABEEE2C
:10F51000007AF5EEC07AF1EE10FA58BFB0EE667AD6
:10F5200077EE877AFDEEE77A17EE903A19B205206A
:10F530001AF00EFD98F8002000239107CDE90A3358
:10F540002AD494F82032012B26D0B9F90030DFED0F
:10F55000AB6A07EE103AB9F9023007EE903AB8EE0E
:10F56000C77AF8EEE77A27EE267A67EEA67ABDEE3E
:10F57000C77AFDEEE77A0CA88DED0C7ACDED0D7A09
:10F580001AF0FEFC23E54FF00109FEF748BD2423E5
:10F59000FEF7E4BA9A4F79E6D7E9002301210AA8D9
:10F5A00084F82012CDE90A231AF0EAFC0FE50021C5
:10F5B000FEF711BC154691461146934606929646B3
:10F5C000FFF751B88F4F0A223B6893FBF2F32820D4
:10F5D00019B21AF0BDFCB9F80830002B4AD1B9684D
:10F5E00081F3100109B204201AF0B2FCEAE4F989AF
:10F5F000854B4FF4F369112009FB01F191FBF3F105
:10F6000009B21AF0A5FCFB89642109FB03F393FB03
:10F61000F1F393FBF1F201FB123109B219201AF058
:10F6200097FC98F80030398998073FF548AF45E7CF
:10F630003B7899FBF3F9AAE4744F27E61023FEF711
:10F640008DBA09B239201AF083FCB4E4704B1B6800
:10F650009B067EF5A4A89AF80030002B7DF4CEAC72
:10F660006C4F6D4B3B602D2384F83032D1E6202364
:10F67000FEF774BA14F05CFD01B2B4E794F85D32A1
:10F68000072B08BF84F85DB294F85D22DFF89CB1C7
:10F69000089208EB021A0BF10603DAF8041004933F
:10F6A000084607912FF04EFEDAF8082005925FFA1F
:10F6B00080FA10462FF046FEC3B20AEB0300089A08
:10F6C0000799079308308BF8070022F00F008BF89A
:10F6D0000A0002F00F0203EBCA008BF80D208BF832
:10F6E0000E0052460BF10F0030F068FE079B1A46E1
:10F6F000DDE904310AF10900184430F05FFE9BF89F
:10F70000073003F1010AC3B1013B0BF1070EDFF82B
:10F7100010C104985EFA83FE002310F8011F5940BF
:10F720008B00CA0883EA410302F018024B404CFAEE
:10F7300002F253408645DBB2EFD1049A06980AF8EC
:10F7400002302FF0A7FA94F85D320022013384F8DA
:10F750005D3284F85C229BF802305BB11BF8051027
:10F76000D9F80000FDF716FC01359BF80230EDB228
:10F77000AB42F3D894F85C320322013384F85C3254
:10F7800088F874203A70FEF749B90823FEF7E6B905
:10F79000C0B2821DD2B242F040018BF807101F495F
:10F7A000059C049102F1010EBAB1053001F1010A84
:10F7B0005AFA80FA8C4600221CF8010F5040820051
:10F7C00082EA4002C1084240154801F0180140FA9F
:10F7D00001F14A40E245D2B2EED1049906980EF802
:10F7E000012088F875302FF055FAB4E79646FEF7F9
:10F7F0003ABF00BF18A90020E4380E3F0050C347AD
:10F80000004704084C5D0020A0860100044704085E
:10F810009C5D00206C6100205C62002036A9002005
:10F820000007090E9C5E0020E05A002030A900204D
:10F830001546914611469346CDE905229646FEF7B8
:10F8400012BF0D4AB2F900B0FCE515469646FEF728
:10F850000ABF154691469646FEF705BF15469146E6
:10F8600011469646FEF7FFBE154691461146934651
:10F870009646FEF7F8BE00BF4C5D002038B50C463A
:10F88000097849B1054601342B6828461B6898471A
:10F8900014F8011B0029F7D138BD00BF064B53F8FF
:10F8A00020302BB11A689B8851690B4201D1138318
:10F8B00070475383704700BFA0900020036803F196
:10F8C0003F4202F57E022DE9F04F920A464DAA5CB6
:10F8D00002F01F0552090124032A04FA05F47ED020
:10F8E000042A77D0022A30D001F00306721E012AC2
:10F8F000C1F3810EC1F300188588C1F341114FF0A7
:10F9000000024FF0010C25D94FF0030E0CFA02F063
:10F91000A84315D150001F680EFA00F4E4432740B5
:10F920001F60D3F8008006FA00F747EA08071F6057
:10F93000DF683C40DC60DC6801FA00F02043D860FE
:10F940000132102AE2D1BDE8F08F284A556C2C43D1
:10F950005464C9E74FF003090CFA02F737EA0500CF
:10F9600033D15000D3F800A009FA00F4E4430AEAC6
:10F97000040AC3F800A0D3F800B006FA00FA4AEA75
:10F980000B0AC3F800A0D3F808A004EA0A0AC3F8D7
:10F9900008A0D3F808B00EFA00FA4AEA0B0AC3F836
:10F9A00008A0D3F804A02AEA07075F60D3F804A0F0
:10F9B00008FA02F747EA0A075F60DF683C40DC604C
:10F9C000DC6801FA00F02043D8600132102AC3D16C
:10F9D000BDE8F08F054A156B2C43146384E7034A96
:10F9E000156C2C4314647FE7E83E0408003802409D
:10F9F0002DE9F04F4A484B494B4B4C4C4FF0010A14
:10FA00004FF002094FF004084FF0080E4FF0100CB1
:10FA100020274026802530F8022B12F0010F03D05A
:10FA20001960A3F804A0083312F0020F03D0196084
:10FA3000A3F80490083312F0040F03D01960A3F860
:10FA40000480083312F0080F03D01960A3F804E013
:10FA5000083312F0100F03D01960A3F804C0083364
:10FA600012F0200F02D019609F80083312F0400F6F
:10FA700002D019609E80083312F0800F02D0196006
:10FA80009D80083312F4807F05D04FF4807B19608D
:10FA9000A3F804B0083312F4007F05D04FF4007BC4
:10FAA0001960A3F804B0083312F4806F05D04FF446
:10FAB000806B1960A3F804B0083312F4006F05D00E
:10FAC0004FF4006B1960A3F804B0083312F4805FA0
:10FAD00005D04FF4805B1960A3F804B0083312F42A
:10FAE000005F05D04FF4005B1960A3F804B0083341
:10FAF00012F4804F05D04FF4804B1960A3F804B086
:10FB00000833D20B04D04FF4004219609A800833B6
:10FB100001F58061A1427FF47EAFBDE8F08F00BFA8
:10FB20006C40040800000240AC8700200010024036
:10FB30002DE9F04FBF4B1D788BB0002D71D1BE4B1E
:10FB4000BE4C1E78DFF81083DFF810A3A4F10A077B
:10FB500006F0010607F26E2B54F80A0CC8B34FF0FA
:10FB6000CC0909FB0579FDF711FA90B354F80A0C9A
:10FB7000FDF704FA14F8023C024673B9242830D089
:10FB800054F80A0C002EEED1232A00F0AE819AF828
:10FB900032309342E7D11FF0BDFB012B27D0022B5F
:10FBA0002ED0032B00F00381042B00F05F81052B86
:10FBB00000F08B81062B20D114F801CCBCF1000F92
:10FBC00000F0DF81BCF1010F00F02D82002304F86A
:10FBD000023CCC345C4505F10105BDD10BB0BDE85C
:10FBE000F08F012304F8023C54F80A0CBBE74D28BF
:10FBF0000CBF0223002304F8023C54F80A0CB2E7BD
:10FC000000233C2804F8023C00F057813E28F4D140
:10FC10000122032304F8012C04F8023C54F80A0CD6
:10FC2000A1E7874B18680028D8D01DF0DDFBDFF86E
:10FC300030A2DFF82082DAF80000FDF7A7F90028EB
:10FC4000CCD0DAF80000DFF81C92FDF797F909280C
:10FC5000D9F800601AD03F2818D0002E6CD10428A3
:10FC600000F0DD810C2800F09B807F28E3D0A0F11C
:10FC70002003DBB25E2BDED82028DCD0731C08F812
:10FC80000600C9F800300BF095FAD4E7002E65D1D4
:10FC90006C4B354603F52077002D46D01033BB4220
:10FCA000FAD1DFF8C4B12868DBF80020845D935DE9
:10FCB0009C42304402EB060140F0AF81741E444484
:10FCC000324613B9FD2A40F2AB8004F8013F0132FD
:10FCD000C9F8002010F8013F11F8017F9F42F0D0D1
:10FCE0000AB15D4513D058480BF06CFA5D4508D851
:10FCF00055F8100B0BF066FA09200BF05BFA5D4526
:10FD0000F6D952480BF05EFAD9F800200026964248
:10FD100091D2741E444414F8010F0BF04BFAD9F839
:10FD2000003001369E42F6D385E703F11002BA4255
:10FD30001D46B6D01346AFE70C2831D00A283ED076
:10FD40000D283CD07F2800F0AE80FF2E3FF673AF29
:10FD5000A0F12003DBB25E2B90D96CE7394C4FF059
:10FD6000000B04F520775D4602E01034BC420DD054
:10FD70003246216840461DF03DFE0028F5D1A346DD
:10FD8000002DF2D125461034BC42F1D1002D8AD18C
:10FD9000BBF1000F3FF44FAF2B480BF013FAA7E76E
:10FDA0002B480BF00FFA29480BF00CFA43E7C02858
:10FDB00069D9002304F8023C54F80A0CD3E60BF08E
:10FDC00080FA2321234830F02AFC002868D0A0EBD9
:10FDD0000803C9F80030A3B15A1E18F802102029F0
:10FDE00040F04081023B43444AB113F801192029F5
:10FDF00002F1FF3040F0AA800246002AF5D1C9F88E
:10FE000000204FF480720021404630F0F1FB094B96
:10FE10001B78002B3FF4E2AE0C480BF0D3F90AE755
:10FE2000511C202008F80200C9F8001008F8013021
:10FE30000A4656E7305D0020045D0020C6B1002070
:10FE4000B83100200015040830470408384704087A
:10FE500040470408BC310020E824002068900020BE
:10FE6000B4310020BC3200207017040814F8043CA0
:10FE700004F8030C5A40052304F8042C04F8023C4F
:10FE800054F80A0C6FE60021042304F8050C04F86A
:10FE9000040C04F8061C04F8023C54F80A0C62E650
:10FEA000D9F8003097E7013E00237148C9F8006097
:10FEB00008F806300BF086F9BDE6032204F8013C91
:10FEC00004F8022C54F80A0C4DE614F8063C14F819
:10FED000050C14F8041C984200F293808A427FF4C7
:10FEE00068AF062304F8023C66E6624BDFF8B8C14F
:10FEF000DB78614A61491060003318BF01238CF838
:10FF000000305F4B5F4A0B6040235F4988F8E03365
:10FF10004FF0010CC8F8D823C8F8D403C8F8DC03A4
:10FF200088F8E163594881F800C00BF091FC58480B
:10FF30000BF048F94FF4006023F05EFA9AF8323083
:10FF4000232B3FF428AE14F8023C33E6C9F8002016
:10FF5000504C002304F5207708F8023003E01034F9
:10FF6000BC4200F081802168404608F07DFE0028F8
:10FF7000F5D0BC4278D2E36898470023C9F8003036
:10FF80003FE7454B06940FCB0DF1280E0DF1080904
:10FF900089E80F0014F8051C4EF824CD611814F8F8
:10FFA000033C0791724649464FF0010E06A8ADF892
:10FFB00022C0ADF820308DF824E023F025FA48B1B6
:10FFC000CC20029A354B494600FB0570CDE9023240
:10FFD00021F036F9DDF80490002304F8023CB9F171
:10FFE000000F3FF4F6AD54F80A0C21F0ADF9CC3413
:10FFF00054F8D60CC8475C4505F101057FF4ACAD5B
:020000040801F1
:10000000ECE509EB03005140013304F8041C04F84B
:10001000063C827254F80A0CA5E5324660E6204898
:1000200004F0E0FBDAE514F8053C14F8032C069420
:10003000234407936E2A4FF00003ADF82630CDF825
:100040002230ADF820207FF4C1AD06A81DF054FD8C
:1000500006A81DF045FD06A81DF042FD06A81DF0EE
:100060003FFDB3E51A4673E70E480BF0ABF884E7A3
:1000700068470408EC900020B4310020B83100201B
:10008000C0280020D1810008305D00206C470408A2
:100090003847040800150408F4110408B8BE00200D
:1000A000BC3100204C4704088C770020002301223B
:1000B000C27083700380037143718371C3710372D3
:1000C0004372704700230A2203604360C381C0F873
:1000D0000630C0F80A300280704700BF03788B42B8
:1000E00086BF024B33F81100002070470C29002016
:1000F000034B187E10B100221A760120704700BF12
:100100000C29002038B50446FAF702F9474B0022C3
:100110005A769A7E012A13D9DA6940F6AC51821ACE
:100120008A420DDD424A1278172A07D11A8C4149BA
:10013000013292B201251A844A808D8000229A767B
:10014000E2B27E2A23D0997E01B3997E1B2952D830
:1001500093F88410002963D0002182F0200283F8F4
:100160008410997E022903D1012A08BF83F87820E0
:1001700093F822109C7E987EC1EBC10103EB8101B4
:1001800021440130C0B281F82320987638BD9A7E90
:10019000012A2CD993F82220274993F823400132D1
:1001A000A1FB0251490801EB4101521AD2B294421B
:1001B0000BD09C7E93F8221083F82220C1EBC10162
:1001C00003EB8101621E81F83F2093F878202AB169
:1001D00001210022597683F87820D867144A1278D2
:1001E000172A17D00022C3F8800083F88420012248
:1001F0009A76D86138BD0E4A12780021172A99766E
:10020000C4D11A8C0B49013292B202201A844A805E
:10021000888038BDD3F880200649821A0A80E1E739
:100220007D2A9ED1012283F8842038BD0C2900202C
:100230009587002098870020ABAAAAAAF0B4BC4DED
:1002400095F8AB6005F188020244B41E1444A24242
:1002500000F06B81013A013C002341F2210112F8C8
:10026000017F83EA07231FB2BBB2002FACBF5B0044
:1002700081EA43039BB21F0454BF5B0081EA43033E
:100280009BB21F0454BF5B0081EA43039BB21F046F
:1002900054BF5B0081EA43039BB21F0454BF5B0061
:1002A00081EA43039BB21F0454BF5B0081EA43030E
:1002B0009BB21F0454BF5B0081EA43039BB21F043F
:1002C00054BF5B0081EA4303A2429BB2C7D10644FC
:1002D000B21E013E2A442E4492F8881096F88820D7
:1002E00002EB012292B29A4201D0F0BC704795F81D
:1002F000AC20002A00F01581431CDBB25C1C2C44AE
:100300002B444FF4AF6193F8886094F8883003EB86
:1003100006239BB201FB03F31B1303F54873012A69
:100320002B8000F0FE80C31CDBB25C1C2C442B44F1
:10033000022A93F8886094F8883003EB06239BB276
:1003400001FB03F34FEA233303F548736B8000F09E
:10035000E880431DDBB25C1C2C442B44032A93F839
:10036000886094F8883003EB06239BB201FB03F30B
:100370004FEA233303F54873AB8000F0D280C31DEE
:10038000DBB25C1C2C442B44042A93F8886094F85C
:10039000883003EB06239BB201FB03F34FEA2333C0
:1003A00003F54873EB8000F0BC8000F10903DBB279
:1003B0005C1C2C442B44052A93F8886094F8883000
:1003C00003EB06239BB201FB03F34FEA233303F550
:1003D00048732B8100F0A58000F10B03DBB25C1C9D
:1003E0002C442B44062A93F8886094F8883003EB59
:1003F00006239BB201FB03F34FEA233303F5487353
:100400006B8100F08E8000F10D03DBB25C1C2C448C
:100410002B44072A93F8886094F8883003EB06236E
:100420009BB201FB03F34FEA233303F54873AB811F
:1004300077D000F10F03DBB25C1C2C442B44082A5C
:1004400093F8886094F8883003EB06239BB201FB95
:1004500003F34FEA233303F54873EB8161D000F1D6
:100460001103DBB25C1C2C442B44092A93F88860EE
:1004700094F8883003EB06239BB201FB03F34FEAA9
:10048000233303F548732B824BD000F11303DBB207
:100490005C1C2C442B440A2A93F8886094F888301A
:1004A00003EB06239BB201FB03F34FEA233303F56F
:1004B00048736B8235D000F11503DBB25C1C2C4411
:1004C0002B440B2A93F8886094F8883003EB0623BA
:1004D0009BB201FB03F34FEA233303F54873AB826E
:1004E0001FD000F11703DBB25C1C2C442B440C2AF8
:1004F00093F8886094F8883003EB06239BB201FBE5
:1005000003F34FEA233303F54873EB8209D000F17C
:100510001903DBB25A1C2A442B4493F8883092F812
:10052000883001232B76F0BC70470023CFE600BF54
:100530000C290020794B5B68C3F3080370B5B3B98D
:10054000EFF311839BB9764A764D1368AC6800BF10
:1005500011688B42F9D1744A15684FF47A7101FB26
:1005600005F2141BB4FBF5F401FB034320E0EFF3A9
:100570001181102383F312886A4C6C4AA5682368A2
:10058000DE0344BF01231360654B48BFA5681E68A6
:100590001368C9B281F31188634A14684FF47A7101
:1005A000334401FB04F2521BB2FBF4F201FB0323C0
:1005B0005F4CD4F8B020C4F8B0309B1AB3F5FA5FA2
:1005C0001AD9002384F8B43084F8B530A1282FD08C
:1005D000A22800F09C8094F8B52094F8AB30002558
:1005E000A2B16A1C6119D5B2C0B29D4281F88800DF
:1005F00084F8B4500CD070BD94F8B450002DE5D000
:1006000094F8B52094F8AB30002AEAD19D42F2D19B
:1006100094F8B630052B72D0062B03D194F88930AC
:100620001E2B0DD0002384F8B43084F8B53070BD93
:1006300001221B2384F8B52084F8AB300025D0E7D5
:100640006A1E002A4FF0000150DD08460B46234485
:10065000013093F88830DBB283EA0105ED074FEAF9
:10066000530348BF83F08C0383EA5105EE074FEA3A
:10067000530348BF83F08C0383EA9105ED074FEAEB
:10068000530344BF83F08C03DBB283EAD105EE074A
:100690004FEA530344BF83F08C03DBB283EA1115A6
:1006A000ED074FEA530344BF83F08C03DBB283EAC8
:1006B0005115EE074FEA530344BF83F08C03DBB2BE
:1006C00083EA9115ED074FEA530344BF83F08C038F
:1006D000DBB283EAD1155908EB0748BF81F08C01E2
:1006E000C0B248BFC9B290420346B0DB224492F880
:1006F00088308B4296D10320FFF7A0FD92E70020BF
:10070000FFF79CFD94F889301E2B8BD198E70122CE
:10071000232384F8B52084F8AB308FE700ED00E0A8
:10072000D490002010E000E0D8900020D09000206D
:100730000C29002007299DBF034B03EB8101B1F871
:10074000B8000020704700BF0C2900201A4B93F816
:10075000D82032B193F8DC200021A82A83F8D810E1
:1007600001D00020704793F8EF20002AF9D110B48F
:10077000DFED126A03F1DC0103F1B40003F1EC02D6
:10078000B4EE047ACC780B7903EB042307EE903AAD
:10079000F8EEE77AB0EE666AA7EE876A02318A421F
:1007A000FCEEC67A17EE903A40F8043FEAD10120F9
:1007B0005DF8044B704700BF0C2900200080BBC3CC
:1007C00010B50446F9F7A4FD0F4BD3F8F420C3F895
:1007D000F400801A41F288329042E4B205D983F8DD
:1007E000DC40012283F8F82010BD93F8F820991816
:1007F000142A81F8DC4003D1012283F8D82010BDEF
:100800000132D2B2EEE700BF0C290020034B03EB0C
:100810004101B1F8FC00C008704700BF0C2900205E
:10082000724B93F81C21002A00F0C28070B493F838
:100830001D41B3F81E5103EB4401002091F82361E0
:1008400091F8242183F81C0142EA0622954202D045
:10085000002070BC704793F82121012A00F0AA8083
:10086000812AF6D10320102C40F2A68093F825416E
:1008700093F8235193F8241193F8262141EA052196
:1008800042EA04221024A3F8FC10A3F8FE2083F807
:100890001D4193F8271193F82821032C42EA0122E5
:1008A000A3F80021D5D093F8291193F82A21042C1C
:1008B00042EA0122A3F80221CBD093F82B1193F83E
:1008C0002C21052C42EA0122A3F80421C1D093F87F
:1008D0002D1193F82E21062C42EA0122A3F80621BD
:1008E000B7D093F82F1193F83021072C42EA012258
:1008F000A3F80821ADD093F8311193F83221082CD8
:1009000042EA0122A3F80A21A3D093F8331193F805
:100910003421092C42EA0122A3F80C2199D093F842
:10092000351193F836210A2C42EA0122A3F80E2150
:100930008FD093F8371193F838210B2C42EA01221B
:10094000A3F8102185D093F8391193F83A210C2C93
:1009500042EA0122A3F812213FF47BAF93F83B1146
:1009600093F83C210D2C42EA0122A3F814213FF414
:1009700070AF93F83D1193F83E210E2C42EA01220C
:10098000A3F816213FF465AF93F83F1193F8402187
:10099000102C42EA0122A3F818217FF45AAF93F8F1
:1009A000411193F8422142EA0122A3F81A2150E7AB
:1009B00000207047104656E7002C3FF44AAF93F8EA
:1009C000231193F82421012C42EA0122A3F8FC20F0
:1009D0003FF43FAF93F8251193F82621022C42EA09
:1009E0000122A3F8FE207FF454AF32E70C29002047
:1009F000654B5B68C3F3080370B4B3B9EFF31183BD
:100A00009BB9624A624D1368AC6800BF11688B42A3
:100A1000F9D1604A15684FF47A7101FB05F2141B95
:100A2000B4FBF5F401FB034320E0EFF31181102345
:100A300083F31288564C584AA5682368DE0344BFE6
:100A400001231360514B48BFA5681E681368C9B2E3
:100A500081F311884F4A14684FF47A71334401FBD3
:100A600004F2521BB2FBF4F201FB03234B49D1F811
:100A700048219A1AB2F57A6F17D891F84C21C1F82B
:100A80004831BAB1022A20D0242A91F81D3178D9F0
:100A900001320233D2B25B009A4281F84C211CDB56
:100AA00001339A4265D070BC70470022C1F84831CA
:100AB00081F84C21A828F6D1002281F81C21A1F848
:100AC0001E2191F81D31044603E0C4B281F81D4196
:100AD00023468D1885F82041DAE7B1F81E31C0B2FF
:100AE00083EA002000B20028B8BF41F2210283B29D
:100AF000B4BF82EA43035B009BB2180446BF41F2D5
:100B0000210282EA43035B009BB21A0446BF41F212
:100B1000210282EA43035B009BB21E0446BF41F2FE
:100B2000210282EA43035B009BB21D0446BF41F2EF
:100B3000210282EA43035B009BB21C0446BF41F2E0
:100B4000210282EA43035B009BB2180446BF41F2D4
:100B5000210282EA43035B009BB21A0446BF41F2C2
:100B6000210282EA43035B009BB2A1F81E3170BCF4
:100B700070470022012381F84C2181F81C3170BCA0
:100B80007047C4B2A5E700BF00ED00E0D49000209C
:100B900010E000E0D8900020D09000200C29002028
:100BA000F8B5124D95F8652102B9F8BD104B1C68D7
:100BB0002368DE693EB1204605F5A871B0470023E1
:100BC00085F86531F8BD05F5A877BE1800E0236803
:100BD0009B68204698470028F9D0236817F8011B26
:100BE0001B6820469847B742F1D1E8E70C2900205E
:100BF0009C62002003788B4210D9094B03EB8101E2
:100C000093F89831D1F868011BB900F5777080B27C
:100C10007047400800F5777080B270470020704739
:100C20000C290020324B5B68C3F3080370B4B3B9DE
:100C3000EFF311839BB92F4A2F4D1368AC6800BFA7
:100C400011688B42F9D12D4A15684FF47A7101FB76
:100C500005F2141BB4FBF5F401FB034320E0EFF3B2
:100C60001181102383F31288234C254AA568236839
:100C7000DB0344BF012313601E4B48BFA5681E68F9
:100C80001368C9B281F311881C4A14684FF47A7151
:100C9000334401FB04F2521BB2FBF4F201FB0323C9
:100CA000184AD2F89C11C2F89C315B1A41F2883183
:100CB0008B420AD9C0B2012382F8A40182F8A03184
:100CC000002382F8B43170BC704792F8A0310F2B2A
:100CD000F9D8D1180133DBB2C0B2102B81F8A401CE
:100CE00082F8A031ECD1012382F8B43170BC704796
:100CF00000ED00E0D490002010E000E0D89000204B
:100D0000D09000200C290020C36833F8110000EBBC
:100D10008000C01000F55C7080B27047036993F8E2
:100D20002320002A00F0C3802DE9F043714ADC7DC6
:100D300012780021162A04F0040604F0080583F84E
:100D4000231000F0B680002E40F0BE801DB11A8C3A
:100D500042F001021A8493F80290997993F801C045
:100D6000C268DE7893F80480DF7909F0070001F0AB
:100D70000F014FEAC11E4CEA002106F03F06187A27
:100D80001180997893F80AC0760146EAD106D9789D
:100D900056804FEA880848EA911193F805809E7BB7
:100DA00008F0010841EA8821918059794EEA510101
:100DB000D18007F07F07997993F807E03F0147EA70
:100DC0001117597A1781400040EADE1001F0030143
:100DD00040EA41205F7BD97A50810CF01F0C587A91
:100DE0004FEA8C1C4CEA90009081187B93F80AC063
:100DF00007F0070740EA072006F03F065F7B1082F6
:100E0000C90041EA5C117601D18146EAD7015182DD
:100E1000D97B93F80E8093F810E093F811C0DE7C34
:100E20009F7C587D890041EA98110EF0010E41EA3D
:100E30008E21918293F812E0197C0CF00F0C760051
:100E40004FEACC1C46EADE1E4CEA51011E7D93F8A7
:100E500011C0D18207F07F073F01997D47EA1C1737
:100E600006F0030693F814C017834EEA46265F7D0A
:100E7000568314F0010F40F2147300F01F0014BFEA
:100E80001E46AD26800114F0020F4FEAC10140EA70
:100E90009C0008BFAD2341EA5711002D9083D183F8
:100EA000168453840CBF01200320BDE8F083104654
:100EB000704711491F8C0C8066B147F002021A84FA
:100EC00012B29DB94A8046E71A8C4DB942F002022F
:100ED0001A8440E745B147F001021A8412B2F1E7E3
:100EE00042F003021A8436E73AB2EBE747F0030216
:100EF0001A84F3E79587002098870020394B5B68B8
:100F0000C3F30803F0B413BBEFF31183FBB9364A04
:100F1000364E1368B56800BF1468A342F9D1344A4D
:100F200016684FF47A7404FB06F2551BCA69B5FBC8
:100F3000F6F504FB03539A1A40F6AC54A2422DDC9A
:100F400091F822406CB3182C37D9F0BC7047EFF3FE
:100F50001184102383F31288244D264AAE682B682F
:100F6000DB0344BF012313601F4B48BFAE681F68FB
:100F70001368E4B284F311881D4A15684FF47A743B
:100F800004FB05F23B44921BB2FBF5F204FB032386
:100F9000CA6940F6AC549A1AA242D1DD002281F807
:100FA00022200F28D1D10122CB61087081F82220A4
:100FB000002381F82330F0BC7047631CDBB2192B8F
:100FC00081F822300855F3D10B4B1B78162B08BF44
:100FD0000A4B4FF0010081F8230008BF9A80F0BC53
:100FE000704700BF00ED00E0D490002010E000E06A
:100FF000D8900020D090002095870020988700206E
:10100000094BDFED0A6ADFED0A7A03EB810191ED0E
:101010006E7AB8EE477AE7EE267AFCEEE77A17EEBC
:10102000903A98B2704700BF0C29002001F11F3F91
:1010300000405C44714A92F8F83133B192F8FE31C5
:101040000021162B82F8F81101D00020704792F889
:10105000FD31022BF0B440F2CE8002F5FE70184450
:1010600002F5FF71D32311F8014F634013F0800F95
:101070004FEA430318BF83F0D503DBB213F0800FB0
:101080004FEA430318BF83F0D503DBB213F0800FA0
:101090004FEA430318BF83F0D503DBB213F0800F90
:1010A0004FEA430318BF83F0D503DBB213F0800F80
:1010B0004FEA430318BF83F0D503DBB213F0800F70
:1010C0004FEA430318BF83F0D503DBB213F0800F60
:1010D0004FEA430318BF83F0D503DBB213F0800F50
:1010E0004FEA430318BF83F0D5038842DBB2BAD17D
:1010F00092F81512994202D00020F0BC704792F885
:10110000040292F8036292F8081292F80C3292F8F4
:10111000104292F80052B2F800C2D2F8007200F009
:101120000F00C00140EA560001F01F0192F807626B
:10113000C2F8C401890141EA960103F03F0392F825
:101140000B6292F80F02C2F8D0115B0143EAD6039A
:1011500092F8FF11C2F8DC3104F07F04B2F80432D7
:10116000D2F80462240105F0070544EA101041EAB0
:101170000521C3F30A13C2F8E801B2F80852C2F815
:10118000B811B2F80A42D2F80C02B2F80E12C2F844
:10119000C831D2F81032C0F38A10C1F34A01C3F348
:1011A000CA13CCF3CA0CC7F38A37C6F3CA366D0923
:1011B000C4F30A04C2F8E001C2F8E411C2F8BCC1E9
:1011C000C2F8C071C2F8CC61C2F8D451C2F8D8419B
:1011D000C2F8EC3192F8143292F81302B2F81212FB
:1011E000DB0043EA5013C1F38A01C2F8F431C2F8BC
:1011F000F011012081E7D3237AE700BF0C290020FA
:10120000944B5B68C3F3080370B443BBEFF31183E3
:101210002BBB914A914D1368AC6800BF11688B429B
:10122000F9D18F4A15684FF47A7101FB05F2141B4E
:101230008C4AB4FBF5F401FB0343D2F83C1201F2F3
:101240004C41994233D201240021C2F83C3282F849
:10125000FC0182F8404282F8F81170BC7047EFF34D
:101260001181102383F312887C4C7F4AA568236880
:10127000DE0344BF01231360774B48BFA5681E6897
:101280001368C9B281F31188754A14684FF47A71F2
:1012900001FB04F23344521BB2FBF4F201FB0323C3
:1012A000704AD2F83C1201F24C419942CBD392F8E9
:1012B00040120029C7D002298ABF92F8FD410524B7
:1012C00002348C42C9DD4B1CDBB29C421144D4BFBA
:1012D0000125002582F8403281F8FC0182F8F8519E
:1012E000BBDC92F8FE510023162D82F84032B4D0B8
:1012F0006B00290648BF83F0D503DBB213F0800FE3
:101300004FEA430318BF83F0D503DBB213F0800F1D
:101310004FEA430318BF83F0D503DBB213F0800F0D
:101320004FEA430318BF83F0D503DBB213F0800FFD
:101330004FEA430318BF83F0D503DBB213F0800FED
:101340004FEA430318BF83F0D503DBB213F0800FDD
:101350004FEA430318BF83F0D503DBB292F8FD01D7
:1013600013F0800F4FEA430318BF83F0D503022820
:10137000DBB247D93D490844023111F8016F73408F
:1013800013F0800F4FEA430318BF83F0D503DBB29D
:1013900013F0800F4FEA430318BF83F0D503DBB28D
:1013A00013F0800F4FEA430318BF83F0D503DBB27D
:1013B00013F0800F4FEA430318BF83F0D503DBB26D
:1013C00013F0800F4FEA430318BF83F0D503DBB25D
:1013D00013F0800F4FEA430318BF83F0D503DBB24D
:1013E00013F0800F4FEA430318BF83F0D503DBB23D
:1013F00013F0800F4FEA430318BF83F0D5038142F7
:10140000DBB2BAD1224492F8FB219A427FF425AF95
:101410007A2D08D07C2D06D0282D7FF41EAF144BDA
:1014200001221A7019E7134A136E572B3FF715AFB5
:10143000114912480D684C68082199541344012140
:10144000C3F80150C3F80540136E017009331366E9
:1014500003E700BF00ED00E0D490002010E000E0C2
:10146000D89000200C290020D0900020082B0020CC
:1014700090620020A06200200D2B002091620020CD
:1014800070B5404D404C2B7806461BB1D4F8443221
:10149000834232D93D4B1B68DA070FD594F84932A5
:1014A00094F84A229A422DD194F8680228B9D4F8C7
:1014B0008002B0428CBF0020012070BD13F40053A5
:1014C0002ED1D4F87422324884F868329047C3078A
:1014D000EAD5D4F84C322F4A00F0020000281E440E
:1014E00013BF0121002101230023012051702B7023
:1014F000C4F8446284F8680270BD00232B7084F83D
:101500004832C7E7D4F84C22224984F84A323244A0
:1015100000200123C4F84422087084F84832C3E74D
:10152000B4F850320BBBB4F85232F3B9B4F85432B9
:10153000DBB9B4F85632C3B9B4F85832ABB9B4F821
:101540005A3293B9B4F85C327BB9B4F85E3263B9FD
:10155000B4F860324BB9B4F8623233B9B4F86432DB
:101560001BB9B4F86632002B9ED0D4F84C3209492E
:10157000334400200122C4F84432087084F8482221
:1015800092E700BF065D00200C290020489A002049
:10159000782B002078000020002070470020704742
:1015A000024B03EB4101B1F8840270470C29002083
:1015B000044B93F8A80218B1002283F8A822012056
:1015C000704700BF0C290020024B03EB8101B1F8EA
:1015D000AC0270470C29002003788B4283BF034B79
:1015E00003EB4101B1F8E402002070470C29002010
:1015F00038B5394C0546F8F78BFED4F83833C4F8C3
:101600003803C01AB0F57A7F1CDD0023282284F845
:101610003C3384F83E3384F83F3384F83D233D2D3A
:1016200042D03E2D0DD12D4AC4F84023012384F829
:101630003E330123157084F83C3394F83D239A42DD
:1016400020D038BD94F83C23002AE8D0531CDBB2EC
:10165000D4F8401384F83C33062B8D54EDD194F824
:101660003E33012B27D094F83F33012B27D00023A2
:10167000282284F83C3384F83E3384F83F3384F8DE
:101680003D2338BD94F83E33012B04BF022384F878
:101690003E3394F83F33012B15D00022282384F8E1
:1016A0003C2384F83D3338BD0D4AC4F84023012360
:1016B00084F83F33BDE78B78282BD4D8F1E78B78BB
:1016C000092BD4D8EDE7022384F83F33F8F720FE46
:1016D000C4F84403E1E700BF0C2900201C2C0020C3
:1016E000102C002030B40246002305251E2400E003
:1016F0000232032BD4BF0021012100F81310013363
:10170000042B04D0122B5470F2D130BC70475570AA
:10171000EEE700BF024B036043608360C360704725
:10172000E803D007024B03EB4101B1F850027047C8
:101730000C290020024B03EB4101B1F85002704725
:101740000C29002030B4264C94F83E33022B02D0F2
:10175000002030BC704794F81253EDB1013D04F203
:10176000113353FA85F504F54470002210F8013B5B
:10177000534083EA0313DBB2120AD90042EA032280
:10178000854281EA131382EA0302EFD122B10020DD
:1017900084F83E0330BC7047B4F810335BBA9BB298
:1017A00043F60162934209D043F60362934205D0A7
:1017B000002384F83E33012030BC7047094AA2F16F
:1017C0002E0102F12005D0799379023203EB002338
:1017D000C3F3CC03AA4221F8023FF4D1E8E700BFEB
:1017E0000C2900201C2C00204E4B5B68C3F308031F
:1017F00070B4B3B9EFF311839BB94B4A4B4D1368E7
:10180000AC6800BF11688B42F9D1494A15684FF4A2
:101810007A7101FB05F2141BB4FBF5F401FB0343E1
:1018200020E0EFF31181102383F312883F4C414AEB
:10183000A5682368DB0344BF012313603A4B48BF0C
:10184000A5681E681368C9B281F31188384A146804
:101850004FF47A71334401FB04F2521BB2FBF4F2F1
:1018600001FB0323344AD2F84813591AB1F5FA7F21
:1018700014D90021C2F8483382F84C1382F84D1372
:10188000C3B2042B26D0202B24D092F8501309B9D0
:10189000552838D0814216D1002109E092F84D1325
:1018A00099B992F84C13C2F84833C3B20029E8D072
:1018B00092F84E0354180138814284F858331DD0F1
:1018C000013182F84C1370BC7047013982F84D1316
:1018D00070BC7047002102244FF6FF7082F8544319
:1018E000A2F852035418581E814282F8503382F8ED
:1018F0004E3382F84F1384F85833E1D1012382F834
:10190000783370BC704701241F2582F85003A2F879
:10191000521382F8583382F84F4382F8544382F8C6
:101920004E53CDE700ED00E0D490002010E000E041
:10193000D8900020D09000200C29002070B540F2F3
:10194000014444EA8004F8F7E3FC0C4E054696F89F
:101950009C3306EB8303D3F87C03E3070AD51AF024
:10196000A7FC640805F1340507D0F8F7D1FC8542DF
:10197000FBD8ECE71AF096FCF3E770BD0C290020C9
:101980000D49B1F89D3330B508224AF2010580EACD
:10199000030414F0010F4FEA530318BF6B4002F128
:1019A000FF3218BF9BB212F0FF024FEA5000EED197
:1019B000A1F89D3330BD00BF0C290020084628F057
:1019C0002DBA00BF0FB400B583B004AB054953F87E
:1019D000042B019300201CF0E7F803B05DF804EB42
:1019E00004B07047BD1901080EB470B583B007ACE0
:1019F0000646482054F8045B28F010FA202028F00E
:101A00000DFA304628F07CF93A2028F007FA2A46E9
:101A100023460949019400201CF0C6F804460A2018
:101A200028F0FCF9054A136803341B1B136003B04C
:101A3000BDE8704003B07047BD190108A8850020BB
:101A4000F8B50F4BD3F8A053D3F8A443D3F8A86349
:101A5000A9B1831E00EB410727441E4404441D44E2
:101A600034F9022B36F9023F35F9020F134403EB28
:101A7000D373A0EB630028F0B9FAA742F0D1F8BD08
:101A80000C2900202DE9F04FDFF80C913949D9F8E5
:101A9000A053394B2C4685B005F1300B05F11002EF
:101AA00044F8040B5E46029209F56B7A09F56E78EC
:101AB00009F57177FAEC016AB8EC017AF7EC017A72
:101AC000B1EC010A0193FDEEE66ABDEEC77AFDEEC8
:101AD000E77AE4EC016A84ED027AC4ED057A0091BC
:101AE00003912EF061FF019B029A26F8020B9442AB
:101AF00053F8040BB0800099DCD1204905F128038C
:101B0000F1EC017AFDEEE77A17EE902A23F8022B2A
:101B10005B45F5D11A4B1B4A588811781A88AA8759
:101B20009A88DB88E887A5F84020A5F8423071B193
:101B300005F14403144A03EB4101F2EC017AFDEE96
:101B4000E77A17EE900A23F8020B8B42F5D10F4982
:101B50000F4A104BB9F8FA03498852681B88A5F858
:101B60005E00A5F86410A5F86620A5F8683005B0F9
:101B7000BDE8F08F3C9A0020845D0020085D0020C5
:101B800098870020515A0020DC2C0020445D002062
:101B90004C5D0020985E00200C290020F8B52F4CE9
:101BA0002F4D3822002120462EF022FD2D4B95F896
:101BB0000464B3F85020A283103393E8070095F82B
:101BC000033484F820600E2B04F1080686E8070031
:101BD00008D90023A377227F0B2A0AD0002B3AD101
:101BE0000020F8BD01229A4045F601510A42F5D085
:101BF000F1E71D4A1D4913681D4E216043F00203A1
:101C000013601C491548616004224FF480730E274D
:101C1000A277A38277711AF0F5F8B5F810344FF473
:101C20007A7262627BB1144E06F16C07B5F810341B
:101C3000616A00EE103A3046B8EE400A24361CF0D5
:101C400031FBB742F2D195F8023413B1A3770120EA
:101C5000F8BD0120F8BD012BC2D0BAE75C5D0020C1
:101C60000C290020CC9100209C5D002005BE0208BC
:101C700078000020A1030308202D00202DE9F04763
:101C80002DED028BC44FC54DBB7C012B00F0DC82D7
:101C9000022B0CBF0723002385F88034C04B1B7830
:101CA000132B00F2BF800122BE499A400A4208BFAE
:101CB0000023BD4EDFF8089385F8813400233522D8
:101CC0003360C6E90133F360232085F88234C9F814
:101CD000183089F85820FAF773FFB44BD9F8180078
:101CE000C9F81430022389F81030002800F0B082BF
:101CF00095F88334002B00F0B6824FF48071D9F848
:101D000014001DF0BFFAD9F8183013B11A689B8877
:101D100053836B21D9F814001CF062FC8021D9F8A0
:101D200014001CF05DFCD9F8183013B11A689B88B8
:101D300013834FF015084FF0F50A9620FAF740FF8D
:101D4000D9F8183013B11A689B885383D9F8140056
:101D500040F2E93302E0002B00F09B820289013B54
:101D600012F0020F9BB2F6D0A0F80CA040F2E933BB
:101D700002E0002B00F08D820289013B12F0010F7E
:101D80009BB2F6D08389838940F2E93301E0002BCE
:101D900045D00289013B12F0020F9BB2F7D0FF231E
:101DA000838140F2E93301E0002B38D00289013B06
:101DB00012F0010F9BB2F7D08489E4B2D9F8183041
:101DC00013B11A689B881383982C00F06E8240F23E
:101DD0003282AC2C28D0AF2C40F060820821D9F898
:101DE00014001DF04FFA092389F8503099F850205B
:101DF000D9F84C10BB79C5F8841400200B2A89F857
:101E0000553089F8520006D8012303FA02F111F483
:101E1000386110D10846BDEC028BBDE8F0871AF09E
:101E200099FBCBE7002344E70821D9F814001DF003
:101E300029FA0723D8E7DFF8C0C1DFF8C0E1DCF8F2
:101E400000105B4CC9F81C401943CCF800100D2160
:101E50008EF80410FC785749DFF8A4C1C9F80010C7
:101E60000421C9F804C089F85210002C00F0D68172
:101E7000072C00F0D3810A2A0BBF9FED4F7A9FED0C
:101E80004F7A89F8533089F8530007EE903AF8EE0C
:101E9000E77A013B67EE877A494889F85730FCEECC
:101EA000E77A89F85640C6ED007A1AF06FFB3B7866
:101EB0000BB189F85230434C2AF02AFE424A43497A
:101EC0003668434BB3FBF6F320464FF4FA7740F8FD
:101ED0001C1B9BB24FF47A71B3FBF1F302F12801A2
:101EE000C5F89C24C5F88834A8321023C5F8981486
:101EF000A5F88C7420211427A5F89434C5F8A824DB
:101F0000A5F8A41480220021A5F8A07485F88E34C9
:101F10002EF06EFB8022002104F19C002EF068FB65
:101F2000002104F58E7080222EF062FB9FED295A6D
:101F3000DFED365ADFED283A9FED282ADFED282A1B
:101F40009FED283A9FED281ADFED281ADFED286A69
:101F500004F5CE71002307E00133B6EE007A202BA2
:101F6000A1EC017A00F0938007EE903AF8EEE77A60
:101F700067EE857A37EEA57ABDEEC76A16EE102AAF
:101F80002032402AE8D8F4EEE57AF1EE10FA40F378
:101F9000A1819FED186A3DE01C9A00200C290020C9
:101FA0009587002048800800389A002000300140C2
:101FB00090C1793D8DC50208D145634400007A4443
:101FC000CC9100209C2D0020041204080000F84150
:101FD00040420F003C8C4F3EDB0F49C092E741B9B5
:101FE0009730083C15A82ABEDB0FC9BFDB0F49405C
:101FF000DB0FC940E4CB16419C5D00207800002037
:1020000029D30208E4CB16C1E5A6C539DB0FC93FC9
:10201000B0EE677AB4EEC67AF1EE10FA77EE667A31
:10202000F6DCF4EEE37AF1EE10FA40F15B811FED9D
:102030000B6A01E0F0EE477AF4EEC67AF1EE10FAA0
:1020400037EEA67AF6D4B4EEE57AF1EE10FA40F364
:10205000398131EEC77A27EE076AB0EE624AA6EE02
:10206000024A0133202BF0EE430AE4EE060AF7EEB3
:10207000007A66EE474A37EEC77AF6EE007AA4EEAB
:10208000A07A27EE277AA1EC017A7FF46DAF0C23BA
:1020900003FB06F306EE103AB8EE466A5FED267AC9
:1020A0001FED260ACB4B9FEDCC3ADFEDCC3ADFEDAE
:1020B000CC1A9FEDCC2ADFEDCC2ADFEDCC6ABCEE4A
:1020C000C66AB0EE401AB8EE466A03F16C0226EE1C
:1020D000276A03F1D80EFDEEC67A36EE000A17EE37
:1020E000905AFDEEC07A203517EE904A0021203438
:1020F000F7EE004A0EEB0100C826402D868000F264
:10210000F480B4EEC36AF1EE10FA40F35C81B0EEF5
:10211000467A9FEDB75ADFEDB75A01E0B0EE677A25
:10212000B4EEE57AF1EE10FA77EE457AF6DCF4EEED
:10213000E37AF1EE10FA40F143819FEDAD5ADFED05
:10214000AE5A01E0F0EE477AF4EEE57AF1EE10FADD
:1021500037EE857AF6D4B4EEC17AF1EE10FA40F398
:10216000158133EE477A67EE077AB0EE424AA7EE62
:10217000A14A402CF0EE620AE4EE270A27EE275A25
:10218000DFED9E5AA5EE207AB0EE644AF0EE647A56
:10219000A7EE254AE7EE657AC7EE840A40F2AC80E6
:1021A000F0EE667AB6EE007AF7EE005A84EE845AC4
:1021B0000831DFF868C2924F924E9348C2F800C0CF
:1021C00018299760D660106103F1240302F12402FC
:1021D00043ED050A27EE057A65EE855A67EE857AA6
:1021E00003ED097A03ED077A43ED085A43ED067AC9
:1021F00043ED036A43ED046A43ED016A43ED026A6D
:1022000042ED086A42ED036A42ED046A42ED016A5A
:1022100042ED026A7FF46EAF0120FCE5F979BB78EC
:10222000002940F0C7800A2A46D1042289F85320A9
:102230009FED767A29E6122C30D10821D9F81400C6
:102240001DF020F80823CFE5042385F8803425E528
:102250003420F7F72FFB95F88334C9F81800002BCA
:102260007FF44BAD18B11C2200238271C371092188
:10227000D9F8180019F07AFFD9F818001AF018F8F0
:102280000821D9F814001CF0FDFF012385F88334E0
:1022900033E51AF05FF9D9F8140074E508F1FF3856
:1022A00018F0FF087FF449ADA0E50821D9F8140023
:1022B0001CF0E8FF0B2397E5032289F853209FEDDC
:1022C000547AE2E5B4EEC17AF1EE10FA48BF33EE8B
:1022D000C77AC0E6F0EE477AF4EEE37AF1EE10FA50
:1022E0003FF5A5AEB0EE677AADE6F7EE000A402CFA
:1022F000B0EE604A3FF654AFB4EEC16AF1EE10FAA8
:1023000064DDB0EE407A9FED3A5ADFED3A5A01E0D3
:10231000B0EE677AB4EEE57AF1EE10FA77EE457A30
:10232000F6DCF4EEE37AF1EE10FA0FD5B0EE677A50
:102330009FED2F5ADFED305A01E0B0EE677AB4EE30
:10234000E57AF1EE10FA77EE857AF6D4F4EEC17AFA
:10235000F1EE10FA24DD73EE677A27EEA77AF0EE3D
:10236000425AE7EE215AF0EE628AE7EE258A27EE1E
:10237000278AB8EE005AE8EE287AB6EE007A74EEB4
:10238000E75A67EE857A25EE877A0FE7DFED217A47
:10239000B4EEE77AF1EE10FA48BF33EEC77AE2E620
:1023A0009FED1C7AF4EEC77AF1EE10FA48BF73EE97
:1023B000E77AD2E7052289F853209FED177A64E582
:1023C000B0EE677AC7E6F0EE467AB0E6F0EE407A15
:1023D000A7E700BFB82F0020DB0F4940DB0F49C043
:1023E00092E741B99730083C15A82ABE00000000CA
:1023F000DB0FC940E4CB1641E4CB16C1F304353FF3
:1024000000DFCDBEBA32BDBE0184483EE438DE42B4
:102410000000FA42DB0FC9BF0000FC4100DFCD3EE7
:10242000F0B5174E002383B004460821D6F89C0768
:10243000B37602ADFAF7AEFDD6F89C078121FAF724
:10244000A9FD8923D6F89C6725F8023DE71D14F8FD
:10245000010B3246294617F0E7FCBC42F7D1BDF824
:1024600006301A0A52FA83F3C3F1FF039BB23246D5
:10247000D8B20021ADF8063017F0D6FC03B0F0BD9D
:102480000C2900202DE9F041884C94F8232094F881
:1024900022309A4261D094F8232094F82330C2EB82
:1024A000C20204EB8202C3EBC30304EB830392F882
:1024B0003F1093F824608B1E9E4228D07C4BD4F8AA
:1024C000A0171B78172B64D0002094F82330794A8A
:1024D0000133A2FB0352520802EB42029B1ADBB209
:1024E00084F8233009B9BDE8F081734B1B68591A91
:1024F000B1F5FA7FF7D994F8A437032B02D16F4BCB
:1025000000221A800023C4F8A037BDE8F08194F8B7
:10251000233004F12407C3EBC30307EB830361B14A
:102520001944002213F8015B2A44994292B2F9D16E
:10253000D3B203EB1222FF2A39D05D4BD4F8A01797
:102540001B78172BC0D1238C5D4A01339BB204202A
:102550009080238453800020B7E7F7F7D9FE94F8E2
:10256000CC3703B3637EF3B1E36FC31AB3F5FA7FDD
:1025700019DBE36FC31AB3F5FA6FC4BF00236376A8
:10258000637E03F0FF02002B49D11046D4F8A01758
:10259000A8E7238C4A4A01339BB20320908023840E
:1025A0005380002091E7D4F8A01700209AE794F810
:1025B000233001221C2101FB0323FA18FB5CDBB151
:1025C000012B12D1082ED4F8A0174FD0384B1B780E
:1025D000172B7FF479AF238C394A01339BB2062045
:1025E00090802384538000206FE7314B1B78172B9A
:1025F00030D0D4F8A01767E7192E67D02C4AD4F84A
:10260000A0171278172A7FF45FAF228C2C4D01326D
:1026100092B20626184622846A80AE8055E7244B83
:102620001B78172B03D1E26F254B801AD88094F8C2
:10263000D437D4F8D00703B918B10022214917F0D4
:10264000FFF8637E03F0FF00002B40F01281D4F806
:10265000A01747E7238C1A4AD4F8A01701339BB27E
:10266000052090802384538000202EE794F8CC0727
:1026700000283FF42AAF53780025102BC4F8D05718
:1026800000F0028140F2FD80303B012B3FF61CAF91
:1026900052F8010F0C4BC4F8D807908892799880B3
:1026A0009A712846C4F8D0370FE700BF0C290020E4
:1026B00095870020ABAAAAAAD4900020985E00209B
:1026C0009887002025290020E430002092F802801D
:1026D0005778C36892F803E011799579D67992F822
:1026E00008C008F0070047EA00200EF03F0E977A76
:1026F000188090784FEA4E1E4EEAD00E907BA3F8D9
:1027000002E092F803E0890041EA9E1192F805E0A8
:102710000EF0010E41EA8E21998005F00F055179E6
:1027200092F807E0ED0145EA5101557AD9804FEA68
:102730004C0C4CEADE1C05F0030592F806E0D17A59
:1027400006F07F064CEA452C3601557BA3F80AC0FB
:1027500046EA1E161E8105F00706957A92F809C012
:10276000C90041EA5511157B07F01F0745EA062508
:1027700000F03F00567BD9814001BF0140EAD601FD
:1027800047EA9C079F811D825982D17B92F80EC037
:10279000D67C92F812E0577C957C507D890041EA06
:1027A0009C1192F810C076000CF0010C46EADE167F
:1027B00007F00F0792F810E041EA8C21FF0192F830
:1027C00014C0998247EA5E07917DDF8205F07F059C
:1027D000577C0CF0030C46EA4C262D0145EA1715F0
:1027E0005E83177D567D1D8300F01F008001C900A8
:1027F00041EA561140EA9700D9839883D07D94F836
:10280000A45710F0010F40F2147114BF0E46AD260C
:1028100010F0020F08BFAD2110F0080F0CBF01200F
:102820000320032D1E8459841ED1137E94F8A5170E
:10283000184ED4F8A827642B04EB4105A8BF6423E5
:102840009B02A6FB0363B5F8AC6701315B0901F09D
:102850000F01921B1A4484F8A5170F49A5F8AC374D
:102860001309C4F8A8270B800C4B1968C4F8A017EB
:102870002BE60B48FFF7D4FD0020D4F8A0176076B4
:1028800030E6002B7FF420AE012384F8D4370020FB
:102890001BE600BF1F85EB51985E0020D4900020FE
:1028A0002C13040838B50D4C05460146D4F8E00752
:1028B000FAF770FBB4F8E407082380EA052041F238
:1028C000210210F4004F4FEA400018BF5040013B76
:1028D00080B2F6D1A4F8E40738BD00BF0C2900206F
:1028E0002DE9F047BC4C94F8B40188B010B908B099
:1028F000BDE8F08794F8EC37002284F8B421002B6F
:1029000000F0208194F8A421B44E94F8ED5752B20F
:1029100012F1630FB8BF96F90920002D40D012F1D3
:10292000310F80F2298212F1380F80F2478212F1C2
:102930003D0F80F2478212F1420F80F2478212F17E
:10294000450F80F2478212F1470F80F2478212F161
:10295000490F80F2478212F14A0F00F0478212F1CC
:102960004B0F00F0468212F14C0F00F0468212F13C
:102970004D0F00F0458212F15C0FB8BF642180F268
:102980004282D4F8F037964803FB01F380FB030141
:10299000DB17C3EB611304EB85019BB2C1F868310F
:1029A000727294F8FA2794F8A611D4F8FC3794F8C8
:1029B00000081B78114101F00F018B4210D90B293F
:1029C0000ED8002D40F0898194F8A6C194F8A77123
:1029D00004EB810100EA0C0C07EB0C27C1F86871CD
:1029E00094F8A811114101F00F018B4210D90B2965
:1029F0000ED8002D40F0798194F8A8C194F8A971FF
:102A000004EB810100EA0C0C07EB0C27C1F868719C
:102A100094F8AA11114101F00F018B4210D90B2932
:102A20000ED8002D40F0518194F8AAC194F8AB71F2
:102A300004EB810100EA0C0C07EB0C27C1F868716C
:102A400094F8AC11114101F00F018B4210D90B2900
:102A50000ED8002D40F0458194F8ACC194F8AD71CA
:102A600004EB810100EA0C0C07EB0C27C1F868713C
:102A700094F8AE11114101F00F018B4210D90B29CE
:102A80000ED8002D40F0258194F8AEC194F8AF71B6
:102A900004EB810100EA0C0C07EB0C27C1F868710C
:102AA00094F8B011114101F00F018B4210D90B299C
:102AB0000ED8002D40F01D8194F8B0C194F8B1718A
:102AC00004EB810100EA0C0C07EB0C27C1F86871DC
:102AD00094F8B21141FA02F202F00F029A420FD2B8
:102AE0000B2A0DD8002D40F0088194F8B21194F80B
:102AF000B33104EB8202084003EB0020C2F8680106
:102B000094F8B01194F8B15194F8B23194F8B3211B
:102B10002D0445EA0165154345EA032505F0F02338
:102B2000B3F1E02F62D094F8EC373BB194F8653103
:102B300023B194F8A6311B0600F1E380012008B010
:102B4000BDE8F087F7F7E4FB244E264BB27AA3FBEF
:102B500000135B0CAAB194F8A42194F8A511C9B292
:102B6000122918BF0129D2B200F0EC8001F0EF0168
:102B7000A1F1A201B1FA81F14909002940F0E280F6
:102B8000B17294F8A41194F8A52102EB012292B23B
:102B9000D4F8F41794F8ED57C9B18B423FF401AF64
:102BA000591A012913D195B1B4F8F807D4F8F017E0
:102BB0000D4F101A143801FB00F187FB0170C91783
:102BC000A1EBE00104EB850089B2C0F86811A4F81C
:102BD000F827C4F8F437E4E60C2900207800002038
:102BE0001F85EB5183DE1B4367666666894FDFF8FE
:102BF0003482B9883A7A97F800C097F801E097F8DC
:102C000002908DF808C00023CDF80A30CDF80E30C0
:102C10008DF809E002AB8DF80A90ADF80C108DF834
:102C2000102093E8070005AB03C3D8F800101A8002
:102C300005F0070AB9B1784AC5F342531A44C5F3FF
:102C4000034392F84C21944503F1010301D19E45C1
:102C500009D0104619468DF814208DF8153016F05D
:102C60001FFAADF8180026F0C5FB03287AD0042817
:102C700063D001287BD00022D8F80030002B63D02D
:102C8000914501D08DF8162008A8002300F8193DC1
:102C900026F082FB9DF80730C5F30010834201D077
:102CA00026F09EFB029A059B9A4250D09DF8143064
:102CB0009DF815109DF816203B70BDF818307970FE
:102CC000BA70BB80F6F728F82DE7A9427FF4ACAEC6
:102CD000B6E68D427FF4D8AEE2E6A9427FF474AE48
:102CE0007EE68D427FF4B8AEC2E6A9427FF484AEA0
:102CF0008EE68D427FF4E0AEEAE6AA427FF4F5AEBE
:102D0000FEE6F7F705FBD4F8E83700F57A70306196
:102D1000002B7CD05A68121A002A04DB77E05A682C
:102D2000121A002A04DA03F108019B68002BF6D17D
:102D30003A4A736101200A60D9E5374B9A449AF800
:102D4000642199E792B223E78DF80730AAE7039A46
:102D5000069B9A42AAD1BDF81020BDF81C309A42B9
:102D6000A4D1E0E62C4B9A449AF85C2184E72A4BE4
:102D70009A449AF854217FE76FF0300701232648E0
:102D8000591E00EB410100EB430091F831C190F86E
:102D9000310191F93011A0EB0C00531A03FB00F341
:102DA000791A93FBF1F363445BB2002B01DA002143
:102DB000E7E5642BA8BF64231946E2E56FF0370707
:102DC0000223DCE76FF03C070323D8E76FF04107ED
:102DD0000423D4E76FF044070523D0E76FF04607DC
:102DE0000623CCE76FF048070723C8E717460823F8
:102DF000C5E76FF04A070923C1E717460A23BEE774
:102E000017460B23BBE76FF05B070C23B7E70449BA
:102E10008EE700BF265D0020041204088400002015
:102E2000F4300020345D00202DE9F8438846017815
:102E3000A9B10C4E04468146354606F108072846DE
:102E40002DF0EDFB38B1B842A0EB06003CBFA9EB7A
:102E5000040308F8003019F8011F0029EFD1BDE87C
:102E6000F88300BF701304082DE9F8432C220446B0
:102E700000212DF0BDFB0123174D184ADFF86480B7
:102E80002375292140F26C7313261548A175A261A0
:102E900040F643010E22A383022384F82060E184DC
:102EA000C4F8220084F828202372A377C1462E4656
:102EB00005F10807412130462DF0B1FB30B1B84291
:102EC000A0EB05003CBFA9EB0803235419F8011F30
:102ED0000029F0D1BDE8F88370130408DC051A045A
:102EE000460575031C5304082DE9F04FE24C94F895
:102EF00078338BB023B9002318460BB0BDE8F08FB0
:102F000094F84F3394F84E030022012B84F8782371
:102F100045D094F85853023D15F0FF0500F0A88104
:102F200004F556710D444FF6FF7311F8012B9B1AEF
:102F3000A9429BB2F9D11A0A204490F85713914242
:102F4000D9D190F85623DBB29A42D4D194F85033B9
:102F5000202B40F0868194F854138B1C09938B1D11
:102F6000019301F10803029301F10A03039301F1B4
:102F70000C03049301F10E03059301F11003069372
:102F800001F11603079301F1180301F1040A01F19D
:102F9000120801F11407089301F11A0BAFE094F83D
:102FA0005413B4F852E38B1C671854FA83F6099350
:102FB00001F1040A97F8583397F859C396F8585313
:102FC00096F8597354FA8AF673448A1D96F859E3B1
:102FD00001921D4496F8583354FA82F605EB0C25FD
:102FE00001F1080296F859C302922B4496F85853FF
:102FF00054FA82F603EB072301F10A0254FA82F72E
:103000002B4496F85853039203EB0E2301F10C0264
:1030100097F859E396F8596304921D4497F858338A
:1030200054FA82F705EB0C2501F10E0254FA82FCEA
:103030001D4497F85833059205EB062501F110025F
:103040009CF8586397F859739CF859C306922B441F
:1030500054FA82F503EB0E2301F1120895F859E3B7
:10306000334495F8586354FA88F503EB072301F1CC
:10307000140795F85993334495F8586354FA87F533
:1030800001F1160203EB0C23334495F858C3079261
:1030900054FA82F603EB0E2301F1180295F8595306
:1030A0000892634496F858E396F859C303EB092352
:1030B00054FA82F6734401F11A0B96F858E396F825
:1030C000596303EB052354FA8BF52044734495F8B8
:1030D00058E390F8579395F8595390F8560303EB3B
:1030E0000C239E440EEB062E0EEB052E00EB092959
:1030F0001FFA8EFE1FFA89F9F1457FF4FCAE9DF8A8
:10310000243054FA83F29DF8043054FA83FC9DF87D
:1031100008309CF859939CF858C354FA83F30193F0
:103120009DF80C3054FA83F69DF8103054FA83F56C
:103130009DF8143054FA83F09DF8183054FA83F354
:10314000029354FA88F303939DF81C3092F8598344
:1031500092F8582354FA83F3214405939DF82030C4
:1031600054FA8AFE54FA87F791F859A391F8581344
:10317000049754FA83F39EF8597306939EF858E324
:10318000019B01EB0A2102EB08220EEB072E93F8BC
:10319000598393F85873C4F8AC1296F859330193D5
:1031A0000CEB0921C4F8B81295F859C396F8586386
:1031B00095F85853019BC4F8B02206EB0326049BF4
:1031C000029AC4F8B4E293F859E393F8583392F8AA
:1031D000599392F85813039A019603EB0E23C4F8FF
:1031E000D432059B90F859A3019E90F85803C4F877
:1031F000C06207EB082701EB092192F8598392F886
:10320000582393F85963C4F8CC1254FA8BFB93F803
:103210005813069BC4F8BC7205EB0C2500EB0A2082
:1032200002EB0822C4F8C452C4F8C80293F85953F8
:103230009BF85903C4F8D02293F858239BF85833CD
:1032400001EB062103EB0023C4F8D812C4F8E032E6
:10325000012302EB05221846C4F8DC220BB0BDE8BE
:10326000F08F064816F03CF8002384F84D0343E63F
:10327000FF224FF6FF735FE60C290020642C00202C
:10328000F8B5F7F745F8274E054600F1FA0734463A
:1032900096F89C3306EB8303D3F87C0319F016F8F9
:1032A00038BB94F89C3304EB8303D3F87C0319F008
:1032B0000DF828B3F7F72CF8D4F80838401B9842DB
:1032C000C4F804082BD805F5FA7594F89C3304EB80
:1032D0008303D3F87C0318F0F9FFB0B994F89C335A
:1032E00004EB8303D3F87C0318F0F0FF90B10020C7
:1032F00005E0F7F70DF8B842CAD94FF0FF30F8BD36
:10330000F7F706F8B842CCD9F7E7F7F701F8A84283
:10331000DBD9F2E7F6F7FCFFA842DFD9EDE70120A1
:10332000EDE700BF0C29002038B5002405460470E5
:10333000FFF7A6FF431C11D0012803D12B78A04032
:10334000184328700134082CF2D1054A2B7892F8E2
:103350000C184B4082F80C38012038BD0020FCE7E7
:103360000C2900202DE9F843204C214D2668074602
:103370000236A84695F89C3305EB8303D3F87C030B
:1033800018F0A4FF10BBF6F7C3FF00F12706F6F70D
:10339000BFFF8642FBD800252C464FF0010998F864
:1033A0009C3308EB8303D3F87C0318F08FFF18B12C
:1033B00009FA05F31C43A4B2092D06F134060BD01B
:1033C000F6F7A6FF8642FBD80135E8E723689E4260
:1033D000D0D80020BDE8F88340F201232340B3F5A4
:1033E000007FF6D164083C700120F3E7D490002000
:1033F0000C29002037B502ADFF2305F8013D044636
:103400002846FFF7AFFF00B91CB99DF8070003B0CD
:1034100030BD013CF4E773B5204C002284F89D23B5
:1034200084F89E2384F80D2884F80E280144FF2296
:103430008DF807200546CEB22846FFF793FFF8B176
:1034400015F8010BFEF79CFAEBB2B342F4D194F8F5
:103450000F38EBB11248FFF785FF88B11148FFF72D
:1034600081FF68B10DF10700FFF77CFF40B1B4F8B0
:103470009D23B4F80D389A4202D0C2238DF807304C
:103480009DF80700A0F130035842584102B070BDCA
:103490000DF10700FFF766FFF2E700BF0C290020DF
:1034A000193100201A31002070B5194C94F89C3362
:1034B0000D4604EB8303013D0646EDB2D3F87C03D1
:1034C00026F064FF0135002384F89D3384F89E3391
:1034D00035443078FEF732FA16F8010BFEF750FA51
:1034E000AE42F6D194F80F383BB194F89D03FEF745
:1034F00025FA94F89E03FEF721FA94F89C3304EB26
:1035000083042021D4F87C03BDE8704018F02EBE5F
:103510000C29002013B5FE23ADF8043000238DF8EC
:10352000063003788DF80730044613B901238DF86F
:10353000063004210DEB0100FFF7B6FF0220FFF774
:1035400059FFFF280CD121786068FFF7ADFF2820D4
:10355000FFF750FFA0F130035842584102B010BDB0
:103560000020FBE737B5054608461446FFF7D2FFB3
:1035700078B10123022101A88DF805308DF804509F
:10358000FFF792FF2046FFF735FFA0F130035842C6
:10359000584103B030BD07B50E4B0268934317D0B6
:1035A000FF230421ADF8043043788DF8063083788A
:1035B0008DF807300DEB0100FFF776FF0220FFF7D3
:1035C00019FFA0F130035842584103B05DF804FBE5
:1035D0000120FAE700FFFF0037B5054608460C4614
:1035E000FFF7D9FF60B123788DF80450022101A8BC
:1035F0008DF80530FFF758FF21786068FFF70BFF63
:1036000003B030BD10B5064CD4F8E007F9F7BEFCA6
:103610000028F9D0D4F8E007BDE81040F9F7AEBCB7
:103620000C29002010B5FFF7EDFF0A4AB2F8133855
:1036300083EA00239BB2082141F2210413F4004FD6
:103640004FEA430318BF634001399BB2F6D1A2F899
:10365000133810BD0C29002038B50B4B03EBC00408
:103660000D4694F85422094803EB8203D3F88411E1
:1036700007F089FD94F85A322BB1691C0448BDE863
:10368000384007F080BD38BD04120408174904080B
:1036900006780408F8B50C4C0C4E0D4F04F5207557
:1036A000206807F08FFD616811B1304607F06BFDAF
:1036B000A16811B1384607F066FD103407F001FE2D
:1036C000AC42EDD1F8BD00BF001504080E49040856
:1036D000144904082DE9F04F82468FB091460E46FA
:1036E000154600273378089373780993F3780A9383
:1036F00096F904300B9396F9028096F905300C93F5
:10370000B3790D93B8F1000F4AD0B9F1000F4ED044
:103710002B78089C6A7895F90210E87895F904C02E
:1037200095F905E095F806B09C423ED1099C94427B
:103730003BD1884539D10A9C844236D10B9C6445E3
:1037400033D10C9C744530D10D9C5C4514BF0024D2
:103750000124CDE90121CDE9030C0093CDE905EB6E
:103760003B46144A2146504607F082FE0D9B0693C5
:103770000C9B05930B9B04930A9B0E4ACDE9028395
:10378000099B0193089B009321463B465046013715
:1037900007F084FE102F06F1070605F10705A1D1F9
:1037A0000FB0BDE8F04F07F08CBD0024D1E74C46C8
:1037B000DCE700BF1A4904082DE9F04FDFF820B11B
:1037C00089B08046894616460D4614464FF0000AD9
:1037D000002E71D06A6863689A426BD1AF68A368A3
:1037E000FB1A5F425F4194F90B30049394F90A305D
:1037F0000393B4F908300293B4F906300193B4F995
:10380000043000935A4653463946404607F030FE8E
:1038100095F90B30049395F90A300393B5F9083004
:103820000293B5F906300193B5F9043000935A4676
:103830005346394640460AF1010A07F02FFEBAF115
:10384000080F05F10C0504F10C04C1D10024DFF8C8
:1038500094A0254696B30027012303FA07FB3259AB
:1038600059F8043053403BEA030314BF01230023FB
:1038700012EA0B0F079306D000972B465246079982
:10388000404607F0F5FD59F804301BEA030F06D057
:1038900000972B4652460799404607F0FFFD013737
:1038A0000E2FD9D10135082D04F10C04D2D109B065
:1038B000BDE8F08F002796E73746A9E73746012392
:1038C00059F80420BB40134206D000972B465246BD
:1038D0000121404607F0E2FD01370E2FEFD1E1E76D
:1038E000374904084F4904082DE9F04F064685B0D2
:1038F00088461446894692460027002509EB0503B1
:1039000093F8C0300393002C64D00AEB0503039AAC
:1039100093F8C030D01AD0F1000B4BEB000BCDE97F
:1039200000532E4A3B465946304607F0A1FD039B03
:103930002A4ACDE9005359463B463046013507F047
:10394000ADFD062DDAD10137062F09F106090AF17E
:10395000060AD2D1DFF884B008F1E40A00251AF88B
:10396000019B002C38D063195A4693F8E430A9EB38
:1039700003014F424F41CDE90053394606233046FB
:1039800007F076FDCDE900590623144A3946304642
:10399000013507F083FD0B2DE1D198F8F0506CB1A3
:1039A00094F8F0300193EA1A5442544100230093F2
:1039B0000A4A07232146304607F05AFD00230093A8
:1039C00001950723054A2146304607F067FD05B0FB
:1039D000BDE8F08FA346AAE72746D3E76449040869
:1039E0002DE9FF47DFF86CA0814690460E4615464C
:1039F0000027B8F1000F2AD02B8832889A4224D1B0
:103A000074886A88A21A54425441EA780292AA78C9
:103A10002146CDE9003248463B46524607F028FD94
:103A2000F3780293B378019336F8043B009352463F
:103A30003B4621464846013707F030FD102F05F17F
:103A40000405D6D104B0BDE8F0870024DDE7444684
:103A5000E6E700BF784904082DE9F347DFF868A0DE
:103A600081460F46904602260024B8F1000F28D068
:103A700038F8243037F8241038F8062099421ED13F
:103A8000BD5BA91A4D424D41CDE90032294623467E
:103A90005246484607F0ECFCBB5B019337F82430F4
:103AA00000935246234629464846013407F0F6FC67
:103AB000042C06F10406D8D102B0BDE8F087002539
:103AC000E2E74546E8E700BF8A4904087FB5094BAD
:103AD0000493094B0393094B0293094B0193094B40
:103AE0000093094A094B0A490A4807F06FFC07B0DE
:103AF0005DF804FBDA490408DF490408E9490408D1
:103B0000F2490408FE4904089B490408F290002089
:103B1000A4490408AF4904082DE9F04F324C87B09E
:103B20000746324A2378608802EB8303D3F8848106
:103B30001DF070FBD0E901A304932D4B93F81538C9
:103B400013B9CDF810A09A4607F04003DFF8ACB0E7
:103B500005930025A379002B08BF01239D4206DBB6
:103B6000244B08349C42DCD107B0BDE8F08FA38819
:103B7000049A2B440135D65C1AF80330F21AD2F1BC
:103B8000000949EB020993B9009543465A46494654
:103B9000384607F06DFCC6B9059B002BDAD10095BD
:103BA00043465A464946384607F078FCD2E703F0C8
:103BB0000F021B0940330292CDE900530E4A4346DF
:103BC0004946384607F054FCE5E706F00F0336098E
:103BD00040360293CDE900564346074A49463846E7
:103BE00007F05CFCB6E700BF581404080412040890
:103BF0000C29002000150408184A0408044A040887
:103C00002DE9F04F674BDA7891B09846002A00F022
:103C10009F80654807F01CFE0025DFF8A0A1DFF8B3
:103C2000B0B10795A94608A9E8B21DF017FA9DF8AA
:103C30002830002B65D0012D0C9C40F09680002C84
:103C400000F08A8007EE904ADFED586AF8EEE77AD6
:103C500086EEA77AFDEEC77A17EE906A9AF81648B4
:103C6000089B012C7AD996FBF4F41A46012150489E
:103C700007F089FA0D9A002A00F08B8041F2883013
:103C800002FB04004FF47A73B0FBF3F00F9B002BA0
:103C900000F0818041F2883103FB04114FF47A7CFB
:103CA000B1FBFCF1052D03D0079F0F44814407971A
:103CB00098F803C0BCF1000F6FD04FF47A7C0E9FD0
:103CC000B7FBFCFCCDF810C04FF00A0C91FBFCFEDA
:103CD0000CFB1E11CDE902E190FBFCF10CFB110085
:103CE000CDE900102146334807F070FB012D08D1C3
:103CF0009AF81638012B04D9324609992E4807F054
:103D000065FB0135152D8ED198F80330EBB12B49A9
:103D1000D1F81C28D1F81808D1F8201852094FF40E
:103D20007A73B0FBF3F3264807F050FB0798079B24
:103D30000A2293FBF2F302FB130799FBF2F10097BF
:103D400002FB11921F4807F041FB11B0BDE8F08F54
:103D50001D4807F07DFD5FE726467FE7099A1B486F
:103D6000012107F010FA344684E75CB107EE904A6F
:103D7000DFED0E6AF8EEE77A86EEA77AFDEEC77AF7
:103D800017EE904A089A0A48294607F0FCF90026DF
:103D900070E710467AE7194684E72146584607F04F
:103DA00015FBA3E7EC9000202E4A04080024744978
:103DB000834A0408A54A0408C94A04080C290020BB
:103DC000D94A0408F94A0408794A0408924A0408BE
:103DD000D54A04082DE9F047694B6A48196890B044
:103DE0004FF47A73B1FBF3F107F0F0FA05A819F07C
:103DF000ADFD58B1644A05A90023B2F9002008A816
:103E000019F0B0FF08A9614807F0E0FA604B614D76
:103E10001B78614A6149127809886148DFF8E0A19E
:103E200005EB830305F5B269D3F87C3507F0CEFACC
:103E30005C4B5D4819685D4BB1FBF3F107F0A3F9EA
:103E40001CF052FE4FF47A72594BB0FBF2F102FBB8
:103E500011021B880A2092B289B2B2FBF0F25548D7
:103E600007F091F9544BD3F80080002405F5B665AE
:103E700059F82470A300D7B10126A64016EA080F0E
:103E800013D0F20611D01AF804205B594B4853F8AE
:103E90002220394607F077F9022E06D1484B93F8D5
:103EA000211011B1474807F06EF90134E0E707F03F
:103EB00008FA454A45494648464C07F087FA464ABB
:103EC000464B4748D31A3946B4F8242807F07EFAFF
:103ED00044490A6D002A42D007EE902ADFED426A7B
:103EE000B8EEE77AC6EE877AFDEEE77ACDED037A93
:103EF000D1F8EC305BB107EE903ADFED3B6AF8EEBB
:103F0000E77A86EEA77AFDEEC77A17EE903AC9698E
:103F100059B107EE901ADFED346AF8EEE77A86EED3
:103F2000A77AFDEEC77A17EE901AB4F826082F4E3E
:103F30002F4F6428CDE900310146039B2D48A8BFCF
:103F4000642107F043FA2C4807F03CF92B4B1C681E
:103F5000012534B907F0B5F910B0BDE8F087039238
:103F6000C6E794FAA4F3B3FA83F305FA03F256F81A
:103F70002310384624EA020407F005F9E9E700BFF8
:103F8000D4900020274B040804630020414B040810
:103F90006E5B0020041204084A5D0020445D00208E
:103FA000524B0408B0A80020784B040840420F0090
:103FB000D46F0020884B04089C5D0020A94B0408A6
:103FC0005C5D0020B14B04080000011000080000F7
:103FD000B54B04080C2900200080000800400008B0
:103FE000D94B040828020020002474496C340408CA
:103FF00047510408134C0408594C0408CC5E0020B7
:104000007C0000202DE9F84F184EDFF8689000255D
:104010000746AA4606F2C4580D246C4333193946A4
:10402000D3F8C4B558462CF036FB88B14444594601
:10403000484607F0A8F80021204607F037F907F0B6
:1040400040F9204607F0D6F907F03BF90AF1010ADA
:104050000135B5F5907FDFD1BAF1000F04D10448E6
:10406000BDE8F84F07F0F4BBBDE8F88F0412040870
:104070006F4C0408D477040838B50C4D044620462C
:1040800007F018F830B10A4B0A485978BDE83840B3
:1040900007F09CB920462CF08DF9022804D8C0B254
:1040A00010F026F82C46EAE738BD00BF4A4E040857
:1040B000EC9000207C4C0408022810B50C460FD868
:1040C00010F016F8074807F083FD0748FFF7D4FF04
:1040D00007F0F7F821460820BDE8104007F0F6B8D1
:1040E00010BD00BF8B4C04084A4E040870B50B4E3F
:1040F0000B4D0446204606F0DDFF30B1074B094862
:104100001978BDE8704007F061B920462CF052F9EB
:10411000022802D830702C46ECE770BDEC900020ED
:104120004A4E0408804C0408022810B50C460FD8EB
:10413000F4F774FB074807F04BFD0748FFF7D6FF7D
:1041400007F0BFF821460420BDE8104007F0BEB8D4
:1041500010BD00BF8F4C04084A4E0408F0B585B06E
:10416000054606F0A7FF002863D03349002201204E
:1041700005B0BDE8F040FFF71FBB2D2B03D0A3F126
:104180003002092A50D8052C04DD05B0BDE8F04006
:1041900007F064BB28462CF00DF904AB621C03EB5E
:1041A000440424F80C0C15F8013F303B092BFAD9D4
:1041B00014462B78002BE0D1062CE6D1BDF9043053
:1041C0009AB2072AE1D8BDF90600A0F2EE2292B217
:1041D00040F2DC54A242D8D8BDF90810A1F2EE2278
:1041E00092B2A242D1D8BDF90A209042CDDC9142D0
:1041F000CBDBBDF90C5005F16404A4B2C82CC4D8C3
:10420000BDF90E40112CC0DC0C4E0C2707FB0363DC
:10421000A3F82C08A3F82E18A3F8302883F83258F6
:1042200083F8334805B0F0BD202BAED101352246CE
:10423000BEE70446BDE700BF343100200C29002052
:1042400038B5044606F036FFA0B3244B9B69013312
:10425000172B25D822490C2202FB03121C46D2F848
:10426000745355B91E4A0C210134172C1ADD002451
:1042700001FB0420D0F87453ADB1184B9C611DF0C4
:10428000EDFD2A462146174807F0A0F8144B0C22F2
:1042900002FB043494F86C03BDE838401DF0FABD0D
:1042A0001C46DFE7E4D99C42DED10F48BDE8384028
:1042B00007F0CEBA20462CF07DF81728044607D820
:1042C000074A0C2303FB0023D3F87453002DD4D1E9
:1042D00021460648BDE8384007F078B8780000204D
:1042E000FC220408C14C0408974C0408AB4C040899
:1042F0002DE9F04F014691B006468548854D07F0FF
:1043000065F8854BC3F800D000232B70834B402405
:104310001C70834B0622197830460EF0FBFF0A20F2
:10432000F8F74EFC2B78DBB20C2B40F2ED809DF8B9
:104330000C90B9F1FE0F2ED0B9F1FF0F15BF0F246D
:104340001524002601269C4240F0DE80611EC9B281
:10435000684614F0FFFE10AB1C4414F8413C834245
:1043600040F0CE8006F1FF38B8F1010F9DF80D4006
:1043700013D904F01F07650961374C46694806F0F8
:1043800021FF022E71D0013D042D6AD8DFE805F02F
:104390000A5D616965000226D5E79DF80E709DF8FB
:1043A0000F50EBE7604807F053FA6048DFF8D09110
:1043B000DFF8D0B106F006FF00254FF0030A1DF824
:1043C00005104846013506F0DEFE0C2D55D106F0ED
:1043D00078FF022E5BD06422B4FBF2F102FB1142A3
:1043E0003B46D2B2C9B2524806F0F0FF5FFA88F8F5
:1043F000B8F1010F7BD84F4A4F4B9DF810104F4832
:104400004F4D00290CBF1146194606F0DFFF9DF8FD
:1044100011104C4B4C4800290CBF2946194606F098
:10442000D5FF022E63D19DF81240484806F0CAFE1F
:104430009CB3FF2C41D00A22B4FBF2F102FB1142E3
:10444000D2B2434806F0C2FF2AE0424807F000FA21
:10445000ABE7414807F0FCF9A7E7404807F0F8F957
:10446000A3E73F4807F0F4F99FE700230DF11F0091
:104470008DF83F3007F0ECF997E795FBFAF303EB83
:1044800043039D429BD1584606F09CFE97E73A466F
:104490002146344806F09AFFA8E7284607F0D8F9E5
:1044A0009DF81340304806F08DFE54B1FF2C21D00A
:1044B00021462E4806F08AFF06E02D4807F0C8F98D
:1044C000EEE71F4807F0C4F91D4D1E4E284F00248B
:1044D0000DEB04031A7D8AB1FF2A14BF32463A4617
:1044E00021462448013406F071FF042CF0D111B0AC
:1044F000BDE8F08F1E4807F0ABF9E5E72A46EFE785
:104500001D4807F0A5F9F2E71C4807F0A1F9EEE70E
:10451000F64C04086E5A0020605A00206F5A0020A2
:10452000515A0020074D0408124D0408404D04085C
:10453000574D0408DF4C0408D64C04088E4D04087F
:10454000E64C0408BD510408A54D0408AC4D040810
:10455000C04D0408194D0408214D0408294D0408D4
:10456000384D0408734D0408C84D04080778040842
:10457000EA4C0408D84D0408E34D0408F34D040840
:10458000524D0408767C040838B50D462BF012FF16
:104590000C4B19788842044605D201460A4819F0A6
:1045A0007FFC204638BD2DB1FF2803D1074819F004
:1045B00077FCF6E70139064819F072FC4FF0FF343A
:1045C000EFE700BF515A0020FC4D04080F4E0408CD
:1045D000244E04082DE9F341054606F06BFD044620
:1045E00020B107F03BF902B0BDE8F081284601AAEE
:1045F0002A49DFF8A8802BF016FF274605462646F5
:1046000075B9022CEDD1A7F57A73B3F57A7F1FD96E
:104610004FF4FA624FF47A71214806F0E4FEE2E7C3
:104620004CB1012C0FD001AA414600202BF0FBFE1B
:1046300001340546E4E701212846FFF7A5FF431CA6
:104640000646F0D1CFE728462BF0B4FE0746EAE74E
:10465000B8B208F077F8FF2EBCEEC00A114B0BD1B0
:10466000114AF8EE407A1278AA4212DC10EE101AC3
:104670000E4806F0ABFEB6E7F8EE407A03EB860391
:1046800010EE102A31460A48C3ED007A06F09EFE6D
:10469000A9E7E3EC017A0135E6E700BFBC7B04083B
:1046A000F850040894310020515A0020584E040854
:1046B0004B4E04082DE9F347054606F0FBFC044683
:1046C00018B9324B9B78042B04D807F0C7F802B016
:1046D000BDE8F08701AA2E49DFF8B890DFF8B8A04E
:1046E000DFF8B88028462BF09EFE0127264610B939
:1046F0000EF072FBEBE766B90121FFF745FF431CA3
:104700000446E4D001AA2249002001362BF08BFE9A
:10471000EDE72BF04FFE2F28054630D807B30EF0FB
:104720002FFB062D08D10520F8F74AFAFF2C24D0DC
:10473000E0B2FFF7DDFD08E00120F8F741FAEAB248
:1047400098F80010E0B20EF0E5FD2946504606F05C
:104750003DFE052D18DC1420F8F732FA0027D1E7CA
:104760000628E3D0EBE7FFF7C3FD98F80030F8B276
:10477000834207F10107F6D8E7E70027F5E72F2185
:10478000484606F023FEBDE70027BBE7489C002013
:10479000BC7B0408784E0408674E0408515A002078
:1047A000024BD3F8A80824F0C5B900BF0C2900209B
:1047B0000A4C08B505460A4806F004FDD4F8AC08D2
:1047C00018F012FED4F8A8081CF0BEFD08F02EF870
:1047D0000DB11AF09FFD1AF017FF00BF0C29002041
:1047E000984E04080A4D0B4808B507F0F1F9D5F8C2
:1047F000AC0818F0F9FD084B002485F8B048C5F85E
:10480000B0491C7008F052F92046FFF7D1FF00BFF5
:104810000C290020A44E0408305D0020044808B58F
:1048200007F0D6F9F4F730F80020FFF7C1FF00BF1A
:10483000CB4E0408034808B507F0CAF90120FFF77A
:10484000B7FF00BFD24E040870B506462AF07AFDC5
:10485000124C054690B11122002120462BF0C8FED3
:104860002A460F4930462BF0EFFE38B1102D2A466C
:10487000314628BF102220462BF0F8FE2378074A45
:10488000002B08BF0121064B1CBF0021134601204D
:10489000044ABDE8704006F001BE00BFBA6F0020B8
:1048A000767C0408F04E04082DE9F04188B080467B
:1048B00006F000FC074608B33E4CDFF804810025F3
:1048C00019274FF46176237917FB03630493E37888
:1048D00017FB03630393A37802936378019314F89F
:1048E000053B009342462B4600210120013506F08E
:1048F000D5FD0A2DE7D108B0BDE8F08140462BF088
:1049000059FD092805464FDC8400261808F10100EE
:104910008DF81F7006F0D6FB074660B12BF04AFDFC
:104920000D2808D8244B334483F8B4099DF81F3070
:1049300001338DF81F30384606F0C4FB074670B1CE
:104940002BF038FD431E042B09D81B4B621913446E
:1049500083F8B5099DF81F3001338DF81F303846B4
:1049600006F0B0FB074670B12BF024FD431E072B69
:1049700009D8114B2C441C449DF81F3084F8B6090B
:1049800001338DF81F300B4CF11C0DF11F02214437
:10499000384606F0A4FB9DF81F30052BABD0A219BA
:1049A0000023A3511371A6E709223946034806F0F4
:1049B0001AFDA0E7C03200200C2900200E4F040889
:1049C000F84E04082DE9F341074606F073FB06464E
:1049D00038B100223949012006F072FD02B0BDE86D
:1049E000F08138462BF0E6FC0E2804465FDC0625F5
:1049F0004543781C8DF8076006F064FB304F06468F
:104A000058B12BF0D7FC032807D87B1983F8EC09A1
:104A10009DF8073001338DF80730304606F052FB21
:104A2000804668B12BF0C6FC0D2809D8062303FB8D
:104A3000047383F8E7099DF8073001338DF80730D8
:104A40001E4E691C0DF107023144404606F047FB3B
:104A500006F038FB804668B12BF0ACFC1C2809D866
:104A6000062303FB047383F8EA099DF8073001333A
:104A70008DF80730404606F025FB68B12BF09AFC14
:104A80000D2809D8062303FB04749DF8073084F829
:104A9000EB0901338DF807309DF80730062B9DD0C8
:104AA000721900237351938006F0D8FE96E70E2208
:104AB0003146044806F097FC90E700BFF33200202F
:104AC0000C2900200E4F0408F8B5164D1648174F54
:104AD00006F0BEFED5F8AC0818F086FC1BF05AF9BB
:104AE00000241BF01DF9064648B113201DF0D2F931
:104AF00006F0E7FB0E48BDE8F84006F0A9BE3846D0
:104B000006F041FB782C08D80134D5F8AC0818F031
:104B10006BFC6420F8F754F8E3E706F0D2FB344668
:104B2000F3E700BF0C290020144F04085480040848
:104B30002E4F04087FB5084C19F02AFDD4E9015620
:104B400062880092CDE90160A389218803482A4642
:104B500006F03CFC04B070BD98220020344F0408DD
:104B60007FB5054606F0A6FA044630B10022184982
:104B70000120FEF7B9FE04B070BD28466A4615490B
:104B8000144E2BF050FC01AD78B1032C02D106F08D
:104B900065FEF0E72BF00EFC6A4645F8240031462E
:104BA00000202BF040FC0134EEE7032CEFD1DDE9CF
:104BB0000145039E29463246E0B215F047FE002823
:104BC000E5D033462A462146034806F0FFFBD2E7EC
:104BD000885B0020BC7B04086449040870B5064665
:104BE00006F068FA044630B1002210490120BDE801
:104BF0007040FEF7F5BE30462BF0DCFB0F28054673
:104C00000BDC304606F05EFA0146284615F046FEFB
:104C100050B9BDE8704006F021BE21460F2204487D
:104C2000BDE8704006F0DFBB70BD00BF085C00202F
:104C30000E4F04082DE9F04FDFF868808FB007466B
:104C40008A46164600240DF124095AF824300293AE
:104C5000494602A82AF044F916B356F82430029DBA
:104C60000393EB1A5D420DF1100B5D41594603A809
:104C70002AF036F9CDF800B0234642462946384698
:104C800006F0F6FB2346CDF800904246294638460A
:104C9000013406F003FC202CD7D10FB0BDE8F08F13
:104CA0003546EFE78F4F040870B5064606F002FA66
:104CB000044628B100220F490120BDE87040B9E741
:104CC00030462BF077FB1F2805460BDC304606F0FC
:104CD000F9F90146284615F0A5FC50B9BDE8704029
:104CE00006F0BCBD21461F220348BDE8704006F017
:104CF0007ABB70BD885B00200E4F04082DE9F04F91
:104D00002DED088BDFF80C9193B0804692460D464E
:104D10001446002695ED008AB5EE408AF1EE10FAB1
:104D200070D0D5ED019A95ED029AD5ED038ABAF1CE
:104D3000000F3ED094ED000A94ED01BAD4ED02AA22
:104D400094ED03AAB4EE408AF1EE10FA5FD1F4EECE
:104D50004B9AF1EE10FA5AD1B4EE6A9AF1EE10FACB
:104D600055D1F4EE4A8AF1EE10FA0CBF0127002764
:104D70000FA818F009FDB0EE4B0A83460CA818F0F6
:104D800003FDB0EE6A0A059009A818F0FDFCB0EE2C
:104D90004A0A049006A818F0F7FC059B049A0390B1
:104DA0000292CDE900B34A4633463946404606F002
:104DB0005FFBB0EE480A0FA818F0E6FCB0EE690AF7
:104DC00007460CA818F0E0FCB0EE490A834609A893
:104DD00018F0DAFCB0EE680A049006A818F0D4FCCB
:104DE000049B0390CDE901B3009733464A46002166
:104DF0004046013606F052FB082E05F1100504F17D
:104E0000100487D113B0BDEC088BBDE8F08F0027EC
:104E1000AEE700BF994F04087F2810B5044607D9B4
:104E200064F07F00C0B2E40924F0F8FF7F2CF7D8CB
:104E3000E0B2BDE8104024F0F1BF00BF38B5194D15
:104E40000446472024F0EAFFD5F8443A1B0305D571
:104E5000D5F8A4331868201AFFF7DEFF124C207D26
:104E6000FFF7DAFFD5F8483A2068C01A25F0BEF8F7
:104E7000D5F84C3A6068C01A25F0B8F82089FFF7D9
:104E8000CBFFE089FFF7C8FF208AFFF7C5FFD4E911
:104E90000023217D85F8581AC5F8502AC5F8543AE0
:104EA00038BD00BF0C29002018A90020F0B52B4CFC
:104EB0002B4DD4F8687AD4F86C6A2A492A48D4F879
:104EC0005C3A94F8642A2D78097890F82000B7426B
:104ED00085B027DB84F8745AC4F8703A84F8750AF0
:104EE00084F8761A84F8772A01AD532024F096FFCF
:104EF000D4F8700AFFF790FF94F8740AFFF78CFF5C
:104F000094F8751A94F8762A94F8773A0393284619
:104F1000CDE9011224F0B6FF0023C4F8683A01205D
:104F200005B0F0BDD4F8706A8DF80850B3428DF822
:104F30000B2001938DF809008DF80A1001AD04F5DE
:104F4000276204D095E8030082E80300CDE7696892
:104F500053689942F6D10020E2E700BF0C290020F7
:104F60009C5E0020065D0020A85E00201E4A1F4BAC
:104F7000116800221F29C3F8782AA3F87C2AA3F815
:104F80007E2AA3F8802AC3F8682A23D03F291CD0A0
:104F90004FF4FA42B2FBF1F1A3F8821A1448B3F9C4
:104FA000822A018829B1914201DD1F2A17DC92FB78
:104FB000F1F1A3F8841A81780E48003118BF01215D
:104FC0001202C3F86C2A017070474FF40072A3F804
:104FD000822AE3E74FF48062A3F8822ADEE7012108
:104FE000A3F8841AE7E700BF389A00200C290020B4
:104FF000E46F0020E6800020084B10B5B3F9824A28
:10500000B3F9841A204618F0DDFF054B1B88C0B2A7
:1050100000FB03F090FBF4F0C0B210BD0C2900209F
:10502000E46F00202DE9F04F7B4CB4F87C3A8DB052
:105030000746002B40F0FE80784D2B88002B00F0B7
:10504000A3803846FCF71EFDD4F8A07349203E46E5
:1050500024F0E4FED4F8780AFFF7DEFE56F8040BDD
:10506000FFF7DAFE304629F005FF07F1100029F0BE
:1050700001FFD4F8443ADB0300F1A280D4F8443AAB
:105080009E0300F19480D4F8443A580300F1BF80A5
:10509000032107F1280024F09BFF614BB7F92E0094
:1050A0001B8AC01AFFF7B8FED4F8443AD90400F1BD
:1050B0009F809A0400F192801E0400F18A8007F11B
:1050C0003000032124F084FFD4F8443AD80264D499
:1050D00099025CD4B7F9443007EE903A514BF8EEA0
:1050E000E77A93ED007A77EEC77AFCEEE77A17EE6F
:1050F000900AFFF791FE4C4B1B78012B0ED907F15C
:10510000440808EB430807F1460636F9020BB7F9E5
:105110004430C01A24F06AFFB045F6D1D4F8443ABE
:105120009A052AD4D4F8A0034049C4F8A403431A2A
:105130009B1003EBC30203EB4203C3EB432303EBDC
:1051400083433B4AC4F8A803C3F1010382FB030273
:10515000A2EBE37202EB42029B1A6C2202FB0313E6
:105160000122C4F8A03384F8D02BAB78012B01D1F5
:105170001AF0A8FF0DB0BDE8F08FB7F95E00A0F2FD
:10518000DC5024F033FFCDE7FFF790FE59E7042110
:1051900007F13C0024F01CFF9CE7032107F13600D7
:1051A00024F016FFD4F8443A990293D5EFE7386A11
:1051B00024F01CFFD4F8443A58037FF569AF26E089
:1051C000F86924F013FFD4F8443A9E037FF55BAFEF
:1051D000EDE7B7F86800FFF71FFE70E7B7F8660065
:1051E000FFF71AFED4F8443A1E047FF568AFF0E7E3
:1051F000B7F86430B4F8860AC01AC0F30D00FFF7A0
:105200000BFED4F8443A9A047FF556AFE6E7786A85
:1052100024F0ECFE3CE700BF0C290020E46F0020E6
:10522000489C002094330020515A002098330020DD
:1052300056555555D4F8D45BD4F8D83BAB4207D07B
:10524000CD4BC4F8D85B1B78093B012B40F2B181F0
:10525000D4F8DC6BD4F85C5AAE4207D0C64BC4F825
:10526000DC5B1B78093B012B40F29681B4F8803A55
:10527000C24D002B40F0DD802B88002B00F0D98040
:10528000FFF714FE3846FCF7FDFBD4F8A463D4F80E
:10529000A0A30196502024F0C1FDD4F8A033D4F887
:1052A000A823D4F8A41312681B6808681344A3EB5E
:1052B00040000DF1100824F099FE321D0AF104019E
:1052C000404629F0EFFA404629F0D4FD06F11002DD
:1052D0000AF11001404629F0E5FA404624F0D2FDDB
:1052E00010264FF00109D4F8443A09FA06F21A429E
:1052F00040F0EA800136132EF5D1019B0AF1280116
:1053000003F12806C3460AF1300E404631F9023B4C
:1053100036F902CB8E45A3EB0C0340F8043BF5D1E4
:1053200008A9002651F8043DB60003F10800F6B2C2
:1053300033B10F2803F1800300F2BF8046F001066D
:105340008845EFD1304624F069FD0023994619467F
:1053500006F00300022800F0A480032800F09080EB
:10536000012800F0848009F10109B9F1040F4FEA26
:105370009606EDD1002940F07B81D4F8443A03F43D
:10538000005003F40041DB0400F1CA80002840F023
:105390001A8161B1019ABAF86830B2F868209B1A94
:1053A0000493049BD81780EA4300FFF735FD0321DF
:1053B0003020FCF745FBD4F8443ADE0200F151817D
:1053C000980200F149816E4B44201978FCF738FBB4
:1053D000D4F8443A990507D5019BBAF95E00B3F9B0
:1053E0005E30C01A24F002FED4F8A0136548664A65
:1053F0000B1A9B1003EBC30603EB4603C3EB4323DB
:1054000003EB8343C3F1010382FB0362A2EBE3726C
:1054100002EB42029B1A6C2202FB0303C4F8A03386
:10542000D4F8A423C4F8A8230123C4F8A41384F84F
:10543000D03B564B1B681A067FF597AE544ED4F8F6
:10544000483A32689A424CD0482024F0E7FC306851
:1054500024F0CCFD706824F0C9FDD6E9002338465D
:10546000C4F8482AC4F84C3AFFF7E8FC7DE658F83F
:105470002920002940F0E7801301DBB2014672E7E2
:1054800058F8290000295FD1C0F30720CDE90213A5
:1054900024F0C4FC18F8290024F0C0FCDDE9021354
:1054A00061E758F82900002960D1C0B2CDE90213A4
:1054B00024F0B4FCDDE9021355E7FF2B94BF46F05E
:1054C000020646F003063BE70199B3000AEB03022C
:1054D0000B4452F8240C53F8243CC01A24F086FDE7
:1054E00008E77268D4F84C3A9A42ADD1B4F9823ADE
:1054F000B4F8802A03EBD373B2EB630F00F0C380E0
:10550000244B94F8582A197D914205D11968D4F892
:10551000502A914200F0B0803846FFF78FFC24E615
:10552000019ABAF86430B2F864609B1B04930028B7
:105530007ED100293FF436AFBAF86830B2F868106F
:105540005B1A0593022655E0C0F30330184302911D
:1055500024F064FC58F82900C0F3071024F05EFC26
:1055600058F8293002991B01DBB2FCE6C0F30310A6
:1055700002911843F2E700BFE6800020E46F0020AC
:10558000515A00209833002056555555489A00200E
:105590000084002018A90020452024F03FFC1E2094
:1055A00024F03CFC2846FFF737FC3046FFF734FC7C
:1055B0005CE6452024F032FC002024F02FFC284635
:1055C000FFF72AFC44E6019ABAF86630B2F86600A2
:1055D0001B1A0493012600293FF4E3AE019ABAF89E
:1055E0006830B2F868000CAA02EB86011B1A41F879
:1055F000203C0136B60008EB0603002053F8041DDA
:105600004000C0B209B140F001009845F6D124F045
:1056100005FCB04402E0D8453FF4C9AE5BF8043B5A
:10562000002BF8D0D81780EA4300FFF7F5FBF2E72C
:10563000019ABAF86630B2F866001B1A0593022682
:105640000029D7D0CAE702F00F001843029324F0D4
:10565000E5FB0021029B86E604213C20FCF7F0F9E3
:10566000B1E603213620FCF7EBF9D4F8443AA7E67B
:10567000184624F0D3FB80E65A68D4F8543A9A428C
:105680007FF44AAF71E5B4F87E3A5B063FF4DCAED6
:1056900036E700BF194BB3F87C2AD3F8680AD3F871
:1056A000781A10B40132B3F9824A92B20130013152
:1056B000A242C3F8680AC3F8781AA3F87C2A0FDA62
:1056C000B3F8802AB3F9841A5DF8044B013292B220
:1056D0008A42A3F8802AA4BF0022A3F8802A704738
:1056E000B3F87E2A5DF8044B00210132A3F87E2A2C
:1056F000A3F87C1AA3F8801A704700BF0C29002079
:10570000F0B5A34C04F688238FB093ED000A2BF07C
:105710004BF904F53E6393ED000A05462BF044F97E
:105720000646402024F086FA002853D1994AD4F83E
:10573000E43B57784A2B00F24284DFE813F0DC03A5
:10574000CE03C403B003A7039D038A0380030304AD
:10575000F903EF03E50313040D041D0476036F033F
:1057600065035B03510346033A032E03220313032D
:105770000403F502E7029C028E02800272026402B8
:10578000560248023D022F02230218020D020202B5
:10579000F701EB01DF01D301C801BD01B101A50192
:1057A0009A018F01840179016F0165011E011401C5
:1057B0000A01FF00F400DE00D400CA00C000B600F9
:1057C000AC00A10097008D00830079006F00650098
:1057D0005C004E0000200FB0F0BD6F4B6F491A689F
:1057E0006F48FCF701F9D4F8E43B01330020C4F81A
:1057F000E43B0FB0F0BD927868496A48FCF7F4F8D2
:10580000D4F8E43B0133F1E7674B6449DA89674830
:10581000FCF7EAF8D4F8E43B0133E7E7624B5F4971
:105820001A886348FCF7E0F8D4F8E43B0133DDE77D
:105830005D4B5A499A785F48FCF7D6F8D4F8E43BB8
:105840000133D3E7584B55491A795B48FCF7CCF83C
:10585000D4F8E43B0133C9E7584B50491A7A584809
:10586000FCF7C2F8D4F8E43B0133BFE7534B4B4994
:105870005A8C5448FCF7B8F8D4F8E43B0133B5E748
:105880004E4B464993F820204F48FCF7ADF8D4F82A
:10589000E43B0133AAE7494B40499A7F4B48FCF768
:1058A000A3F8D4F8E43B0133A0E794F8082C3B4973
:1058B0004748FCF799F8D4F8E43B013396E794F8AD
:1058C000FB2B36494348FCF78FF8D4F8E43B01330F
:1058D0008CE7414B31495A794048FCF785F8D4F8B8
:1058E000E43B013382E794F803242C493C48FCF75D
:1058F0007BF8D4F8E43B013378E7B4F800349FED4B
:10590000397A2649384807EE903AF8EEE77A67EE9A
:10591000877AFDEEE77A17EE902AFCF765F8D4F85F
:10592000E43B013362E7314A3149138A31489289B5
:10593000FCF75AF8D4F8E43B013357E72B4A2C49DB
:10594000D3892D485289FCF74FF8D4F8E43B013352
:105950004CE7264B11495A792848FCF745F8D4F80A
:10596000E43B013342E7214B0C491A792448FCF708
:105970003BF8D4F8E43B013338E71C4B0749DA78AD
:105980002048FCF731F8D4F8E43B01332EE700BFA0
:105990000C290020EC900020FC82002007780408ED
:1059A000C8570408BC570408489C0020A85704089E
:1059B0009857040884570408705704083C90002046
:1059C0005C5704084057040824570408105704087B
:1059D000F8560408E856040884710020D8560408D4
:1059E000C85604080000C842BC5604081C9A00208F
:1059F000F4530408A8560408985604088856040866
:105A0000745604086856040894F8F12BA149A2487A
:105A1000FBF7EAFFD4F8E43B0133E7E694F8F02B18
:105A20009C499E48FBF7E0FFD4F8E43B0133DDE6F8
:105A30009B4B98491B689B485A8DFBF7D5FFD4F8C0
:105A4000E43B0133D2E6964B92491B6896481A8D87
:105A5000FBF7CAFFD4F8E43B0133C7E6904B8D490E
:105A60001B6892485A8FFBF7BFFFD4F8E43B013321
:105A7000BCE68B4B87491B688D481A8FFBF7B4FF38
:105A8000D4F8E43B0133B1E6854B82491B68894871
:105A900093F83720FBF7A8FFD4F8E43B0133A5E6E1
:105AA0007F4B7C491B68844893F83620FBF79CFFAA
:105AB000D4F8E43B013399E6794B76491B687F487B
:105AC0009A8EFBF791FFD4F8E43B01338EE6744BDA
:105AD00070491B687A485A8EFBF786FFD4F8E43B7E
:105AE000013383E66E4B6B491B68764893F82D2093
:105AF000FBF77AFFD4F8E43B013377E6684B65495E
:105B00001B68714893F82C20FBF76EFFD4F8E43B38
:105B100001336BE6624B5F491B686C4893F82720A2
:105B2000FBF762FFD4F8E43B01335FE65C4B594975
:105B30001B6867489A8CFBF757FFD4F8E43B0133A6
:105B400054E6574B53491B6862485A8CFBF74CFF8D
:105B5000D4F8E43B013349E6514B4E491B685E489B
:105B6000DA8BFBF741FFD4F8E43B01333EE64C4BC4
:105B700048491B6859481A8CFBF736FFD4F8E43BB8
:105B8000013333E6464B43491B68554893F82620BA
:105B9000FBF72AFFD4F8E43B013327E6404B514999
:105BA0001D6851482B7FEA7E6D7F0095FBF71CFF37
:105BB000D4F8E43B013319E6394B36491B684B48AE
:105BC0001A7EFBF711FFD4F8E43B01330EE6344BA9
:105BD00044491D684648AB7D6A7DED7D0095FBF725
:105BE00003FFD4F8E43B013300E62D4B3D491D682B
:105BF0004048EB7CAA7C2D7D0095FBF7F5FED4F8A0
:105C0000E43B0133F2E5264B36491D683A482B7CCC
:105C1000EA7B6D7C0095FBF7E7FED4F8E43B0133AB
:105C2000E4E51F4B2F491D6834486B7B2A7BAD7B15
:105C30000095FBF7D9FED4F8E43B0133D6E5184BC9
:105C400028491D682E48AB7A6A7AED7A0095FBF7F1
:105C5000CBFED4F8E43B0133C8E5114B21491D6864
:105C60002848EB79AA792D7A0095FBF7BDFED4F888
:105C7000E43B0133BAE50A4B1A491D6822482B79E7
:105C8000EA786D790095FBF7AFFED4F8E43B013379
:105C9000ACE500BF07780408585604085C560408B1
:105CA0005461002044560408345604082856040859
:105CB0001856040800560408E4550408D055040892
:105CC000B8550408A45504089455040884550408DC
:105CD00070550408605504085455040844550408D8
:105CE00030550408B0540408285504082055040809
:105CF000145504080C55040804550408FC54040801
:105D0000F4540408EC540408E0540408AD4BAE49C4
:105D10001D68AE486B782A78AD780095FBF764FE75
:105D2000D4F8E43B013361E5A94BA749A94803EB4B
:105D30000717FD7ABB7A7A7A0095FBF755FED4F8FF
:105D4000E43B013352E5A24B9F49A34803EB0717FD
:105D50003D7AFB79BA790095FBF746FED4F8E43B2F
:105D6000013343E59A4B98499C4803EB07177D792B
:105D70003B79FA780095FBF737FED4F8E43B013322
:105D800034E5934B9649974803EB0717FA89FBF7DD
:105D90002BFED4F8E43B013328E58D4B9049924823
:105DA00003EB07173A7BFBF71FFED4F8E43B013304
:105DB0001CE5874B8A498D4803EB07177A78FBF778
:105DC00013FED4F8E43B013310E5814B8449884845
:105DD0003F01DA5DFBF708FED4F8E43B013305E54B
:105DE00094F816287E498348FBF7FEFDD4F8E43B7F
:105DF0000133FBE4804B7A499A788048FBF7F4FD45
:105E0000D4F8E43B0133F1E47D4B75491A687D48D1
:105E1000FBF7EAFDD4F8E43B0133E7E47A4B9B79E6
:105E2000012B00F0C0801123E0E4B4F8862A774902
:105E30007748FBF7D9FDD4F8E43B0133D6E4754B42
:105E400067491A887448FBF7CFFDD4F8E43B013367
:105E5000CCE4FFF7D1F8B4F9841A0546B4F9820A04
:105E600018F0B0F82A46C3B26C496D48FBF7BCFD88
:105E7000D4F8E43B0133B9E4B4F9822A58496948BB
:105E8000FBF7B2FDD4F8E43B0133AFE4664A67495F
:105E90006748FBF7A9FDD4F8E43B0133A6E403A867
:105EA00017F054FD634B03A9B3F9002006A80023A3
:105EB00017F058FF06AA5D495F48FBF795FDD4F837
:105EC000E43B013392E45D4B5D4A5E495E48FBF77B
:105ED0008BFDD4F8E43B013388E45C4A5C4B5D49BC
:105EE0005D48CDE900325D4B5D4AFBF77DFDD4F89E
:105EF000E43B01337AE45B4A4C495B48FBF774FDB1
:105F0000D4F8E43B013371E4B3B2AAB2574958481C
:105F1000FBF76AFDD4F8E43B013367E44FF07E52AF
:105F200054495548FBF760FDD4F8E43B01335DE488
:105F3000524B2B495A8A5248FBF756FDD4F8E43BA2
:105F4000013353E44D4B26491A8A4E48FBF74CFD6A
:105F5000D4F8E43B013349E4D4F8443ADB0418D4E0
:105F6000102343E4484B29499A8A4848FBF73CFDF3
:105F7000D4F8E43B013339E4234845498378427837
:105F8000007800904348FBF72FFDD4F8E43B013341
:105F90002CE4414B1D491A784048FBF725FDD4F805
:105FA000E43B013322E4B4F9EC3BB4F9EE2B2F4986
:105FB0003B48FBF719FDD4F8E43B013316E401201C
:105FC00009E400BF54610020B0540408D854040808
:105FD000A4800020D0540408C8540408BC54040809
:105FE00007780408A054040894540408885404084A
:105FF000805404086C5404081C9A00205C54040863
:10600000389A002050540408705B0020D48A040899
:1060100038540408E46F0020C0530408AC5304084B
:10602000B4530408A0530408BA6F002017490408A9
:10603000945304080463002080530408E9490408C9
:10604000F249040868530408705304089B49040883
:10605000DF4904084453040854530408FE49040863
:10606000A44904082853040834530408F4530408CA
:10607000FC530408E0530408E8530408489C00203B
:10608000D4530408C85304085C5D00200854040875
:106090001C540408285404087F7F0020105404086E
:1060A000405404082DE9F04F5F4D85B0D5F8E84B1A
:1060B0000193904600290CBF04230623621CDDF8DF
:1060C00038900F9F029367D0A14544DDDFF86CA1A3
:1060D00057B1109BDA1B04FB02F20123B95CD5F81F
:1060E000442A8B4013422FD0019BD5F8E42BA3EB1D
:1060F000080304FB03F408EB0406002A37D158F820
:10610000040029F01FF900F1050B584623F092FD19
:10611000A0BBDAF8000095F80B2CA0EB0B00CAF836
:106120000000002A34D1012385F80B3CD5F8E43B6C
:1061300043BB58F8040023F0E3FD96F904104B1C10
:1061400002D03A48FBF73EFCD5F8E84B01344C4509
:10615000C5F8E84BBCDBA1454FD0D5F8E40B029B5A
:10616000834294BF0020012005B0BDE8F08F4FF0BE
:10617000030B584623F05EFD0028CAD0012005B06D
:10618000BDE8F08F1E442A483179FBF71BFCDBE7A2
:106190002C2023F043FEC9E7D5F8E43B029A934252
:1061A00003D3002005B0BDE8F08F224C039104EB2F
:1061B00083030646D3F88C0429F0C4F80B3023F08F
:1061C00039FD039982460028D8D1D5F8E43B1A4816
:1061D00004EB8304032B98BF3146D4F88C24FBF7DF
:1061E000F1FB164AD5F8E84B136885F80BAC1B1A7F
:1061F00001341360C5F8E84B66E7012023F01AFD6F
:106200000028AAD10D4A13680A20013B136023F02D
:1062100005FED5F8E40B4FF0FF330130C5F8E40B71
:10622000C5F8E83B9BE700BF0C290020E4570408B1
:1062300007780408FC220408D4570408A885002025
:106240002DE9F04F974CA378012B87B000F0A9807F
:10625000032B18BF03234FF0800018BFA3701BF05F
:106260001DFD0746002800F0A48080211BF00CFDD6
:106270007E798D4B97F902C053F826208B4DB2F5ED
:10628000613F14BF002702270023022185F80C0C70
:106290000092CDE901171A46604680211BF03AF9B9
:1062A0000C3E834B032E186000F2E980814B4022A4
:1062B0001A7000287DD0804B804993F815E0804A01
:1062C000804B0F68E678116898797F4A93F80590BB
:1062D000DFF80CA292F8008095F8182C7B4BB4F8EC
:1062E00000C0BAF80240DFF8FCB1A5F8864ABEF15A
:1062F000000FC7F3C03718BF0127003618BF0126AB
:1063000011F0020F08BF0026002110F0FD0F14BF8E
:106310004FF0010A8A46B9EB0109A2F1190E18BF24
:106320004FF00109B8EB010803F144046848C5F8CF
:10633000481A18BF4FF00108BEFA8EFE012A4FEA34
:106340005E1E03F1B00208BF4FF0010EC5F8A04376
:106350001CF1FF3C03F58E74C3E90111C3E903117D
:10636000DBF80030C5F8A423C5F8A84390F800B0C6
:10637000049318BF4FF0010C0A460C460120059506
:10638000D3B2591E15291CD8DFE801F03434343457
:1063900034343434301E1E28241E4A3E3E3E5219E8
:1063A0002C1E4C4B9B6823B1404DD5F8142C9342C6
:1063B0003AD8494B00221A7007B0BDE8F08F314639
:1063C00031B100FA02F10C430133DBB2162B33D8A2
:1063D0000132D5E751460029F3D1F9E749460029B2
:1063E000EFD1F5E741460029EBD1F1E771460029ED
:1063F000E7D1EDE79B4534BF002101210029E3D01F
:1064000000FA02F10C43DFE7049D02EB420129444C
:1064100011F82E1C003118BF01210029F0D1D3E75B
:1064200039460029CDD1D3E7224B40221A7042E7EA
:1064300061460029C5D1CBE7059D1A20C5F8444A1D
:1064400006F0C6FB244CD5F8D41BD5F85C2A85F899
:106450001A0C002302202070C5F8783AA5F87C3A7F
:10646000A5F87E3AA5F8803AC5F8683A85F8D03B99
:10647000C5F8D81BC5F8DC2B07B0BDE8F08FD5F800
:10648000103C164A03EB4303A2FB03235B0906D02F
:10649000402BA8BF4023DBB2064A137009E7012353
:1064A000FAE700BFE46F00200C3404080C29002038
:1064B000AC850020B08500203C900020489A002048
:1064C0009C5D0020705B00209587002054330020E5
:1064D000515A002098220020E6800020D34D6210FF
:1064E000445D00205461002008B5084B9B78032BC5
:1064F00006D0FFF7A5FE064B012283F81B2C08BD32
:10650000802028F021FB0028F3D008BDE46F002094
:106510000C29002038B5FBF7B1FB054618B1094B33
:106520001868FBF73BFB09241AF05CF80028FBD144
:106530001AF058F818B1013CF6D1284638BD1AF0C7
:1065400031FAF8E7389A002070B502392DED048B46
:10655000D0E90023856806290CD8DFE801F04C5209
:10656000575D626A040059425342C0E900136D420C
:106570000A4685603149097FD1BB314E07EE903A1A
:1065800006EE902AB8EEE78A96ED030A96ED007AB9
:10659000D6ED067AF8EEE68A28EE000A06EE905A64
:1065A000A7EE280A0446B8EEE69AA7EE890A2AF072
:1065B000FBF996ED040A96ED017AD6ED077A206094
:1065C00028EE000AA8EE870AA9EE270A2AF0ECF9BD
:1065D00096ED050A96ED027AD6ED087A606028EE0F
:1065E000000AA8EE870AA9EE270A2AF0DDF9A060C2
:1065F000BDEC048B70BD5142C0E900311A460B4618
:10660000B8E752425B42C0E90023B3E75942C0E910
:10661000001213460A46ADE752426D4202608560A1
:10662000A8E711466D42C0E9012503601A460B46F2
:10663000A0E75B426D42C0E901359BE7780000208E
:1066400028350020944B954A596AB2F80034A2F8D4
:106650001034002900F00D8107EE903AB8EE676A19
:1066600007EE901AF8EE677A9FED8D7A9FED8D0A0E
:10667000DFED8D2A9FED8D3A9FED8D1ADFED8D1A9E
:106680009FED8D2A9FED8D5A26EE276AF0EE400A87
:1066900026EE076A2DED028BFDEEC67A36EE000A75
:1066A00017EE900AFDEEC07A02F2144317EE901A2C
:1066B0002030203102F59062F7EE004A402800F2C7
:1066C000A580B4EEE26AF1EE10FA40F3DC80B0EEA1
:1066D000467ADFED7B5ADFED7B6A01E0B0EE677A48
:1066E000B4EEE67AF1EE10FA77EE657AF6DCF4EEC7
:1066F000C37AF1EE10FA40F1BD80DFED715ADFEDA3
:10670000726A01E0F0EE477AF4EEE67AF1EE10FA02
:1067100037EEA57AF6D4B4EEE07AF1EE10FA00F393
:10672000A280DFED6A7AB4EEE77AF1EE10FA48BFA4
:1067300033EE477A67EE077AB0EE614AA7EE814AF8
:106740004029F0EE423AE7EE843A67EE275ADFED51
:10675000606AA5EEA37AB0EE644AF0EE647AA7EE22
:10676000264AE7EE667AC7EE843A55D8B4EEE06A78
:10677000F1EE10FA40F38A80B0EE407ADFED505A25
:10678000DFED506A01E0B0EE677AB4EEE67AF1EE42
:1067900010FA77EE657AF6DCF4EEC37AF1EE10FAD1
:1067A00077D5DFED475ADFED486A01E0F0EE477A32
:1067B000F4EEE67AF1EE10FA37EEA57AF6D4B4EEFE
:1067C000E07AF1EE10FA51DCDFED407AB4EEE77AD0
:1067D000F1EE10FA48BF33EE477A67EE077AF0EE33
:1067E000616AE7EE816AF0EE428AE7EEA68A67EE1A
:1067F000275AB8EE008AA5EEA87AF6EE006A74EE83
:10680000C75A27EE087A65EEA66A0BE0F7EE003A63
:106810004029B0EE634AA9D9B0EE457AF6EE006A97
:10682000F7EE005AC4EE847A243343ED053A67EE5E
:10683000A66A67EEA55A27EE877A43ED096A43ED0B
:10684000076A43ED085A03ED067A03ED035A03ED98
:10685000045A03ED015A03ED025A9A427FF42EAF17
:10686000BDEC028B704732EEC77A63E732EEC77A2F
:10687000B3E77047B0EE677AB4EEE07AF1EE10FA63
:106880007FF74FAFEFE7F0EE467A30E7F0EE407A71
:1068900082E7B0EE677A92E75C5D00200C29002069
:1068A00027D4D236DB0FC93FDB0F4940DB0F49C08D
:1068B00092E741B99730083C15A82ABE00000000B5
:1068C000DB0FC940E4CB1641E4CB16C1DB0FC9BFD7
:1068D000F304353F254B5B68C3F3080370B4B3B9C9
:1068E000EFF311839BB9224A224C1368A06800BFC2
:1068F00011688B42F9D120490D684FF47A7404FB7A
:1069000005F1081AB0FBF5F004FB03031FE0EFF3F9
:106910001180102383F31288164A1849956813686A
:10692000DB0342BF01230B609568114AC0B21668B1
:106930000B6880F3118810490C684FF47A70334467
:1069400000FB04F1491BB1FBF4F100FB03130C48FD
:106950000C49126882600124022280F8214081F8EB
:10696000442CC1F8403C70BC704700BF00ED00E013
:10697000D490002010E000E0D8900020D0900020BB
:10698000A85E00200C290020274B5B68C3F3080396
:1069900030B4B3B9EFF311839BB9244A244C136884
:1069A000A06800BF11688B42F9D1224A14684FF4E5
:1069B0007A7101FB04F2101AB0FBF4F001FB03033F
:1069C00020E0EFF31181102383F3128818481A4A4C
:1069D00084680368DB0344BF01231360134B48BF83
:1069E00084681D681368C9B281F31188114A106860
:1069F0004FF47A712B4401FB00F2121BB2FBF0F250
:106A000001FB03230D490E488A68022403F5B713DE
:106A100003F5587302F2DC5280F8444CC0F8403C55
:106A20008A6030BC704700BF00ED00E0D4900020C9
:106A300010E000E0D8900020D0900020A85E002058
:106A40000C2900202DE9F0478B4D8C4C8C4B288B6A
:106A50008C4A8D4F8D4EC4F84C32DFF868E2C4F892
:106A60007072002384B00FFA80F984F8453CC4F8B2
:106A7000746204F6444102F1240CDEF8003022F87E
:106A8000029F03F59673944541F8043FF5D1DFF872
:106A90003882DFF838E2D8F800C07D4B1CF4805F04
:106AA00008BFB5F92490AEF8069003F164010AE03E
:106AB0001FFA89F293F8019009F104092EF81920C0
:106AC000053399421AD01A78002AF9D193F802A016
:106AD000DA789245F4D20AF1FF3909EB890909EB1A
:106AE000890909F561790132BAF1000FE0D102EBB1
:106AF000820202EB820202F56172DBE71CF0080FF2
:106B000032D11CF4804F41D11CF0010F0CF4005322
:106B100015D103BB1CF4004F22D16B7D13B10223AE
:106B200084F8A43795F8282094F86C12131D8B4232
:106B3000A8BF0B4684F8683D04B0BDE8F08744F672
:106B40002062A4F86E2293B30822524B84F86C2280
:106B5000C4F87032DEE744F62063A4F86E32F3E73F
:106B6000012384F8A437DDE72B7A0C2B26D8DFE845
:106B700013F0AF00AF007E024D02CD022E012E01B8
:106B80007201AE01EA01AF0025002F00122244F687
:106B90002063414984F86C22A4F86E323F4A404B8E
:106BA000C4F87012C4F87422C4F84C32ACE70C225A
:106BB0003C4B84F86C22C4F87032ABE7082016F026
:106BC000B7FCD8F800C0C4F87072C4F8746298E7D3
:106BD0000A220301344993FBF2F3344AC4F87022C9
:106BE000A3F5B063C4F878129BB2002221F81230EA
:106BF0000132122AFAD142F6F8212D4B84F86C2288
:106C00004020A4F86E12C4F874321BF047F8002834
:106C1000D4D0AB7A697A90F90200264A002B0CBFD7
:106C200000230823002918BF43F001034FF0030C91
:106C30004FF4E131CDE901C30091002340211AF066
:106C400069FCC4F89C07002800F0B8801A4B1A7839
:106C5000002A40F0E082194A1949116002221A7094
:106C6000012394F8A42784F8CC37002A40F0A680AA
:106C7000032384F8A437A1E03C9000200C290020D5
:106C8000A08601006E5E0020991501089D1501087F
:106C90009C35002035170108A1150108B115010820
:106CA000400D03002517010850360020090D01088A
:106CB000852401080501010803620020DC5A002038
:106CC00021240108D4900020489A0020705E002002
:106CD000B74BC4F8FC3740201AF0E0FF814600288B
:106CE0003FF46CAF4FF0000A84F8ECA713F0B6F94C
:106CF0002A7A012A03460FD0C0F0A7820A2A1FD1A0
:106D0000D8F8002012F480621CBF80F00102D2B2D9
:106D100002F0010284F8EC270321072284F8FA1715
:106D200084F8002801214FF4006284F89811C4F817
:106D3000F0270C2142F6F82284F86C12A4F86E2297
:106D4000697A9C489C4AC4F874220031C4F87002E5
:106D500018BF01214AB299F9020094F8ECC7002B40
:106D600040F03382BCF1000F40F0538295F80AC026
:106D7000BCF1000F00F09D82012342F008024FF4A5
:106D8000E131CDE90132009100238C4A40211AF013
:106D9000C1FB8B4B18606B7D94F86C22013BDBB21E
:106DA0009A4284F8ED379CBF002384F8ED3728B170
:106DB00094F8EC3713B1012384F8F43C031C18BF9A
:106DC0000123002B3FF4FAAED8F800C099E6062B59
:106DD0004FF00C0240F0C68184F8B63084F86C2283
:106DE000002384F8AC20DFF820922376212284F857
:106DF000B53084F8B43084F8AB2042F6F821714AFB
:106E0000714BA4F86E124020C4F87022C4F874329A
:106E10001AF044FF824600283FF4D0AE13F01EF96A
:106E2000697A9AF902C0AB7A003118BF01214AB2DF
:106E3000002800F0F281002B40F0648203220291CE
:106E40000192CDF800906046604A40211AF062FB42
:106E50005F4B1860B2E70E234FF0000944F6206143
:106E60005C4A84F86C3240205B4B84F85093A4F861
:106E70006E12C4F87022C4F874321AF00FFF0028A2
:106E80003FF49CAEB0F800C0697A90F90200AB7A8A
:106E9000B1EB09010CF4825C18BF0121BCF5825FE3
:106EA0004AB200F0F08184F84D93002B00F0A581E8
:106EB00042F008024FF0010C4FF4E1310292CDE9AB
:106EC000001C4B46454A40211AF024FB76E710206F
:106ED00041F27C534249434A84F86C024FF0000966
:106EE000A4F86E3240202823C4F87012C4F874222B
:106EF00084F83C9384F83D331AF0D0FE00283FF428
:106F00005DAEAA7A6B7A384990F9020000914A4541
:106F10000CBF4A4608224B4518BF42F0010203212C
:106F20004B46CDE90112314A40211AF0F3FA012112
:106F3000C4F8400DF6F716F8D4F8403DB3EB09035A
:106F400018BF01233DE72A490A23020192FBF3F20D
:106F50000023A2F5B06241F823200133102BFAD1AF
:106F600041F60B21234A84F86C324020224BA4F8CE
:106F70006E12C4F87022C4F874321AF08FFE002822
:106F80003FF41CAE6B7A1D4A90F902000092003368
:106F900018BF01230322CDE9012340210023184A11
:106FA0001AF0B8FA174A031C18BF0123106008E74B
:106FB000782B0020F50B0108E1280108250C0108B9
:106FC0009C620020DD000108F10001083505010880
:106FD000FC610020C9150108E92E0108E917010824
